:020000040800F2
:10000000F0FF0120592804082D1F0208FD82010875
:10001000E9280408E9280408E92804080000000089
:10002000000000000000000000000000811F020826
:100030007F1F0208000000007D1F020879F0010800
:10004000E9280408E9280408E9280408E92804083C
:10005000E9280408E9280408E99A0008159C000822
:10006000D99B00089D9B0008619B00081DC60008E5
:100070000DC60008FDC50008EDC50008D9C500087B
:10008000C5C50008B1C50008E92804080000000043
:10009000000000000000000000000000259B000898
:1000A00009890108F58C0108E9280408B58D0108C3
:1000B000358C0108758B0108A98A01086DE60008D6
:1000C00073E6000861E6000867E60008E92804080E
:1000D000E92804089DF1010801F101080000000071
:1000E000AF9A0008E92804082F1F0208000000004A
:1000F0000000000000000000000000009DC5000896
:1001000000000000E9280408D9890108E92804084A
:1001100000000000000000000000000000000000DF
:1001200089C5000875C5000861C500084DC50008EF
:1001300039C50008000000000000000000000000B9
:10014000000000000000000000000000952A0208E6
:1001500025C5000811C50008FDC40008E9280408E9
:1001600055E600085BE60008000000000000000003
:10017000000000000000000000000000000000007F
:1001800000000000E9280408000000000000000052
:08019000E9280408E92804082D
:08019800F02304000100000047
:1001A00010020100042B0020002B002000000000A2
:1001B000A00600080312330008360020403B002050
:1001C00000000000A406000825005A006C3A002038
:1001D000C63A00200000000000000000F6110C00EC
:1001E0004C380020FC39002000000000D806000830
:1001F00015007000583800208C39002000000000E5
:10020000000000002A006000C83800202C390020BF
:1002100000000000796702082C001000203B00203D
:10022000303B002000000000390501082B002400AD
:10023000973B0020733B00200000000009050108E7
:10024000290064006C370020083A002000000000FC
:10025000000000001400020068310020283900204E
:1002600000000000E40600081010020068360020BC
:10027000003C002000000000E606000828001000F6
:1002800058360020043C002000000000E1E7000890
:1002900023001000782F0020143C002000000000F4
:1002A000F9E700081900050050360020243C002022
:1002B00000000000E8060008F8210600C63400200F
:1002C0002C3C002000000000EE0600081B00F4009B
:1002D0008C4B002008600020000000007D7A03089D
:1002E0000E02020018530020FC60002000000000F5
:1002F000F40600082F001100CE5F002000610020EE
:1003000000000000F606000805100600FC5F002053
:10031000146100200000000008070008F5216E00AD
:10032000044B00201C61002000000000230502088F
:1003300026000E009C6100208C610020000000005F
:10034000F90402080B201000744B0020AC6100205F
:10035000000000000E0700081F101C00E44A0020E7
:10036000BC610020000000001E070008050201001B
:100370005C4F0020D8610020000000003A07000810
:1003800003010A002A4D0020DC610020000000006B
:100390003C0700080A020A00247100203471002082
:1003A00000000000460700081D000100B06B00209F
:1003B00040710020000000005007000827000400E2
:1003C000D06B00204471002000000000520700089C
:1003D000012008008C690020487100200000000006
:1003E000560700081A000A006C69002050710020AE
:1003F000000000005E07000803000100C069002043
:100400005C710020000000000000000016000800E1
:10041000F8720020D07C002000000000680700086F
:1004200007020200AC7C0020F87C002000000000E5
:100430007007000802000C00EC720020FC7C002019
:10044000000000000000000006020C00847C002078
:10045000087D002000000000ED20030808020900CC
:100460000E7C0020147D002000000000A92003085D
:10047000F7010600087C0020207D0020000000001D
:10048000720700080E20EA00D67F00207886002040
:1004900000000000E5670208130004006C830020E0
:1004A00064870020000000007807000801010400B4
:1004B000567F002068870020000000000000000038
:1004C000000104004E7F00206C8700200000000027
:1004D0007C07000802010300497F0020708700208C
:1004E000000000002D2003080902010034860020CE
:1004F0007487002000000000800700080C106000D6
:10050000E68000207887002000000000012003081A
:10051000010205005E7F0020D88700200000000057
:1005200075720308000205002C7D0020E087002082
:1005300000000000000000001E0004006881002090
:10054000E8870020000000008207000822000C005D
:100550003C850020EC870020000000008607000892
:10056000040080006CB50020A8BE00200000000040
:1005700000000000F901040044AA002028BF002068
:100580000000000071800008FD0124001CAA00206A
:100590002CBF00200000000001800008061016009B
:1005A000449D002050BF0020000000001568020894
:1005B000FB0101007C9C002068BF002000000000BF
:1005C0006D200308FC010900489B00206CBF00203F
:1005D00000000000752003080A101E00109B002078
:1005E00078BF0020000000009207000834001000CF
:1005F000F091002098BF002000000000A1670208D1
:1006000011020800C8910020A8BF002000000000CF
:10061000B007000812120400C0910020B0BF0020F3
:1006200000000000B807000812200E00AC91002066
:10063000B4BF002000000000BC07000818202C00F8
:1006400044910020C4BF002000000000E91A010806
:100650000D002C0070910020F0BF00200000000071
:100660000D210308020203001C8800201CC000208A
:1006700000000000000000000C0201000C880020B7
:1006800020C0002000000000CA070008FE01090089
:10069000488A002024C0002000000000C920030870
:1006A000000000000000000000000000000000004A
:1006B000000000000000000000000000000000003A
:1006C000000000000000000000000000000000002A
:1006D0000000000000000100000000000000000019
:1006E00000000000030000050000280100000401D4
:1006F000F4011900000000000000000000000000EC
:1007000000000000000000002000030100002B2179
:10071000231E64010100000001000A0129000000FD
:1007200000000000010000000500000102030000BD
:1007300000000000000000000000000004010100B3
:100740006C160000000000004A01B400D601000051
:10075000000020030000E8036400040A00017E0595
:10076000EA05B40532000000C40900001901282878
:10077000013C220100000000480404009001000038
:10078000000000000100C800141E010064002C01DC
:10079000280000300100005A000000000000900115
:1007A0002C01C800640002000000000000000000EE
:1007B0000000000001010101FFFFFFFF0000000138
:0B07C0000000054653443431000001E6
:1007CB000100000080010000080000000400000090
:1007DB0000000000000000000102030406070809E6
:1007EB00D6010000C1F50008000000000000000069
:1007FB00010000000001010100000000FFFFFFFFEE
:10080B0001000000685E0C00010102FFFFFF000009
:10081B000403090412010002020200408304405742
:10082B00000201020301000009024300020100C0A3
:10083B003209040000010202010005240010010529
:10084B00240100010424020205240600010705828D
:10085B00030800FF09040100020A0000000705015C
:10086B00024000000705810240000000FF0000006D
:10087B0000FFFF0000000000AA5505010000010069
:10088B0000000101FFFF0000000000000102030453
:10089B000102030406070809E7200208ED1F0208FE
:1008AB00C921020841F9010837FC010851F9010877
:1008BB006DF901081BF901080DF901080000000092
:1008CB00000000002D202D2D202D2D2D2D202D2D28
:1008DB002D2D0000000000000000000000000000B3
:1008EB00000000AA550B010000AA5507010000AA41
:1008FB00550902000000000001000000C012AA55BB
:10090B0003009F00FF1FFF1FDC9304080000000083
:10091B000000000041200308A08601000400000035
:10092B0000000000000000000000000000000000BC
:10093B000000000000000000000000006CAD040887
:10094B002C930408000000003DB902087D00000054
:10095B000600000000000000000000000000000086
:10096B00000000000000000000000000000000007C
:10097B0034930408000000000000000055970108A4
:10098B00E80300000300000000000000000000006E
:10099B00000000000000000000000000000000004C
:1009AB0000000000E4A304080000000000000000A9
:1009BB006174020810270000030000000000000013
:1009CB00000000000000000000000000000000001C
:1009DB000000000000000000F0A30408000000006D
:1009EB00B1010108A9C90108204E00000500000053
:1009FB0000000000000000000000000000000000EC
:100A0B000000000000000000000000007C950408BE
:100A1B00000000000000000039F201081027000060
:100A2B0001000000000000000000000000000000BA
:100A3B0000000000000000000000000000000000AB
:100A4B00F4A304080000000000000000C5760108B4
:100A5B00E80300000500000000000000000000009B
:100A6B00000000000000000000000000000000007B
:100A7B000000000000A404080000000000000000BB
:100A8B0065290308204E0000030000000000000051
:100A9B00000000000000000000000000000000004B
:100AAB00000000000000000010A40408000000007B
:100ABB00000000005D270308204E0000030000002B
:100ACB00000000000000000000000000000000001B
:100ADB0000000000000000000000000020A404083B
:100AEB00000000000000000021780108400D030009
:100AFB0003000000000000000000000000000000E8
:100B0B0000000000000000000000000000000000DA
:100B1B00A094040800000000000000003537030813
:100B2B001027000001000000000000000000000082
:100B3B0000000000000000000000000000000000AA
:100B4B00000000004C9304080000000000000000AF
:100B5B0091AF030810270000030000000000000005
:100B6B00000000000000000000000000000000007A
:100B7B000000000000000000389304080000000093
:100B8B0000000000FD7E010850C3000001000000C2
:100B9B00000000000000000000000000000000004A
:100BAB0000000000000000000000000030A404085A
:100BBB000000000000000000917A0108A86100000D
:100BCB000100000000000000000000000000000019
:100BDB00000000000000000000000000000000000A
:100BEB003CA40408000000000000000019C4030826
:100BFB00A0860100010000000000000000000000C2
:100C0B0000000000000000000000000000000000D9
:100C1B0000000000849504080000000000000000A4
:100C2B00ED9E0108A00F0000010000000000000075
:100C3B0000000000000000000000000000000000A9
:100C4B00000000000000000048A4040800000000A1
:100C5B00000000001D170208102700000100000013
:100C6B000000000000000000000000000000000079
:100C7B00000000000000000000000000A894040821
:100C8B000000000000000000056002081A4100008F
:100C9B000100000000000000000000000000000048
:100CAB000000000000000000000000000000000039
:100CBB00E495040800000000000000009501020804
:100CCB0010270000010000000000000000000000E1
:100CDB000000000000000000000000000000000009
:100CEB0000000000A8A304080000000000000000A2
:100CFB009D9C03081A410000010000000000000049
:100D0B0000000000000000000000000000000000D8
:100D1B00000000000000000054A4040800000000C4
:100D2B0000000000413B0208400D030000000000E2
:100D3B0000000000000000000000000000000000A8
:100D4B000000000000000000000000005CA404088C
:100D5B00000000000000000081760108400D030038
:100D6B000000000000000000000000000000000078
:100D7B000000000000000000000000000000000068
:100D8B0064A404080000000000000000B9B50308CB
:100D9B00A08601000300000000000000000000001E
:100DAB000000000000000000000000000000000038
:100DBB000000000070A40408000000000000000008
:100DCB002927030840420F0000000000000000002C
:100DDB000000000000000000000000000000000008
:100DEB0000000000000000007CA4040800000000CC
:100DFB0000000000E122030850C3000000000000C7
:100E0B0000000000000000000000000000000000D7
:100E1B0000000000000000000000000001000000C6
:100E2B00FFFFFFFF0000803F0000000000000000FC
:100E3B00000000000000803F0000000000000000E8
:100E4B000000000000000000000000000000000097
:100E5B000000000000000000000000000000803FC8
:100E6B000000000000000000000000000100000076
:100E7B000000803F0000803F0000000000000000E9
:100E8B00000000000000803F00000000E87C002014
:100E9B000800000000000000D87C002008000000C3
:100EAB00B45E040805080400000000001C6504087B
:100EBB003C5704080865040800000000000000000F
:100ECB00E05E040805080A00000000001C65040829
:100EDB003C570408246404080000000000000000D4
:100EEB00E00101010100000069740308000000002B
:100EFB009C08002074B304080000000000000000F0
:100F0B000000000000000000177304080000000040
:100F1B0000000000280900200400000020B3040892
:100F2B000D000000E59703083C22002000000000A4
:100F3B00DCAC04080D0000000D98030830220020E3
:100F4B00000000004CAE0408080000000000000088
:100F5B00242200200400000048AD04080D0000000E
:100F6B001D7503081822002000000000FCAD0408CA
:100F7B0003000000119B03080C220020000000005E
:100F8B0084B3040803000000119B03080022002017
:100F9B000000000048AA0408010000000000000047
:100FAB000000000000000000000000000E00000028
:100FBB0000000000000000000000000074B30408F3
:100FCB000000000000000000000000000000000016
:100FDB00177304080000000000000000280900201F
:100FEB0004000000CCB2040803000000F5880308DD
:100FFB00F42100200800000048AD04080D0000009B
:10100B001D7503081822002000000000FCAD040829
:10101B0003000000119B03080C22002000000000BD
:10102B0084B3040803000000119B03080022002076
:10103B000000000048AA04080100000000000000A6
:10104B000000000000000000000000000E00000087
:10105B000000000000000000000000008CB304083A
:10106B000000000000000000000000000000000075
:10107B00177304080000000000000000280900207E
:10108B0004000000D4B2040803000000119B030805
:10109B00482200200000000048AA040801000000BC
:1010AB000000000000000000000000000000000035
:1010BB000E00000000000000000000000000000017
:1010CB0020700020702D720008000000000000004E
:1010DB0000000000B01D0020FFFFFFFFFA00000022
:1010EB0001000000010000002D202D2D202D2D2DA5
:1010FB002D202D2D2D000000000000000000000011
:10110B0000000000000000001CAA040824AA040828
:10111B0040AA0408000000000000000000000000CE
:10112B0000000000B4A9040804000000AD950308FA
:10113B00000000000000000048AA040801000000A5
:10114B000000000000000000000000000000000094
:10115B000E00000000000000000000000000000076
:10116B001EB600200100C409000000001CB60020C0
:10117B000100C409000000001AB600200100C409D8
:10118B000000000018B600200100C4090000000098
:10119B0014B600200100C4090000000016B60020A0
:1011AB000100C4090000000012B600200100C409B0
:1011BB000000000010B600200100C4090000000070
:1011CB00707F00200100C800010000006E7F00202E
:1011DB0032003075320000006C7F0020055A05008C
:1011EB00697F002000FF01006B7F002001000000E1
:1011FB0048090020677F00200200000038580408CF
:10120B00687F002000FF01006A7F002001000000C2
:10121B0048090020667F00200200000038580408AF
:10122B005C7F002080C1803E050000005A7F0020BB
:10123B0080C1803E05000000547F002080C1803EAD
:10124B0005000000527F002080C1803E0500000099
:10125B004C7F002000FF0100487F00200A32010074
:10126B00477F00200400000004640408467F002030
:10127B0002000000186404080000000000000000D9
:10128B00500900200C4F00209CFF2C010000000097
:10129B00220700200A000000246404083C7F002081
:1012AB00E0150C17000000002407002008000000C8
:1012BB003C57040823070020050000001C650408A8
:1012CB003E7F0020020000003C6404085A8100208D
:1012DB000100FF7F01000000598100200200000087
:1012EB0048640408CB7F0020030000005864040806
:1012FB00CA7F00200300000058640408C880002047
:10130B000000F40101000000C68000200000F40181
:10131B0001000000C48000200000F4010100000067
:10132B00C28000200000F40101000000C0800020FA
:10133B0000FF0100E4800020E803D0070A00000052
:10134B00E2800020006401000A000000D78000202A
:10135B0000640100D680002000640100DE800020C4
:10136B00006401000A000000DD8000200064010021
:10137B000A000000DC800020006401000A0000006D
:10138B00E1800020006401000A000000E0800020E2
:10139B00006401000A000000DF80002000640100EF
:1013AB000A000000DB80002000FF01000A000000A3
:1013BB00DA80002000FF01000A000000D980002025
:1013CB0000FF01000A000000D27F00200000F401A2
:1013DB0001000000D07F00200000F401010000009C
:1013EB00CE7F00200000F40101000000CC7F002024
:1013FB000000F40101000000D28000201400E8037B
:10140B0001000000D0800020E803307501000000CF
:10141B00CF80002000C80100CE80002000C8010052
:10142B00CD80002000C80100CC80002000640100AA
:10143B000A000000CB80002000FF01000A00000022
:10144B004F81002000C801004E81002000C8010020
:10145B004D81002000C801004C81002000C8010014
:10146B004B81002000C801004A81002000C8010008
:10147B004981002000C801004881002000C80100FC
:10148B004781002000C8010070AA0408000000007A
:10149B0000000000000000000000000080AA04080B
:1014AB000900000000000000F40900200400000007
:1014BB0088AA04080900000000000000E8090020C9
:1014CB0004000000BCB0040809000000000000008C
:1014DB00DC0900200400000050A0040809000000F3
:1014EB0000000000D00900200400000090AA0408AE
:1014FB000900000000000000C409002004000000E7
:10150B0098AA04080900000000000000B809002098
:10151B0004000000A0AA040809000000000000005D
:10152B00AC09002004000000A8AA04080900000070
:10153B0000000000A00900200400000048AA0408D5
:10154B00010000000000000000000000000000008F
:10155B00000000000E000000000000000000000072
:10156B0000000000D0AB04080000000000000000E9
:10157B00000000000000000090930408070000002A
:10158B0000000000180A002000000000E0AB040877
:10159B0008000000000000000C0A00200000000002
:1015AB00ECAB04080800000000000000000A00205B
:1015BB000000000048AA0408010000000000000021
:1015CB000000000000000000000000000E00000002
:1015DB00000000000000000000000000F4AB040855
:1015EB0000000000000000000000000000000000F0
:1015FB0004AC04080D00000000000000540A002099
:10160B00000000000CAC04080D00000000000000FE
:10161B00480A00200000000014AC0408070000007A
:10162B0000000000400A0020000000001CAC040871
:10163B000D00000000000000340A00200000000034
:10164B0024AC04080D00000000000000280A002054
:10165B00000000002CAC0408070000000000000094
:10166B00200A00200000000048AA04080100000026
:10167B00000000000000000000000000000000005F
:10168B000E00000000000000000000000000000041
:10169B0034AC040800000000000000000000000053
:1016AB0000000000909304080C00000000000000F4
:1016BB00727F00200000000048AC04080C00000002
:1016CB0000000000747F00200000000058AC0408EC
:1016DB000C00000000000000AA7F002000000000AA
:1016EB0068AC04080C000000000000009E7F002086
:1016FB00000000007CAC04080C000000000000009F
:10170B00767F002000000000CCA604080C0000002F
:10171B0000000000787F00200000000088AC040867
:10172B000C000000000000007A7F00200000000089
:10173B009CAC04080C000000000000007C7F002023
:10174B0000000000A4AC04080C0000000000000026
:10175B007E7F002000000000ACAC04080C000000F1
:10176B0000000000BC7F002000000000C4AC040897
:10177B000C00000000000000807F00200000000033
:10178B00D0AC04080C00000000000000827F002099
:10179B000000000068A304080C000000000000001B
:1017AB00847F002000000000D8AC04080C0000006F
:1017BB0000000000867F002000000000E4AC04085D
:1017CB000C00000000000000887F002000000000DB
:1017DB00F0AC04080C000000000000008A7F002021
:1017EB0000000000FCAC04080C000000000000002E
:1017FB008C7F00200000000008AD04080C000000E6
:10180B00000000008E7F00200000000014AD0408D3
:10181B000C00000000000000A27F00200000000070
:10182B001CAD04080C00000000000000A07F00208D
:10183B000000000024AD04080C00000000000000B4
:10184B00AE7F00200000000030AD04080C0000004B
:10185B0000000000B07F0020000000003CAD040839
:10186B000C00000000000000B67F0020000000000C
:10187B0030A404080C00000000000000907F002042
:10188B000000000048AD04080C0000000000000040
:10189B00987F00200000000050AD04080C000000F1
:1018AB0000000000927F0020000000005CAD0408E7
:1018BB000C00000000000000947F002000000000DE
:1018CB0068AD04080C00000000000000967F0020AB
:1018DB000000000070AD04080C00000000000000C8
:1018EB009A7F002000000000B09304080C00000059
:1018FB0000000000A47F0020000000007CAD040865
:10190B000C000000000000009C7F00200000000085
:10191B0088AD04080C00000000000000AC7F002024
:10192B000000000094AD04080C0000000000000053
:10193B00A67F0020000000009CAD04080C000000F6
:10194B0000000000A87F002000000000A4AD0408E8
:10195B000C00000000000000B27F0020000000001F
:10196B00ACAD04080C00000000000000B47F0020A8
:10197B000000000048AA040801000000000000005D
:10198B000000000000000000000000000E0000003E
:10199B00000000000000000000000000B4AD0408CF
:1019AB00000000000000000000000000000000002C
:1019BB00C0AD04080D00000000000000AC0A0020C0
:1019CB0000000000C8AD04080D000000000000007E
:1019DB00A00A002000000000D0AD040807000000A2
:1019EB0000000000980A002000000000DCAD040895
:1019FB000700000000000000900A0020000000001B
:101A0B00E8AD04080900000000000000840A002073
:101A1B0000000000F4AD0408090000000000000005
:101A2B00780A00200000000000AE04080900000046
:101A3B00000000006C0A00200000000010AE04083B
:101A4B000900000000000000600A002000000000F8
:101A5B0048AA04080100000000000000000000007C
:101A6B0000000000000000000E000000000000005D
:101A7B00000000000000000024AE0408000000007D
:101A8B0000000000000000000000000034AE04085D
:101A9B000500000000000000C97F002000000000CE
:101AAB0048AA04080100000000000000000000002C
:101ABB0000000000000000000E000000000000000D
:101ACB0000000000000000003CAE04080000000015
:101ADB000000000000000000000000001773040865
:101AEB0000000000000000000401002004000000C2
:101AFB0048AE04080D00000011960308000B0020EF
:101B0B000000000020B304080D000000217403083E
:101B1B00F40A002000000000DCAC04080D000000FB
:101B2B0005740308E80A0020000000004CAE04080E
:101B3B000800000000000000DC0A00200400000088
:101B4B0048AD04080D0000004D730308D00A0020B7
:101B5B000000000054AE0408090000000000000063
:101B6B00C40A002004000000FCAD040803000000C0
:101B7B00119B0308B80A00200000000048AA0408C3
:101B8B000100000000000000000000000000000049
:101B9B00000000000E00000000000000000000002C
:101BAB00000000005CAE0408000000000000000014
:101BBB0000000000000000006CAE04080D000000E7
:101BCB0000000000180B00200000000074AE040899
:101BDB000A000000000000009283002000000000BB
:101BEB0080AE04080A000000000000009A83002069
:101BFB000000000088AE04080A000000000000008E
:101C0B00A28300200000000090AE04080800000032
:101C1B00000000000C0B00200000000048AA040884
:101C2B0001000000000000000000000000000000A8
:101C3B00000000000E00000000000000000000008B
:101C4B000000000098AE0408000000000000000037
:101C5B000000000000000000ACAE04080D00000006
:101C6B0000000000300B002000000000BCAE040898
:101C7B000400000059980308000000000000000059
:101C8B00C4AE04080D00000000000000240B00206F
:101C9B0000000000D8AE04080400000035980308CB
:101CAB00000000000000000048AA0408010000002A
:101CBB000000000000000000000000000000000019
:101CCB000E000000000000000000000000000000FB
:101CDB00E0AE04080000000000000000000000005F
:101CEB0000000000F4AE0408070000000000000034
:101CFB006C0B00200000000000AF0408080000007F
:101D0B0000000000600B0020000000000CAF040876
:101D1B000800000000000000540B00200000000031
:101D2B0018AF04080800000000000000480B00205A
:101D3B000000000024AF04080800000000000000B1
:101D4B003C0B00200000000048AA04080100000022
:101D5B000000000000000000000000000000000078
:101D6B000E0000000000000000000000000000005A
:101D7B0030AF040800000000000000000309002041
:101D8B00000000003CAF04080B0000000000000046
:101D9B00FC0B00200000000048AF04080B00000003
:101DAB0000000000F00B00200000000054AF0408FE
:101DBB000B00000000000000E40B002000000000FE
:101DCB0060AF04080B00000000000000D80B0020DF
:101DDB00000000006CAF04080B00000000000000C6
:101DEB00CC0B00200000000078AF04080B000000B3
:101DFB0000000000C00B00200000000084AF0408AE
:101E0B000B00000000000000B40B002000000000DD
:101E1B0090AF04080B00000000000000A80B00208E
:101E2B00000000009CAF04080B0000000000000045
:101E3B009C0B002000000000A8AF04080700000066
:101E4B0000000000940B002000000000B0AF04085D
:101E5B0007000000000000008C0B002000000000B9
:101E6B00BCAF04080B00000000000000800B00203A
:101E7B0000000000C8AF04080800000000000000CC
:101E8B00740B00200000000048AA040801000000A9
:101E9B000000000000000000000000000000000037
:101EAB000E00000000000000000000000000000019
:101EBB00D4AF040800000000000000000000000088
:101ECB0000000000E8AF040808000000000000005C
:101EDB002C0C002000000000F4AF040808000000E8
:101EEB0000000000200C00200000000000B00408DF
:101EFB000800000000000000140C0020000000008F
:101F0B000CB004080800000000000000080C0020C2
:101F1B000000000048AA04080100000000000000B7
:101F2B000000000000000000000000000E00000098
:101F3B0000000000000000000000000014B00408C6
:101F4B00000000000000000000090020000000005D
:101F5B0024B004080B00000000000000740C0020EB
:101F6B000000000030B004080B000000000000006F
:101F7B00680C0020000000003CB0040807000000C3
:101F8B0000000000600C00200000000048B00408B6
:101F9B000700000000000000580C002000000000AB
:101FAB0054B004080700000000000000500C002093
:101FBB000000000060B004080800000000000000F2
:101FCB00440C00200000000068B00408080000006A
:101FDB0000000000380C00200000000048AA040894
:101FEB0001000000000000000000000000000000E5
:101FFB00000000000E0000000000000000000000C8
:10200B000000000070B00408000000000000000099
:10201B0000090020000000007CB00408070000004D
:10202B0000000000C00C00200000000084B0040879
:10203B000700000000000000B80C002000000000AA
:10204B008CB004080700000000000000B00C00205A
:10205B000000000018A004080700000000000000AA
:10206B00A80C00200000000020A0040807000000BE
:10207B0000000000A00C00200000000028A00408B5
:10208B000700000000000000980C0020000000007A
:10209B0094B004080700000000000000900C002022
:1020AB00000000009CB004080700000000000000C6
:1020BB00880C002000000000A4B0040807000000FA
:1020CB0000000000800C00200000000048AA04085B
:1020DB0001000000000000000000000000000000F4
:1020EB00000000000E0000000000000000000000D7
:1020FB00000000000000000091770308C80C0020CE
:10210B00C77F00201C00000068640408C67F002005
:10211B0000C80100C47F0020E803D00701000000C5
:10212B0046554C4C53504545444634313100000024
:10213B00657F002000030100647F00200003010085
:10214B00D9760308B1760308A40D00206D76030839
:10215B00217603081C0E002019770308017703086A
:10216B00D00E00208D75030841750308DC1100208B
:10217B00A7770308AD830308B81200208D730308FB
:10218B00000000000813002035890308FD790308BF
:10219B00E4130020CD770308000000008414002016
:1021AB00717803084178030810150020FD780308A7
:1021BB0041790308B0150020D480002001060100EE
:1021CB000D780308E1770308F0160020A1780308C7
:1021DB007D9803087C1700206D790308D9980308B4
:1021EB0044180020CA80002001030100ACB0040891
:1021FB0000000000000000000000000000000000D4
:10220B00B8B00408080000000000000054190020BA
:10221B0000000000C0B00408070000000000000030
:10222B004C19002000000000D0B004080D00000085
:10223B00000000004019002000000000DCB0040882
:10224B0003000000119B030834190020000000005C
:10225B0048AA040801000000000000000000000074
:10226B0000000000000000000E0000000000000055
:10227B000000000000000000E4B0040800000000B3
:10228B00000000000000000000000000F4B0040893
:10229B000A00000000000000ACA6040800000000CB
:1022AB00FCB004080A000000000000009D6E04084A
:1022BB000000000004B104080A0000000000000048
:1022CB0050810020000000000CB104080A0000003F
:1022DB0000000000601900200000000048AA04085C
:1022EB0001000000000000000000000000000000E2
:1022FB00000000000E0000000000000000000000C5
:10230B000000000014B104080000000000000000F1
:10231B00000000000000000020B1040803000000D2
:10232B00119B030898190020000000002CB1040831
:10233B0003000000119B03088C1900200000000013
:10234B0034B1040803000000119B0308801900201E
:10235B00000000003CB10408050000000000000074
:10236B00637F00200000000044B104080700000058
:10237B0000000000781900200000000050B1040894
:10238B000700000000000000701900200000000092
:10239B0048AA040801000000000000000000000033
:1023AB0000000000000000000E0000000000000014
:1023BB0000000000000000005CB1040800000000F9
:1023CB0000000000000000000000000080A70408CF
:1023DB0003000000119B0308C81900200000000037
:1023EB0070B1040803000000119B030828070020AC
:1023FB000000000078B1040803000000119B0308E3
:10240B00BC1900200000000080B10408030000008C
:10241B00119B0308B01900200000000048AD040810
:10242B0003000000119B0308A4190020000000000A
:10243B0048AA040801000000000000000000000092
:10244B0000000000000000000E0000000000000073
:10245B0000000000000000008CB104080000000028
:10246B0000000000000000000000000098B104080C
:10247B000700000025990308241A00200000000023
:10248B006CAD040803000000119B0308181A002010
:10249B0000000000A4B1040803000000119B030816
:1024AB000C1A002000000000ACB10408030000006F
:1024BB00119B0308001A002000000000B4B10408AF
:1024CB000700000009990308F8190020000000001C
:1024DB00AC9F040803000000119B0308EC190020BB
:1024EB0000000000C0B1040803000000119B0308AA
:1024FB00E019002000000000CCB10408030000002C
:10250B00119B0308D41900200000000048AA0408FE
:10251B0001000000000000000000000000000000AF
:10252B00000000000E000000000000000000000092
:10253B000000000061770308317703082C1A002094
:10254B00DD79030800000000B81A0020FD750308B0
:10255B00D9750308441B0020000000000000000098
:10256B00F81B0020B579030841990308981C00203B
:10257B00D8B10408000000000000000000000000BB
:10258B0000000000E4B1040803000000119B0308E5
:10259B00A41D002000000000ECB1040803000000A3
:1025AB00119B0308981D002000000000A89404084C
:1025BB0003000000119B03088C1D0020000000008D
:1025CB00F8B1040803000000119B0308801D0020D4
:1025DB000000000004B2040803000000119B030874
:1025EB00741D0020000000000CB204080200000063
:1025FB00C1990308000000000000000014B2040899
:10260B0002000000C1990308010000000000000057
:10261B0020B2040802000000C19903080200000068
:10262B0000000000000000000E0000000000000091
:10263B000000000000000000427F002088136F178D
:10264B0001000000447F002088136F17000000007A
:10265B002CB2040800000000000000000000000085
:10266B00000000003CB2040808000000000000005D
:10267B00841E00200400000048B20408080000007B
:10268B0000000000781E002000000000FCAD0408D4
:10269B000400000039960308000000000000000051
:1026AB0048AA040801000000000000000000000020
:1026BB0000000000000000000E0000000000000001
:1026CB000000000000000000407F002088136F17FF
:1026DB0001000000484F002088136F170000000016
:1026EB00D174030800000000901E00200D84002010
:1026FB0001000000DC6404084A4F002001000000C8
:10270B00E8640408404F002002000000F064040855
:10271B0066B60020000000000000000064B6002038
:10272B00000000000000000062B600200000000066
:10273B000000000060B60020000000000000000058
:10274B005EB6002000000000000000005CB6002018
:10275B0000000000000000003C0100200000000011
:10276B00000000003F7F002002000000FC64040812
:10277B0084B204080000000000000000000000000C
:10278B00000000003CB2040808000000000000003C
:10279B00141F00200400000048B2040808000000C9
:1027AB0000000000081F002000000000FCAD040822
:1027BB0004000000A17403080000000000000000EA
:1027CB0048AA0408010000000000000000000000FF
:1027DB0000000000000000000E00000000000000E0
:1027EB00000000000000000094B20408000000008C
:1027FB00000000000000000000000000A4B204086C
:10280B000D00000089970308441F002004000000FE
:10281B00B0B204080D000000F9740308381F002043
:10282B0004000000BCB204080D0000004D97030823
:10283B002C1F002000000000C8B204080300000099
:10284B0015890308201F002008000000D4B20408DB
:10285B0003000000119B0308482200200000000029
:10286B0048AA04080100000000000000000000005E
:10287B0000000000000000000E000000000000003F
:10288B00000000000000000040AA04080000000047
:10289B00000000000000000000000000B4A90408C4
:1028AB000400000051960308000000000000000027
:1028BB0048AA04080100000000000000000000000E
:1028CB0000000000000000000E00000000000000EF
:1028DB00000000000000000028B304080000000006
:1028EB0000000000000000000000000078960408C3
:1028FB000D00000000000000A41F002004000000D9
:10290B0038B304080800000000000000981F0020E6
:10291B000400000044B3040808000000000000009D
:10292B008C1F0020040000004CB3040808000000BA
:10293B0000000000801F00200400000054B30408B6
:10294B000800000000000000741F002004000000BD
:10295B005CB304080800000000000000681F0020A2
:10296B000400000064B3040808000000000000002D
:10297B005C1F0020040000006CB30408080000007A
:10298B0000000000501F00200400000048AA0408AB
:10299B00010000000000000000000000000000002B
:1029AB00000000000E00000000000000000000000E
:1029BB0000000000B974030800000000B01F0020E5
:1029CB000000000000000000282000200000000094
:1029DB0000000000C8200020464F0020040000002B
:1029EB0008650408444F0020E0150C170000000098
:1029FB00434F0020080000003C570408424F0020C2
:102A0B00050000001C650408000000000000000029
:102A1B00182100200800000081FE0108A3FB01081B
:102A2B00AD0A020800000000E9F8010869FD010881
:102A3B0053FE0108CBFC0108000000000000000061
:102A4B00DDF80108C1F80108BFF80108BDF801085D
:102A5B00B7F80108B5F80108BBF80108B9F8010887
:102A6B00D1F80108C3F80108850A0208990A02087F
:102A7B00710A02085D0A0208490A020801000000F7
:102A8B0000600240106002400000000000000000E7
:102A9B00000B000000000000000000000000000020
:102AAB0000600240286002400100000000000000AE
:102ABB00060C0000000000000000000000000000F9
:102ACB000060024040600240020000000000000075
:102ADB00100D0000000000000000000000000000CE
:102AEB00006002405860024003000000000000003C
:102AFB00160E0000000000000000000000000000A7
:102B0B000060024070600240040000000000000002
:102B1B00200F00000000000000000000000000007B
:102B2B0000600240886002400500000000000000C9
:102B3B002610000000000000000000000000000054
:102B4B0000600240A0600240060000000000000090
:102B5B003011000000000000000000000000000029
:102B6B0000600240B8600240070000000000000057
:102B7B00362F0000000000000000000000000000E5
:102B8B0000640240106402400000000000000000DE
:102B9B0000380000000000000000000000000000F2
:102BAB0000640240286402400100000000000000A5
:102BBB0006390000000000000000000000000000CB
:102BCB00006402404064024002000000000000006C
:102BDB00103A0000000000000000000000000000A0
:102BEB000064024058640240030000000000000033
:102BFB00163B000000000000000000000000000079
:102C0B0000640240706402400400000000000000F9
:102C1B00203C00000000000000000000000000004D
:102C2B0000640240886402400500000000000000C0
:102C3B00264400000000000000000000000000001F
:102C4B0000640240A0640240060000000000000087
:102C5B0030450000000000000000000000000000F4
:102C6B0000640240B864024007000000000000004E
:102C7B0036460000000000000000000000000000CD
:102C8B000000803FC824002000000000000000006E
:102C9B000000000000000000000000000000000029
:102CAB000000000000000000000000000000000019
:102CBB000000000000000000000000000000000009
:102CCB0000000000000000000000000000000000F9
:102CDB0000000000000000000000000000000000E9
:102CEB000000000000000000430000000000000096
:102CFB0000000000000000000000000000000000C9
:102D0B000000000000000000430000000000000075
:102D1B0000000000000000000000000000000000A8
:102D2B000000000000000000430000000000000055
:102D3B000000000000000000000000000000000088
:102D4B000000000000000000430000000000000035
:102D5B000000000000000000000000000000000068
:102D6B000000000000000000430000000000000015
:102D7B000000000000000000000000000000000048
:102D8B0000000000000000004300000000000000F5
:102D9B000000000000000000000000000000000028
:102DAB0000000000000000004300000000000000D5
:102DBB000000000000000000000000000000000008
:102DCB000000000000000000832C04085F2C0408A6
:102DDB0000000000D2B40408B0A90408177304085B
:102DEB001773040817730408177304081773040880
:102DFB001773040817730408177304081773040870
:102E0B00FFFFFFFFFFFFFFFFFFFFFFFFFFFF0000C5
:102E1B00010041534349490000000000000000003D
:102E2B000000000000000000000000000000000097
:102E3B00000041534349490000000000000000001E
:102E4B000000000000000000000000000000000077
:042E5B000000000073
:108000000A4B30B503F1100493F900205D78072A7C
:10801000C8BF143A811804330D7313F8025C8554F9
:1080200013F8012C0A769C42EED130BD9435040839
:1080300003682DE9F041DD691DB12B46BDE8F04133
:108040001847002A174611DD04460E460F4400E08B
:1080500023689B68204698470028F9D0236816F8C3
:10806000011B1B6820469847BE42F1D1BDE8F08154
:1080700000233D213E22017042708370C37070471F
:108080000028F0B403DA2D230B7040420131092897
:1080900004464FF0010307DD03EB83035B00B0FBF5
:1080A000F3F2092AF8D883B10F48A0FB0326B4FBEA
:1080B000F3F2092A02F1570C02F1300709DD03FB44
:1080C0001244F30801F801CBEFD100230B70F0BC90
:1080D000704703FB1244F30801F8017BE5D100234C
:1080E0000B70F0BC704700BFCDCCCCCC884270B4D4
:1080F0004FF0010442D301FB04F4B0FBF4F58D42D0
:10810000F9D2ECB142BB092D04FB150005F157066D
:1081100005F130020EDDB4FBF1F403F8016B7CB124
:10812000B0FBF4F5092D04FB150005F1570605F128
:108130003002F0DCB4FBF1F403F8012B002CEFD19A
:1081400000221A7070BC704703F8016BB4FBF1F4A5
:10815000002CF5D0B0FBF4F5092D04FB150005F15A
:10816000370605F13002EFDCB4FBF1F403F8012B24
:10817000002CEFD100221A7070BC70470546002A0F
:10818000EAD1C0E72DE9F04714461D460646002314
:108190004FF47A72204629463AF092F9DFF8488186
:1081A0004B4A4C4F88FB00310144C31782FB002C23
:1081B000C3EB611188FB012887FB00278444464AF2
:1081C000C3EBEC2CC1EB011E82FB0C29A0EB8E0E45
:1081D0000744424A86F806E0C3EB27474FEAEC7EA5
:1081E00008EB010ACEEBA90E82FB07824FEAE17889
:1081F0000EEB4E0EC8EB6A18ACEBCE0CC8EB0818B1
:10820000DFF8E8E086F804C0A1EB880171718EFB0D
:108210000010F917C1EBE21240F2B55101FB1272E6
:10822000C3EBE050B2F5896F4FEA80073FDA40F2C6
:10823000DA239A4243DCB2F5B77FB4BF4FF0000EA9
:108240004FF0010E4FEA4E08254B08EB0E0103EBF1
:10825000C1031FFA8EFCD88C224908EB0E0301EBF8
:10826000C30116310B2301E031F8020D90421BDDF2
:10827000013BF9D11A4BC64403EBCE0E0123BEF8E5
:108280001000B37007F2B2770132121ABC44F270D8
:10829000A6F800C0204629464FF47A7200233AF02F
:1082A0000FF93281BDE8F0870133DBB2E9E74FF027
:1082B000030CE64640F296504FF00608CCE74FF02C
:1082C000020CE64640F229404FF00408C4E700BF24
:1082D000C5B3A29107452EC2ABAAAA2A73B06D16E8
:1082E00094350408A435040889888888792D0311F9
:1082F00003685A1C0260197070472DE9F047089C0A
:108300002578002B804689460CBF4FF0200A4FF09D
:10831000300A661C25B3002A26DD334601E00246FA
:1083200098B113F8011B501E0029F8D1971E60B1B7
:108330003D46013D51464046C8476B1C002BF8DCCA
:10834000257827EAE770013045B1041B29464046ED
:10835000C847301916F8015B002DF7D1BDE8F0874A
:10836000002A03DC2846F9E70020EEE7571EDFE786
:10837000D0E9012300EB830101339342D0ED037A6E
:1083800081ED040A836004BF0023836000EB830354
:1083900093ED047A036870EE277A9A42C0ED037A6F
:1083A00077EEC77AC0ED037A0CDA013307EE103AA4
:1083B000F8EEC76AB7EE007A87EEA60A036030EEE1
:1083C000070A704707EE102AB8EEC77A87EE870AC9
:1083D000704790ED057A90ED004AD0ED066AD0ED39
:1083E000014AD0ED047A90ED035AD0ED025AA4EE82
:1083F000007AB0EE406AB0EE470AB0EE667AA4EEBC
:10840000867A67EEC07AA5EE407AE5EE867A80ED50
:10841000057AC0ED067A7047D0ED057A90ED013A05
:10842000D0ED003AD0ED064A90ED024A90ED077A81
:1084300090ED035A90ED086AD0ED045AC0ED067A2B
:10844000F0EE406A27EE830AC0ED056AA3EEA60AA5
:1084500080ED087AA4EE240AA5EE470AA5EEC60A26
:1084600080ED070A7047D0ED007A90ED017A30EE8A
:10847000670AE7EE007AB0EE670AC0ED007A70474F
:1084800070470A44914215D030B40139551E41F26B
:10849000210211F8014F082380EA042004044CBF94
:1084A00082EA40004000013B80B2F7D18D42F0D11A
:1084B00030BC704770476D4B2DE9F04F1C686C4B1A
:1084C000B3F80AE0B3F804809A894FEA0E2AB4EBB5
:1084D0000A044FEA1E6B4FF0000587B065EB0B05F1
:1084E000CDE900450746009C1889019EA0FB044584
:1084F00000FB0655E00940EA45604FEA08448C4617
:10850000E9114FEA184510EB0408D888009C41EBAC
:108510000509CDE90489A0FB0445B3F8028000FBFE
:108520000655200A40EA05604FEAC83429124FEA8E
:10853000584510EB040841EB05090099A2FB010125
:1085400002FB06114FEAD05A4AEA412A1AF5FA63A9
:108550004FEAE15B4BF10004B3F5FA6FCDE9023469
:1085600074F10003414E64DA0524AAFB040104FB04
:108570000B1100FB0BF40AFB0144DDE90423A0FB13
:108580000A0121444D104FEA3004121B4FEA9004B7
:1085900063EB050344EA8174B8EB0408CDE90423D6
:1085A000DDE9023433484FEAA10569EB05094FF0D4
:1085B000FF31834274EB010326DA40F6AC501AEB2C
:1085C00000024FF000014BEB010302FB03F1A2FBA1
:1085D000022303EB4103D400DD00101B45EA527572
:1085E00063EB0501DDE9044524184D41CDE904455F
:1085F0000B24A2FB040104FB031149104FEA3000D5
:10860000B8EB000869EB0109DDE900325343009A39
:10861000DDE90201A2FB02AB0BEB430B4FEADA727E
:1086200042EA4B02801A4FEAEB7361EB0301CDE99A
:10863000020197B17168A1FB082301FB0933540DB6
:108640005D1544EAC324DDE90423A21A65EB0303A4
:108650001D46D30B43EA45433B60BCF1000F02D0FB
:10866000029BCCF8003007B0BDE8F08F98260020C0
:10867000C836002024FAFFFF2DE9F04FDFF8DCC1F7
:10868000754CDCF808502288B4F90AA0C2EB251317
:108690005200C2EBE502B4F902505B436A43B4F9FD
:1086A00004501B135D43AD1305EBE225B5F5FA321B
:1086B0004FEAE57B85B04BF1FF33CDE90023DDE9DF
:1086C00000325343009AA561A2FB0289CDE9020161
:1086D000B4F908200199009809EB43095143D317D5
:1086E00000FB0311A2FB00230B444FEAEA7B0AFBC9
:1086F00009F11F0308FB0B13AAFB080119444FEAF9
:10870000102A4AEA016A16034FEA212B47EA125758
:108710001AEB0602E6884BEB070312F1000A43F559
:10872000004BAAFB060106FB0B114A10CB1752EABD
:10873000030100F08E80B4F91060009806FB09F187
:10874000F71708FB0711A6FB08673944B4F90E8038
:108750008B4601994FEAE87908FB01F100FB09110A
:10876000A8FB00898944DCF80C104FEA4947C1F5A1
:10877000801C47EAD837B2464FEA4846B4F90C8025
:108780001AEB060A66464BEB070BF7174FEAC806CB
:10879000019600260096F907DDE900674FEACC70E4
:1087A00016EB0A0647EB0B0741EA5C01801B61EB05
:1087B000070140F6354C8946A0FB0C010CFB091162
:1087C00039F07EFEB4F91620B4F914A04E13470B0D
:1087D00047EAC14702FB06FCD31707FB03CCA2FB09
:1087E00007236344564307FB0366A2FB0723334476
:1087F000560E46EAC31632184FEA636747EB010389
:1088000080460AFB01F14FEAEA7B08FB0B17AAFB43
:1088100008013944C60C46EA413612EB06084FEA15
:10882000E147B4F9122043EB07094FEA182141EA66
:10883000096113010B44029A0AB11B0A1360039BDE
:1088400023B105EB850580352D121D6005B0BDE80F
:10885000F08F0023EFE700BFDC36002098260020D1
:10886000704770472DE9F041334B344E1A8A7489B2
:10887000B6F91450B6F90480B6F90E70B6F920C0F6
:108880005B69121B34895443E213B6F91240154454
:10889000E40294FBF5F4B6F902501444A4F57A6EA0
:1088A0000EFB0EF20EFB05F50EFB08FEB6F90C8072
:1088B000F4611213574302FB08F2121402EB6E32FA
:1088C000ED1205EBE7270232B6F90050B6F806E0E4
:1088D000921002F5004207EB85070EFB02F207FA41
:1088E0000CF74FEAD23E02374CF25032A3EBA70707
:1088F00042FA0CF37B4355BF5B00B3FBFEF3B3FBC3
:10890000FEF35B0078B11A1202FB02F540F6DE328C
:108910006A430B4D12145D4302EB254202F6CF620F
:1089200003EB2213036021B10A235C4308342411B2
:108930000C60BDE8F08100BF98260020A43600201E
:1089400043E3FFFF4FF40063838270474FF40063FB
:1089500083827047012380F8483070474FF40063EA
:1089600083827047F0B4037C456902681F2B37D9B6
:10897000203B2021546899400C4223D010249C4075
:10898000D160D4605168D940CE074ED4EFF3118343
:10899000502282F31288AA6B1168C90709D454685F
:1089A000002C52D1D5E909618E4243D1012285F8CC
:1089B0005C20DBB283F31188037C02681F2B19460D
:1089C00014D9203B082150689940084200D0D1605A
:1089D0000421506801FA03F3184223D1F0BC704718
:1089E000202416689C4026420FD11946082310689F
:1089F0008B40184200D093600423106803FA01F101
:108A00000842EBD09160F0BC70471021994094600F
:108A100091601168D940CC07B8D5012101FA03F360
:108A20009360B3E7D360F0BC7047012101FA03F310
:108A3000D360ABE7AF690F44D7600ED82E69711AC7
:108A40005160AC62002185F85C10116841F00101B1
:108A5000DBB2116083F31188AEE7711A5160AE6228
:108A6000F0E770B4037C01681F2B26D9A3F1200521
:108A700020224C68AA40224214BF01220022D2B117
:108A800042691C481C4C02EB420200EB4212257862
:108A900054682068CDB9E56856892C6824F0010433
:108AA0002C6082891F2B22EA060282811AD820229A
:108AB00002FA03F38B6070BC704720220C689A4066
:108AC000224214BF01220022D9E7A469226822F0C1
:108AD00001022260828922F480721204120C1F2B80
:108AE0008281E4D9A3F1200220239340CB6070BCA3
:108AF000704700BF6C9D0020689D0020844B1A7851
:108B0000002A00F00481834B1978834B30B400298C
:108B100065D11868B3F82C5141628489012A44EA6E
:108B200005048481A3F82C1157D0D3F83001B3F891
:108B30005C5241628489022A44EA05048481A3F8D4
:108B40005C124AD0D3F86002B3F88C534162848936
:108B5000032A44EA05048481A3F88C133DD0D3F89A
:108B60009003B3F8BC5441628489042A44EA0504A2
:108B70008481A3F8BC1430D0D3F8C004B3F8EC550A
:108B800041628489052A44EA05048481A3F8EC152E
:108B900023D0D3F8F005B3F81C5741628489062A24
:108BA00044EA05048481A3F81C1716D0D3F82007E3
:108BB000B3F84C5841628489072A44EA0504848149
:108BC000A3F84C1809D0D3F85028B3F87C49516267
:108BD000908920439081A3F87C1930BC70475C6871
:108BE000198961602568186845F0010540F20D316A
:108BF0002560A0F848108489012A44F48074848197
:108C0000EBD0D3F83441B3F83851D3F83001656074
:108C1000256845F001052560A0F848108489022ADE
:108C200044F480748481D8D0D3F86442B3F8685295
:108C3000D3F860026560256845F001052560A0F85D
:108C400048108489032A44F480748481C5D0D3F801
:108C50009443B3F89853D3F890036560256845F0C2
:108C600001052560A0F848108489042A44F4807422
:108C70008481B2D0D3F8C444B3F8C854D3F8C00444
:108C80006560256845F001052560A0F848108489D5
:108C9000052A44F4807484819FD0D3F8F445B3F856
:108CA000F855D3F8F0056560256845F001052560A5
:108CB000A0F848108489062A44F4807484818CD0FA
:108CC000D3F82447B3F82857D3F820076560256800
:108CD00045F001052560A0F848108489072A44F46E
:108CE000807484813FF479AFD3F85428B3F85808DE
:108CF000D3F850385060106840F001001060A3F8BD
:108D000048109A8942F480729A8130BC704770474B
:108D10006CA00020689D002070A0002010B4037C8F
:108D200002681F2B09D9203B2021546801FA03F364
:108D30001C4214D15DF8044B70472021146801FADD
:108D400003F31C42F6D00C49406800240C70016803
:108D50005DF8044B21F00101016093607047064902
:108D6000406800240C7001685DF8044B21F001019B
:108D70000160D360704700BF754E00202DE9F041BF
:108D8000C40023189B00B749CA585268958AADB2EF
:108D9000EFB2FE070B4461D4BE0737D5BFF35F8F38
:108DA0001D7EEDB2012D00F0BB80AF4E138BBFF3E3
:108DB0005F8F231801EB83031D7E022D00F0CE8010
:108DC000231801EB83031D7E032D05D19B7E1BB170
:108DD000737E002B40F01A81938896F918C043F4F3
:108DE00080639380231801EB83031B7E013363456B
:108DF0000AD1B37E00257576002B40F08A8020448E
:108E000001EB800000234375BDE8F081964E17F01A
:108E1000040F96F918C04DD117F0400700F0B2804A
:108E2000178A1D6AFFB205F80C705FFA8CF56F1C8B
:108E300093F818E07BB2DF1CBE4533769C4600F009
:108E40000981271801EB87073F7EBB42CAD105F194
:108E5000020C4FFA8CFC86F818C0C3E71588824EC6
:108E600025F400652D042D0C1580158845F48065CA
:108E700015809D7E00273776002D3DD0757E002D14
:108E800037D0231801EB830301251B7E7576022B57
:108E900003D1138843F400631380231801EB830389
:108EA0009B7D43F001031382204401EB8000037E8D
:108EB000BDE8F0819F7E757E4FF0010E86F81AE0C6
:108EC000002F5CD0002D78D1231801EB83035B7E4B
:108ED000002B00F0A48013880CF1010C4FFA8CFCDD
:108EE00043F4007386F818C013801388DF05FCD4A0
:108EF00078E7DB7DFF2BC4D0231801EB83039D7D36
:108F000005F0FE051582DB7DFF2BCDD0FF233376E8
:108F1000CAE7938823F440731B041B0C93806EE70D
:108F20009B7E514E002B3FF441AF737E002B3FF4EC
:108F30003DAF138823F480631B041B0C1380BFF325
:108F40005F8F138B1388B57643F400731380938877
:108F500096F918C043F48063938043E79B7E002B0F
:108F60003FF42EAF737E002B3FF42AAF138896F99F
:108F700018C023F480631B041B0C138016E0002D23
:108F8000A2D0A8E72D067FF52DAFBCF1FF3F6DD035
:108F9000DD6915F80C5015820CF1010C1D7E4FFA9D
:108FA0008CF39D429C4633767FF41CAF938823F468
:108FB00080631B041B0C938014E71F7ED3F8208072
:108FC0005FFA8CF5AE44022F4FFA8EFE17882DD92A
:108FD00027F480673F043F0C1780178AFFB208F818
:108FE0000C701788D3F820C047F400731380138ADD
:108FF000DBB20CF80E30938805F1020C4FFA8CFCB2
:1090000043F4806386F818C093806EE7938896F9DE
:1090100018C023F480631B041B0C9380E2E61388C2
:10902000012543F48073138075765EE747F400777B
:109030001780178AFFB208F80C70178AD3F82080BF
:1090400005F1030C4FFA8CFCFBB286F818C008F847
:109050000E304AE7978827F480673F043F0C9780DB
:10906000EFE600BF187C002098260020DD7D1582E9
:109070009D7E37761DB91B7E002B7FF415AF93883C
:1090800023F480631B041B0C93800DE730B504466A
:10909000806DA160838923F400531B041B0C838122
:1090A000A37985B013F0040F009108BF0025617902
:1090B00018BF4FF48055ADF804501A0300251B0269
:1090C00003F48063ADF80A50ADF80C50CD07ADF84D
:1090D000083002F4005244BF0423ADF80A30ADF862
:1090E00006204CBF0C2308238A07694648BFADF809
:1090F0000A3019F0FBFFA37913F0080FA36D9A8AC9
:1091000005BF22F00802120442F00802120C9A82F3
:109110009A8942F400529A8105B030BDF8B50468CE
:10912000C4F30D0405460E4604B32F6819F0CCFFB6
:10913000092840F08880454C236923F4407323615B
:10914000236943F400732361236943F0010323611E
:109150003E6019F0B9FF2369092823F00103236158
:1091600071D12B6804332B60002035E0384B394A2D
:1091700093422BD902F58042934226D902F58042D0
:1091800093422AD902F58042934228D902F58032CF
:10919000934226D902F50032934224D902F50032D7
:1091A000934222D902F50032934220D902F50032CF
:1091B00093421ED902F5802293421CD9B3F1016F6C
:1091C0001BD305200FF0F2FFFBE7082419F07CFF0A
:1091D000092814D04FF0FF30F8BD1024F6E718240A
:1091E000F4E72024F2E72824F0E73024EEE73824DF
:1091F000ECE74024EAE74824E8E75824E6E7134F81
:109200003B6923F440733B613B6943F400733B616A
:109210003B6923F0F8033B613B6943F002031C43C5
:109220003C613B6943F480333B6119F04DFF3B697E
:1092300023F002033B613B69092823F0F8033B61FB
:109240003FF473AFC6E76FF00100C5E7003C024092
:1092500000400008FF3F0008F8B504460D468E1890
:109260000027B542206900D1F8BDE368591CE160D0
:10927000234415F8012B1A720429F2D118B9A168F8
:109280002046FFF74BFFC4E90370EAE7002A12DD2E
:1092900070B504460D468E18236820469B68984793
:1092A0000028F9D0236815F8011B1B682046984751
:1092B000B542F1D170BD704703685B6A03B11847CE
:1092C000704703681B6A03B11847704703682DE9AC
:1092D000F041DD691DB12B46BDE8F0411847002A79
:1092E000174611DD04460E460F4400E023689B68D4
:1092F000204698470028F9D0236816F8011B1B6800
:1093000020469847BE42F1D1BDE8F08103689B69D1
:10931000184703685B69184703681B6918470368A7
:10932000DB68184703689B68184703685B68184741
:1093300003681B681847014B1868F9E7F8400020DC
:1093400038B50C46097849B1054601342B682846E2
:109350001B68984714F8011B0029F7D138BD064B4C
:1093600053F820302BB11A689B8851690B4201D108
:109370001383704753837047B089002003682DE939
:10938000F04F03F13F4404F57E04534EA40A012537
:10939000345D04F01F066409032C05FA06F500F09D
:1093A0009580042C00F08D80022C46D08588B5FA7B
:1093B00085F0C0F11F0080B2C40803EB840400F004
:1093C0000700266A80000F27874026EA07062662E4
:1093D000276A01F0030602FA00F0721E3843012AE0
:1093E000C1F3810EC1F3001820624FEA51114FF012
:1093F00000024FF0010C25D94FF0030E0CFA02F0D9
:10940000A84315D150001F680EFA00F4E44327402A
:109410001F60D3F8008006FA00F747EA08071F60CC
:10942000DF683C40DC60DC6801FA00F02043D86073
:109430000132102AE2D1BDE8F08F284C666C35432A
:109440006564B3E74FF003090CFA02F737EA050049
:1094500033D15000D3F800A009FA00F4E4430AEA3B
:10946000040AC3F800A0D3F800B006FA00FA4AEAEA
:109470000B0AC3F800A0D3F808A004EA0A0AC3F84C
:1094800008A0D3F808B00EFA00FA4AEA0B0AC3F8AB
:1094900008A0D3F804A02AEA07075F60D3F804A065
:1094A00008FA02F747EA0A075F60DF683C40DC60C1
:1094B000DC6801FA00F02043D8600132102AC3D1E1
:1094C000B9E7064C266B354325636FE7034C266CE2
:1094D000354325646AE700BF3C6504080038024054
:1094E000036803F13F4202F57E022DE9F04F920A34
:1094F000464DAA5C02F01F0552090124032A04FA12
:1095000005F47ED0042A77D0022A30D001F0030679
:10951000721E012AC1F3810EC1F300188588C1F3C0
:1095200041114FF000024FF0010C25D94FF0030E0E
:109530000CFA02F0A84315D150001F680EFA00F48F
:10954000E44327401F60D3F8008006FA00F747EA9B
:1095500008071F60DF683C40DC60DC6801FA00F04F
:109560002043D8600132102AE2D1BDE8F08F284AAA
:10957000556C2C435464C9E74FF003090CFA02F709
:1095800037EA050033D15000D3F800A009FA00F4FF
:10959000E4430AEA040AC3F800A0D3F800B006FACC
:1095A00000FA4AEA0B0AC3F800A0D3F808A004EABC
:1095B0000A0AC3F808A0D3F808B00EFA00FA4AEA7B
:1095C0000B0AC3F808A0D3F804A02AEA07075F60D3
:1095D000D3F804A008FA02F747EA0A075F60DF68D9
:1095E0003C40DC60DC6801FA00F02043D8600132C6
:1095F000102AC3D1BDE8F08F054A156B2C431463C4
:1096000084E7034A156C2C4314647FE73C65040827
:109610000038024010B50409013C032C17D80E4B4A
:1096200033F8142000F00F0042FA00F313F00103A6
:109630000FD0012303FA00F00138104038F090FFFA
:10964000064A074B125D104403EBC00010BD00201A
:1096500010BD184610BD00BF006704080867040865
:10966000248800202DE9F04F4A484B494B4B4C4C85
:109670004FF0010A4FF002094FF004084FF0080EB6
:109680004FF0100C20274026802530F8022B12F0D6
:10969000010F03D01960A3F804A0083312F0020FE1
:1096A00003D01960A3F80490083312F0040F03D01C
:1096B0001960A3F80480083312F0080F03D0196072
:1096C000A3F804E0083312F0100F03D01960A3F8D8
:1096D00004C0083312F0200F02D019609F800833B5
:1096E00012F0400F02D019609E80083312F0800FF4
:1096F00002D019609D80083312F4807F05D04FF4AA
:10970000807B1960A3F804B0083312F4007F05D001
:109710004FF4007B1960A3F804B0083312F4806F93
:1097200005D04FF4806B1960A3F804B0083312F42D
:10973000006F05D04FF4006B1960A3F804B0083334
:1097400012F4805F05D04FF4805B1960A3F804B079
:10975000083312F4005F05D04FF4005B1960A3F8E2
:1097600004B0083312F4804F05D04FF4804B1960D9
:10977000A3F804B00833D20B04D04FF400421960B0
:109780009A80083301F58061A1427FF47EAFBDE885
:10979000F08F00BF0067040800000240248800200A
:1097A0000010024000B9704703682DE9F04F03F143
:1097B0003F4404F57E04534EA40A0125345D04F0B1
:1097C0001F066409032C05FA06F500F09580042CA9
:1097D00000F08D80022C45D08588B5FA85F0C0F167
:1097E0001F0080B2C40803EB840400F00700266A5F
:1097F00080000F27874026EA07062662276A01F0C5
:1098000003068240701E3A4301282262C1F3810E92
:10981000C1F300184FF000024FEA51114FF0010C54
:1098200025D94FF0030E0CFA02F0A84315D15000D1
:109830001F680EFA00F4E44327401F60D3F800804D
:1098400006FA00F747EA08071F60DF683C40DC6063
:10985000DC6801FA00F02043D8600132102AE2D11E
:10986000BDE8F08F284C666C35436564B4E74FF073
:1098700003090CFA02F737EA050033D15000D3F898
:1098800000A009FA00F4E4430AEA040AC3F800A0BD
:10989000D3F800B006FA00FA4AEA0B0AC3F800A0AF
:1098A000D3F808A004EA0A0AC3F808A0D3F808B05D
:1098B0000EFA00FA4AEA0B0AC3F808A0D3F804A08B
:1098C0002AEA07075F60D3F804A008FA02F747EA1C
:1098D0000A075F60DF683C40DC60DC6801FA00F08A
:1098E0002043D8600132102AC3D1BDE8F08F064C66
:1098F000266B354325636FE7034C266C354325649F
:109900006AE700BF3C6504080038024000B97047B0
:10991000036803F13F4202F57E022DE9F04F920AFF
:10992000464DAA5C02F01F0552090124032A04FADD
:1099300005F47ED0042A77D0022A30D001F0030645
:10994000721E012AC1F3810EC1F300188588C1F38C
:1099500041114FF000024FF0010C25D94FF0030EDA
:109960000CFA02F0A84315D150001F680EFA00F45B
:10997000E44327401F60D3F8008006FA00F747EA67
:1099800008071F60DF683C40DC60DC6801FA00F01B
:109990002043D8600132102AE2D1BDE8F08F284A76
:1099A000556C2C435464C9E74FF003090CFA02F7D5
:1099B00037EA050033D15000D3F800A009FA00F4CB
:1099C000E4430AEA040AC3F800A0D3F800B006FA98
:1099D00000FA4AEA0B0AC3F800A0D3F808A004EA88
:1099E0000A0AC3F808A0D3F808B00EFA00FA4AEA47
:1099F0000B0AC3F808A0D3F804A02AEA07075F609F
:109A0000D3F804A008FA02F747EA0A075F60DF68A4
:109A10003C40DC60DC6801FA00F02043D860013291
:109A2000102AC3D1BDE8F08F054A156B2C4314638F
:109A300084E7034A156C2C4314647FE73C650408F3
:109A40000038024010B1036882885A83704710B111
:109A5000036882881A83704718B10368828809B93D
:109A60005A8370471A83704710B40A4B0A4A1C780D
:109A700001238340234052F8200029B9B3FA83F12F
:109A800049095DF8044BE7E7191C18BF01215DF88F
:109A9000044BE1E7AC890020B089002030B10368B5
:109AA00082881B691A4214BF0120002070472DE9EB
:109AB000F0410B4E346873691C400FD0DFF82480EE
:109AC0000127B4FA84F3C3F11F0307FA03F558F82A
:109AD000230003689847AC437561F2D1BDE8F0817B
:109AE000003C0140EC8900202DE9F0410B4E346828
:109AF00073691C400FD0DFF828800127B4FA84F383
:109B0000C3F11F0307FA03F558F8230003689847C9
:109B1000AC437561F2D1BDE8F08100BF003C01406B
:109B2000EC8900202DE9F0410B4E346873691C402C
:109B30000FD0DFF828800127B4FA84F3C3F11F03A4
:109B400007FA03F558F8230003689847AC4375619A
:109B5000F2D1BDE8F08100BF003C0140EC8900205B
:109B60002DE9F0410B4E346873691C400FD0DFF8CB
:109B700028800127B4FA84F3C3F11F0307FA03F521
:109B800058F8230003689847AC437561F2D1BDE8EB
:109B9000F08100BF003C0140EC8900202DE9F0413C
:109BA0000B4E346873691C400FD0DFF82880012702
:109BB000B4FA84F3C3F11F0307FA03F558F823003E
:109BC00003689847AC437561F2D1BDE8F08100BFEE
:109BD000003C0140EC8900202DE9F0410B4E346837
:109BE00073691C400FD0DFF828800127B4FA84F392
:109BF000C3F11F0307FA03F558F8230003689847D9
:109C0000AC437561F2D1BDE8F08100BF003C01407A
:109C1000EC8900202DE9F0410B4E346873691C403B
:109C20000FD0DFF828800127B4FA84F3C3F11F03B3
:109C300007FA03F558F8230003689847AC437561A9
:109C4000F2D1BDE8F08100BF003C0140EC8900206A
:109C5000084A094808B5536C43F480435364002113
:109C6000402239F049F8054B4FF0FF321A60C3F833
:109C7000032008BD00380240EC8900202C8A002017
:109C800010B58B680160044698470022FF2301212C
:109C9000A2736373217310BD03681B6A184770B405
:109CA0004E1C0568C2728672AC69A44670BC6047DF
:109CB0002DE9F041044618460D4616461F4637F07A
:109CC00031FF2844A0722068E672294645693B4668
:109CD00032462046AC46BDE8F0416047036810B507
:109CE00004461B689847236820469B689847A37BD7
:109CF0000133A37310BD03681B69184710B50368CF
:109D000004469B689847FF2301226373227310BDAA
:109D10000B4B984211D0A3F57843984202D04FF0F4
:109D2000FF3070470122074B03EB02135A890132BF
:109D300092B25A81588980B270470022F3E700BF7F
:109D40000030014070360020F0B5876983B00646C8
:109D500017B13B68BA885A837069DFF8A8E0838935
:109D6000C3244FF47A734FF0060C6D464FF6FF7123
:109D70000EF1010E03E0013B9BB28B4220D0028921
:109D80009207F8D5A3B283814FF47A7302E0A3B2AD
:109D90008B4215D00289D20703F1FF34F7D58289AF
:109DA00092B20DB12A700135BCF1000F0BD00CF14D
:109DB000FF3CFF24BEF1000FE1D09EF80040D7E742
:109DC000FFF7A6FFB76917B13B68BA881A839DF8F9
:109DD00005009DF801509DF802109DF803409DF884
:109DE00004209DF8063041EA052143EA002342EAB7
:109DF00004220120A6F84410A6F84620A6F8483010
:109E000003B0F0BD04360408F8B584894FF6FF7638
:109E10004FF47A7433B319B30F78013101E0B442CF
:109E200018D00589013CAD07A4B2F8D5BCB2848135
:109E30004FF47A7402E0BCB2B4420BD00589ED074E
:109E400004F1FF37F7D58589ADB20AB1157001323B
:109E5000013BDFE7FFF75CFF003018BF0120F8BDD2
:109E6000FF27DEE70120F8BD08B540F2E93300E046
:109E7000A3B10289013B12F0020F9BB2F8D089B264
:109E8000818140F2E93300E043B10289013B12F0E5
:109E9000010F9BB2F8D08089C0B208BDFFF738FF30
:109EA000C0B208BD427A4AB110B5044604F10A01B5
:109EB000D0E9003098470023637210BD7047437AA1
:109EC0005A1C0344D2B242729972037A93420AD85E
:109ED0004AB110B5044604F10A01D0E900309847B0
:109EE0000023637210BD704728B1302801D031289B
:109EF00002D129B3002070473228FAD03328F8D095
:109F00003428F6D03528F4D02028F2D02128F0D0FB
:109F10001028EED01128ECD01228EAD01328E8D06F
:109F20001428E6D01528E4D0162803D1B1FA81F020
:109F3000400970471728DDD1B1FA81F04009704718
:109F400001207047302829D0312829D0322829D043
:109F5000332829D0342829D0352829D020282BD0BF
:109F600021282BD0102825D0112829D0122829D01B
:109F7000132829D0142829D0152829D0162805D02F
:109F8000172808BF0F2302D0002070470E23114A64
:109F900003EB4303134493F87A0070470023F6E77A
:109FA0000123F4E70223F2E70323F0E70423EEE7BB
:109FB0000523ECE70823EAE70623E8E70723E6E7BB
:109FC0000923E4E70A23E2E70B23E0E70C23DEE7BB
:109FD0000D23DCE794350408024A136823EA0000E5
:109FE000106070476C830020F8B5174D2B78A82BB4
:109FF00028D16B78BE2B25D1022229464FF6FF705F
:10A00000FEF73FFA114FAC1C22884AB1A618BE4297
:10A0100018D2052A16D92146FEF733FA3446F3E75B
:10A0200021460222FEF72DFA0222A118FEF729FA94
:10A030000634074B641B1C8041F60F53C31A584269
:10A040005841F8BD0020FCE70040000800800008EF
:10A05000DA3400202DE9F04FDFF84C914D4F8BB0F2
:10A060000326A7EB09071022002106A838F044FEBA
:10A07000CDE90497484B1A69002A04DA474A5A6026
:10A0800002F188325A6001228DF82420F322DA602E
:10A09000434B444C1B88ADF800300222694604A8AB
:10A0A000FFF7DAF8022269464FF6FF70FEF7E9F98A
:10A0B000DFF8F8A080464FF0000B544539D30AACC6
:10A0C000002524F8245D0222214604A8FFF7C4F8E5
:10A0D000022221464046FEF7D4F940BAC043ADF80B
:10A0E0000800022202A904A8FFF7B6F8079878B181
:10A0F00006ABC0F104022946184438F0FDFD08986B
:10A1000018B9069904A8FFF709F8002308900793E7
:10A110009DF82430089A23B11F490B6943F000438E
:10A120000B61013E2DD0002A9DD1FFF75DFF50B39A
:10A130002CE065888DF80DB0C5F30B05AB1DADF8AF
:10A1400008302388C3F30B02ADF80A201B0B06224C
:10A1500002A904A88DF80C30FFF77EF8062202A9A8
:10A160004046FEF78EF9616880462A4604A8FFF74C
:10A1700073F8616840462A46FEF783F91434804636
:10A180009BE7002AD1D005200FF010F80BB0BDE8F6
:10A19000F08F00BF00800008003C024023016745AB
:10A1A0003C360408A001000800400008A006000892
:10A1B0000378202B024600F10100F9D0092BF7D0DB
:10A1C0002D2B00F0A4802B2B03BF5378B7EE000A91
:10A1D0000246B7EE000AA3F13001C8B209289FED8C
:10A1E000577A10D8F2EE046A07EE901AF8EEE77A82
:10A1F00012F8013FE7EE267AA3F13001C8B2092830
:10A20000B0EE677AF0D92E2B63D003F0DF03452B35
:10A2100002D020EE070A704710B451782D294FD094
:10A220002B2979D0A1F13003092B02F101027AD850
:10A230000024002303EB830301EB430312F8011F07
:10A24000A1F130000928A3F13003F3D9B3F59A7FC7
:10A250001A4628BF4FF49A72072B6CD9DFED386A83
:10A260001346F7EE007A083B072B67EEA67AFAD87A
:10A2700002F00702DAB1F2EE046A012A67EEA67A6A
:10A2800015D0022A67EEA67A11D0032A67EEA67AC5
:10A290000DD0042A67EEA67A09D0052A67EEA67AC1
:10A2A00005D067EEA67A062A18BF67EEA67A002CBC
:10A2B0003BD087EE277A5DF8044B20EE070A704703
:10A2C0009178A1F13003092B02F1020230D8012468
:10A2D000AFE75378A3F13001C8B2092802F10102B7
:10A2E00093D8F2EE046AF0EE665A07EE901AF8EE92
:10A2F000E77A12F8013F87EEA66AA3F13001C8B2EF
:10A30000092866EEA56A37EE067AEED97DE753781E
:10A31000BFEE000A02465EE79178A1F13003092BF7
:10A3200002F1020284D9F7EE007A27EE277AC2E71B
:10A33000F7EE007ABDE7F7EE007A9BE70000000039
:10A3400020BCBE4CB5EEC00ADFED317AF1EE10FA5A
:10A35000CCBF30EE270A30EE670ADFED2E7A20EE12
:10A36000270A30B5FDEEC07A87B017EE904A054651
:10A3700084EAE470002303A9A0EBE470CDE9003384
:10A38000029336F077FE002CACBF20232D2303A8C8
:10A390008DF8003037F0C6FB012803A924D002282D
:10A3A0002DD0032805BF3023684668468DF801305C
:10A3B00038F0AAFC684637F0B5FB0338C4B2224631
:10A3C0006946284638F0D6FC00232B55284637F03E
:10A3D000A9FB2E22431C2A540DEB0401E81838F087
:10A3E000AFFC284607B030BD302368468DF80130F9
:10A3F0008DF802308DF8033038F086FCDAE7302330
:10A4000068468DF801308DF8023038F07DFCD1E7D8
:10A410006F12033A00007A44F8B50646154608461E
:10A42000B6FBF2F434B905FB14640C4B1B5D00F869
:10A43000013BF8BDB4FBF2F75FB905FB1747074BCB
:10A4400005FB1464DA5D00F8012B1B5D00F8013B8D
:10A45000F8BD3846FFF7E0FFEFE700BFA06D040846
:10A460000F4B2DE93048D3E9004554EA05020AD1E3
:10A47000034640F2011200201880988098715A809B
:10A480001881BDE83088074B1A6814EB020B45F1C0
:10A49000000C5A466346FDF775FE0120BDE8308882
:10A4A00008730020E489002030B403888278164DB8
:10A4B000C478A3F2B27303F0030101EB4101013A46
:10A4C00002EB810205EB4202611E158A027940F21D
:10A4D000B5549B0804FB03132B4403EB430302EB2B
:10A4E000C303427981790089C3EB031302EB830331
:10A4F000C3EB031301EB83034FF47A720021C2FB19
:10A50000030130BC704700BF9435040802B370B437
:10A510008E1803E0121B14D1B14215D010F8012B94
:10A52000A2F14103192B11F8013BA3F1410598BF9A
:10A530002032192D03F12004ECD9D21A01D1002BBD
:10A54000EAD1104670BC70470022104670BC7047BC
:10A55000104670474FF0FF32FFF7D8BFA0F16103FC
:10A56000192B98BF20387047A0F14103192B98BFD1
:10A5700020307047202805D0093804288CBF0020DF
:10A580000120704701207047613819288CBF0020D6
:10A5900001207047413819288CBF002001207047E6
:10A5A000303809288CBF002001207047A0F130030B
:10A5B000092B07D920F02000413819288CBF002032
:10A5C000012070470120704730B402681146531CC7
:10A5D000036011F8024B0160D31C5178036093783B
:10A5E000151D05601B0443EA0123D078234343EA89
:10A5F000006030BC70470368591C1A46016012F8AD
:10A60000021B0260587841EA0020704703685A1C18
:10A6100002601878704738B504460068154638F06F
:10A6200051FA22682A44226038BD036810B40A0E29
:10A630005C1C04601A7003680A0C5C1C04601A70CD
:10A6400003680A0A5C1C04601A7003685A1C0260E2
:10A6500019705DF8044B7047036810B40A0A5C1C5B
:10A6600004601A7003685A1C026019705DF8044B8C
:10A67000704703685A1C026010B4197003680A0A14
:10A680005C1C04601A7003680A0C5C1C04601A707D
:10A690000368090E5A1C026019705DF8044B70477C
:10A6A00003685A1C026019700368090A5A1C026088
:10A6B000197070472DE9F043002489B006460D4615
:10A6C0001F46A04605E025290CD030460134A84796
:10A6D000039A531C039311780029F4D1204609B042
:10A6E000BDE8F083931CCDE903385078302842D080
:10A6F000A0F13003DBB2092B4FF0000945D96C28DB
:10A700002AD0642873D019D9732858D063D97528F2
:10A7100040F0828007F1040C386805AB00220A2162
:10A720006746FDF7E3FC05AB049A009329464B46C8
:10A730003046FDF7E2FD039A0444CAE725283CD0E1
:10A7400051D958286BD06328C2D139783046A847F0
:10A7500004370134039ABCE7039B5A1C03921B780D
:10A76000642B52D016D8252B27D064D9582B18D05B
:10A77000632BEAD0ADE7D31C03939078A0F13003AC
:10A78000DBB2092B4FF00109B9D804AA03A934F0B0
:10A79000DDF9B4E7732B12D051D9752B2DD0782B5E
:10A7A00097D1A3F15802B2FA82F23868520905AB88
:10A7B00010210437FDF79AFCB5E7252185E73B68B2
:10A7C000049A0093294600233046FDF796FD04378E
:10A7D0000444039A7DE76E287FF47AAF039A3B68BE
:10A7E00004371C6075E700283FF478AF70E73868DD
:10A7F00005A9FDF745FC043795E7386805AB00224D
:10A800000A21FDF773FC04378DE73B1D386805A965
:10A810001F46FDF735FC86E778287FF459AFA0F195
:10A820005802B2FA82F23868520905AB1021FDF7DE
:10A830005DFC043777E7002B3FF450AF49E76E2B00
:10A84000CDD046E70EB400B584B005AB019053F807
:10A85000042B0649039301A8FFF72CFF019B00225C
:10A860001A7004B05DF804EB03B07047F182000881
:10A870002DE9F04707468CB01E469246002A5DD16E
:10A88000154614460A8840F2B1739A4236D98B783D
:10A89000581E0B2832D891F803C00CF1FF301E2847
:10A8A0002CD891F804E0BEF1170F27D891F8059045
:10A8B000B9F13B0F22D888793B281FD8B1F808801E
:10A8C000B8F57A7F1AD24FF001085EBB098904916E
:10A8D000002CB4BF2D212B21002CB8BF6442CDE940
:10A8E0000290CDE905140795CDE900CE38462B49F5
:10A8F000FFF7A8FF40460CB0BDE8F08700232849C9
:10A90000ADF828304FF0010C18468DF82A30ADF81C
:10A910002C3099469E461A4698460991634609A9E5
:10A92000002ED3D0CDE90290CDE900CE38461D49A6
:10A93000FFF788FF40460CB0BDE8F0871A4C84FB57
:10A940000234A318D417C4EB6314C4EB0415A2EBB0
:10A9500085052DB2002D0846B8BF6D42FFF7A4FD56
:10A960004FF47A7200238046894637F0A9FD3C23D4
:10A970000AFB030A4FF47A7200234046494637F037
:10A980009FFD4FF47A7192B20023C1FB0A2309A8FC
:10A99000FDF7F8FB24B209A974E700BFE86D0408CD
:10A9A00000000101C86D0408898888880FB430B59B
:10A9B00083B006AB0A490B4853F8042B09680068BA
:10A9C0000193FFF777FE084C05462068FEF7A1FCCF
:10A9D0000028FAD0284603B0BDE8304004B07047E4
:10A9E000E47B0020E87B0020F8400020DFED2E7A99
:10A9F000B4EEE70AF1EE10FA4ADDDFED2C6A9FEDC6
:10AA00002C7A01E0B0EE670AB4EEC70AF1EE10FA54
:10AA100070EE667AF6DC9FED277AF4EEC77AF1EEF7
:10AA200010FA3ED5DFED216A9FED237A01E0F0EECA
:10AA3000407AF4EEC77AF1EE10FA37EEA60AF6D4B1
:10AA4000DFED1E7AB4EEE70AF1EE10FA14DDDFED69
:10AA5000167A37EEC00A60EE006A9FED196A9FED24
:10AA6000197ADFED197AA6EE867A20EE266AE6EEEE
:10AA7000877AA6EE270A7047DFED147AB4EEE70A6C
:10AA8000F1EE10FA44BFDFED0B7A37EEC00AE2E7D1
:10AA90009FED087AF0EE407AF4EEC77AF1EE10FA04
:10AAA000C0D4B0EE670ACBE7DB0F4940DB0FC940EB
:10AAB000E4CB1641DB0F49C0E4CB16C1DB0FC93F25
:10AAC00092E741B99730083C15A82ABEDB0FC9BFF1
:10AAD00080EAE073A3EBE0738B4205DB002801DD25
:10AAE000401A704702D170470020704708447047F1
:10AAF000F0EEC07AB0EEE07AB4EEE77AF1EE10FA5A
:10AB0000B4BFB0EE676AB0EE476AB5EE406AF1EEE8
:10AB100010FA46D0B4EEE77AF1EE10FA8CBFF0EE00
:10AB2000675AF0EE475AC5EE866A9FED1F3A9FEDD1
:10AB30001F6A9FED1F4A9FED1F5ADFED1F3ADFEDA1
:10AB40001F4ADFED1F5AA6EEC36AE6EEA34AA6EE41
:10AB5000864AB7EE006AA6EE845AA6EEA46AE6EE2E
:10AB6000855AC5EE866AB4EEE77AF1EE10FA48BF70
:10AB7000DFED147AF5EEC00A48BF77EEE66AF1EE33
:10AB800010FA48BFDFED107AB5EEC00A48BF77EE85
:10AB9000E66AF1EE10FA48BFF1EE666AB0EE660AB8
:10ABA0007047DFED076ADEE739094E3DE3B59E3EAB
:10ABB00088FA163E45FE7F3F99FB243F69A2163E68
:10ABC000A7DFA834DB0FC93FDB0F4940DFED317A47
:10ABD00030EE277AFDEEC76A16EE903A2033402B0E
:10ABE00002D99FED2D0A7047B4EEE70AF1EE10FA94
:10ABF0004DDD9FED2A6ADFED2A6A01E0B0EE677A4B
:10AC0000B4EEE67AF1EE10FA77EE467AF6DC9FEDD6
:10AC1000257AF4EEC77AF1EE10FA35D5DFED1F6A2A
:10AC20009FED217A01E0F0EE407AF4EEC77AF1EE82
:10AC300010FA37EEA60AF6D4DFED167AB4EEE70A7C
:10AC4000F1EE10FA1BDCDFED197AB4EEE70AF1EE53
:10AC500010FA44BFDFED137A37EEC00A60EE006AE7
:10AC60009FED136A9FED137ADFED137AA6EE867AD5
:10AC700020EE266AE6EE877AA6EE270A7047DFED19
:10AC80000F7A37EEC00AE9E7B0EE670AD4E7F0EED4
:10AC9000477ABCE7DB0FC93F00000000DB0FC9406B
:10ACA000E4CB1641DB0F49C0E4CB16C1DB0FC9BFB3
:10ACB00092E741B99730083C15A82ABEDB0F4940FE
:10ACC000FDEEC07A17EE903A2033402B45D8DFEDE9
:10ACD0002D7AB4EEE70AF1EE10FA4DDDDFED2A6AC7
:10ACE0009FED2A7A01E0B0EE670AB4EEC70AF1EEF2
:10ACF00010FA70EE667AF6DC9FED257AF4EEC77AEC
:10AD0000F1EE10FA3BD5DFED206A9FED227A01E0EB
:10AD1000F0EE407AF4EEC77AF1EE10FA37EEA60ABA
:10AD2000F6D4DFED1D7AB4EEE70AF1EE10FA17DD86
:10AD3000DFED147A37EEC00A60EE006A9FED176A05
:10AD40009FED177ADFED177AA6EE867A20EE266A57
:10AD5000E6EE877AA6EE270A70479FED130A704742
:10AD6000DFED127AB4EEE70AF1EE10FA44BFDFED40
:10AD7000087A37EEC00ADFE7F0EE407ABCE7B0EEC3
:10AD8000670ACEE7DB0F4940DB0FC940E4CB164131
:10AD9000DB0F49C0E4CB16C1DB0FC93F92E741B9D5
:10ADA0009730083C15A82ABE00000000DB0FC9BF81
:10ADB00007EE901AF8EE677A9FED837A27EE800A05
:10ADC00020EE070AFDEEC07A17EE903A2033402BB2
:10ADD00000F28180DFED7D7AB4EEE70AF1EE10FA41
:10ADE00040F3E680B0EE407A9FED796ADFED796A54
:10ADF00001E0B0EE677AB4EEE67AF1EE10FA77EEA3
:10AE0000467AF6DC9FED747AF4EEC77AF1EE10FA2A
:10AE100040F1D1809FED6E6ADFED706A01E0F0EEE7
:10AE2000477AF4EEE67AF1EE10FA37EE867AF6D447
:10AE3000DFED6B7AB4EEE77AF1EE10FA40F3A7801B
:10AE4000DFED627A37EEC77A27EE076ADFED655AE3
:10AE5000DFED657ADFED656A9FED655AE6EE257AEE
:10AE600067EE065AE6EE276AF7EE007AA5EEA67AB6
:10AE7000F0EE675AE7EE055AE7EE457A87EEA55AF7
:10AE8000DFED577A30EE277AFDEEC76A16EE903A7C
:10AE90002033402B24D99FED577AF6EE006AB7EEA7
:10AEA000006AF7EE004AC4EEA57A0023836143618D
:10AEB0000362C36180ED045A67EEA66A27EE866AD4
:10AEC00027EE877AC0ED006AC0ED026A80ED016A64
:10AED00080ED037A7047B7EE005AF0EE455ACFE79F
:10AEE000B4EEE70AF1EE10FA6BDD9FED396ADFEDA3
:10AEF000396A01E0B0EE677AB4EEE67AF1EE10FA64
:10AF000077EE467AF6DC9FED347AF4EEC77AF1EE0E
:10AF100010FA53D59FED2E6ADFED306A01E0F0EEB6
:10AF2000477AF4EEE67AF1EE10FA37EE867AF6D446
:10AF3000DFED2B7AB4EEE77AF1EE10FA33DCDFEDD9
:10AF40002E7AB4EEE77AF1EE10FA44BFDFED227A02
:10AF500037EEC77A27EE076ADFED224ADFED226A75
:10AF6000DFED227AE6EE246A67EE064AE6EE267AFE
:10AF7000B7EE006AA4EEA77AF6EE006A36EE476AEC
:10AF8000F8EE007A27EE277A66EE266A89E7DFED8B
:10AF90001A7AB4EEE77AF1EE10FA44BFDFED0E7ADA
:10AFA00037EEC77A50E7DFED097A37EEC77AD1E797
:10AFB000F0EE407A26E7B0EE677A39E7B0EE677ACE
:10AFC000B6E7F0EE477A9EE727D4D236DB0F49404A
:10AFD000DB0FC940E4CB1641DB0F49C0E4CB16C1FF
:10AFE000DB0FC93F92E741B99730083C15A82ABE4C
:10AFF000F304353F00000000DB0FC9BF70B40668E2
:10B000008E4217D90139751E002311F8014F08220D
:10B01000634013F0800F4FEA430318BF83F0D5035A
:10B02000013ADBB2F5D18D42EFD1721C0260337070
:10B0300070BC7047721C00230260337070BC704794
:10B0400010B44C09012250F8243001F01F0102FA1B
:10B0500001F10B4340F824305DF8044B70474B0975
:10B0600001F01F0150F82320012303FA01F11142DE
:10B0700014BF1846002070472DE9F84FDFF8B4A23E
:10B08000A849DAF8003001220A7013B11A689B88C7
:10B09000538340F2E933A44902E0002B00F087819A
:10B0A0000A89013B12F0020F9BB2F6D005238B8177
:10B0B00040F2E9339C4902E0002B00F078810A89D4
:10B0C000013B12F0010F9BB2F6D08B89964840F2FB
:10B0D000E93302E0002B00F08E810289013B12F07F
:10B0E000020F9BB2F6D0002383818F4940F2E933EF
:10B0F00002E0002B00F07F810A89013B12F0010F72
:10B100009BB2F6D08B89884840F2E93302E0002BED
:10B1100000F06D810289013B12F0020F9BB2F6D064
:10B1200006238381804940F2E93302E0002B00F0DE
:10B130005E810A89013B12F0010F9BB2F6D08B8928
:10B14000794840F2E93302E0002B00F04C8102899B
:10B15000013B12F0020F9BB2F6D0002383817249AB
:10B1600040F2E93302E0002B00F03D810A89013B07
:10B1700012F0010F9BB2F6D08B896C4B6A4C93F89E
:10B180001B8040F2E93348F0010102E0002B00F09F
:10B1900026812289013B12F0020F9BB2F6D00423D4
:10B1A000A381614840F2E93302E0002B00F01781EF
:10B1B0000289013B12F0010F9BB2F6D083895A4CF1
:10B1C00040F2E93302E0002B00F005812289013BC7
:10B1D00012F0020F9BB2F6D089B25348A18140F21F
:10B1E000E93302E0002B00F0F6800289013B12F007
:10B1F000010F9BB2F6D08389DFF83CB1BBF8003079
:10B20000002B45D0DFF83491494F47494E4607257A
:10B2100017F8014F40F2E93302E0002B00F0C38041
:10B220000889013B10F0020F9BB2F6D08D8140F2ED
:10B23000E93302E0002B00F0B6800889013B10F0F2
:10B24000010F9BB2F6D08B8940F2E93302E0002B6C
:10B2500000F0A5800889013B10F0020F9BB2F6D0E8
:10B26000A4B28C8140F2E93302E0002B00F0978019
:10B270000889013B10F0010F9BB2F6D08B893B7817
:10B2800006F8013BBBF80000A6EB09039842BFDCBF
:10B29000254840F2E93302E0002B00F09880028953
:10B2A000013B12F0020F9BB2F6D0072383811E49A7
:10B2B00040F2E93302E0002B00F089800A89013B6B
:10B2C00012F0010F9BB2F6D08B89174840F2E93398
:10B2D00001E0002B77D00289013B12F0020F9BB2F4
:10B2E000F7D0FF238381104940F2E93301E0002BBE
:10B2F00069D00A89013B12F0010F9BB2F7D08B890C
:10B30000094840F2E93301E0002B58D00289013BA3
:10B3100012F0020F9BB2F7D004238381024940F25E
:10B32000E9330FE086830020003800409826002093
:10B33000337D00200488002020070020B426002050
:10B34000002B3CD00A89013B12F0010F9BB2F7D0D1
:10B350008B892B4840F2E93300E063B30289013B5B
:10B3600012F0020F9BB2F8D01FFA88F82449A0F817
:10B370000C8040F2E93300E0EBB10A89013B12F0A6
:10B38000010F9BB2F8D08B89DAF8003013B11A683C
:10B390009B8813831B4A00231370BDE8F88F08466F
:10B3A000FEF7B6FC6BE70846FEF7B2FC4CE7144824
:10B3B000FEF7AEFC8AE61248FEF7AAFCE4E7104866
:10B3C000FEF7A6FCC5E70E48FEF7A2FC98E70C487E
:10B3D000FEF79EFC79E70A48FEF79AFC0CE708485E
:10B3E000FEF796FCEBE60648FEF792FCC5E604483D
:10B3F000FEF78EFCA4E60248FEF78AFC83E600BF57
:10B4000000380040868300202DE9F041A34C2368DA
:10B4100013B11A6899885183A14A1278012A00F061
:10B420009381C0F07781022A00F066819D4D2A78D1
:10B4300012F0400F0CBF4FF4C3724FF4F0729A4EEB
:10B44000328013B11A689B885383984910274FF0B4
:10B45000010840F2E93302E0002B00F053810A8931
:10B46000013B12F0020F9BB2F6D0BBB28B8140F2CF
:10B47000E93302E0002B00F045810A89013B12F01C
:10B48000010F9BB2F6D08B8940F2E93302E0002B2A
:10B4900000F03C810A89013B12F0020F9BB2F6D00A
:10B4A000A1F80C8040F2E93302E0002B00F02E817D
:10B4B0000A89013B12F0010F9BB2F6D08B8901374C
:10B4C000202FC6D123681BB11A689B88138353832E
:10B4D0002978764D40F2E93302E0002B00F03E81FE
:10B4E0002A89013B12F0020F9BB2F6D00023AB81F8
:10B4F0006E4840F2E93302E0002B00F02F81028910
:10B50000013B12F0010F9BB2F6D08389674D40F2E8
:10B51000E93302E0002B00F025812A89013B12F07B
:10B52000020F9BB2F6D089B26048A98140F2E9339C
:10B5300002E0002B00F016810289013B12F0010F9E
:10B540009BB2F6D083895A4B584D197840F2E933B3
:10B5500002E0002B00F00A812A89013B12F0020F61
:10B560009BB2F6D00223AB81504840F2E93302E0AF
:10B57000002B00F0FB800289013B12F0010F9BB20F
:10B58000F6D08389494D40F2E93302E0002B00F008
:10B59000F1802A89013B12F0020F9BB2F6D089B2EA
:10B5A0004248A98140F2E93302E0002B00F0E2803A
:10B5B0000289013B12F0010F9BB2F6D083893D4B0B
:10B5C0003A4D197840F2E93302E0002B00F0D680C2
:10B5D0002A89013B12F0020F9BB2F6D00323AB8104
:10B5E000324840F2E93302E0002B00F0C7800289C4
:10B5F000013B12F0010F9BB2F6D083892B4D40F234
:10B60000E93302E0002B00F0BD802A89013B12F0F3
:10B61000020F9BB2F6D089B22448A98140F2E933E7
:10B6200002E0002B00F0AE800289013B12F0010F16
:10B630009BB2F6D08389204B1C4DD97E40F2E93372
:10B6400041F0040102E0002B00F0A0802A89013BB8
:10B6500012F0020F9BB2F6D00423AB81134840F2E4
:10B66000E93302E0002B00F091800289013B12F0E7
:10B67000010F9BB2F6D083890C4D40F2E93301E013
:10B68000002B67D02A89013B12F0020F9BB2F7D042
:10B6900089B20648A98140F2E93311E0048800200C
:10B6A00018880020080900202007002000380040EA
:10B6B0001F8800202088002098260020002B49D0D9
:10B6C0000289013B12F0010F9BB2F7D083892368F6
:10B6D00013B11A689B881383304C3288304800219C
:10B6E00037F00AFB23782BB12E4B1B78002B51D05F
:10B6F00000232370BDE8F0812B4D08222A704FF4FF
:10B70000C3729CE60846FEF703FBBDE60846FEF75B
:10B71000FFFAD4E6A0212548FEF7A6FB0021234826
:10B72000FEF7A2FB00F00603022B08D000F0050094
:10B73000012804D11C4D236848222A7007E01A4DC5
:10B74000236808222A70DAE7174D48222A704FF43E
:10B75000F07274E61548FEF7DBFAB8E71348FEF717
:10B76000D7FAD3E61148FEF7D3FAECE60F48FEF716
:10B77000CFFA07E70D48FEF7CBFA20E70B48FEF7B4
:10B78000C7FA3BE70948FEF7C3FA54E70748FEF754
:10B79000BFFA71E7FFF770FCAAE700BF00000020C6
:10B7A000B4260020868300200809002000380040CD
:10B7B0002DE9F84F6D4B6E491B6801220A7013B1D9
:10B7C0001A689B88538380216A48FEF74DFB00214D
:10B7D0006848FEF749FB654B1B6813B11A689988E6
:10B7E0001183654C654D22782F68824240F0858038
:10B7F000634A644E1278002A3DD0B6F80622624BA6
:10B80000DFF89081B3F800E002F1640C1FFA8CFCC1
:10B8100000234FF0050B4FF0060A4FF0070902E036
:10B82000624500F08580B41818F80200217F81423B
:10B8300002F1010503F1050110D07718F118207706
:10B84000140A81F808B281F80AA281F80B2281F863
:10B850000C9281F80942063387F80802AAB27245B1
:10B86000DED30022A6F80622002B4AD1404A00234C
:10B870001370BDE8F88FD6F8FC21BA1AB2F57A7FBA
:10B88000BBD913B11A689B885383A0213948FEF7AE
:10B89000EBFA00213748FEF7E7FA344B1B6813B187
:10B8A0001A689B881383DFF8F08098F80030142B17
:10B8B0000FD12378354A03F04003002B00F0070135
:10B8C0000CBF4FF00D0C4FF0100C13805180A2F8FC
:10B8D00006C041072FD400F0050001282FD048B939
:10B8E00023785B0606D5D6F800222B685AB39B1A3C
:10B8F000642B2BD8C6F8FC717FE7FFF785FD214E3E
:10B900007BE71A4A126812B1116892884A830022B2
:10B910001F491848FEF778FA144B1B68002BA5D076
:10B920001A689B881383124A00231370BDE8F88FAE
:10B93000A6F8062298E70023C6F80032DAE7237853
:10B940005A06D0D5D6E7C6F80032D3E7FFF75CFD3C
:10B9500098F80030142BCDD1B6F804320B4A0133DD
:10B960009BB2A6F804329380C4E700BF048800208D
:10B97000868300200038004008090020E489002068
:10B98000188800209826002020070020108800201A
:10B99000A0280020347D00200D8800202DE9F047EC
:10B9A000A24F3B7803B1FEE7DFF89082D8F8003071
:10B9B00001223A7013B11A689B8853839C4B012271
:10B9C0008A461A70014640F2E9339A4802E0002B99
:10B9D00000F088810289013B12F0020F9BB2F6D081
:10B9E0000023838140F2E933924802E0002B00F00B
:10B9F00079810289013B12F0010F9BB2F6D0838955
:10BA00008C4C40F2E93302E0002B00F07F81228968
:10BA1000013B12F0020F9BB2F6D00023A3818548B0
:10BA200040F2E93302E0002B00F070810289013B13
:10BA300012F0010F9BB2F6D083897E4C40F2E933BD
:10BA400002E0002B00F05E812289013B12F0020F20
:10BA50009BB2F6D00923A381764840F2E93302E095
:10BA6000002B00F04F810289013B12F0010F9BB2C5
:10BA7000F6D083896F4C40F2E93302E0002B00F0EE
:10BA80003D812289013B12F0020F9BB2F6D089B2B0
:10BA90006848A18140F2E93302E0002B00F02E81DA
:10BAA0000289013B12F0010F9BB2F6D08389624EEE
:10BAB00060490AF1FF3A00254FF00A0940F2E933E4
:10BAC00002E0002B00F0F5800A89013B12F0020F22
:10BAD0009BB2F6D0A1F80C9040F2E93302E0002BC3
:10BAE00000F0E7800A89013B12F0010F9BB2F6D00B
:10BAF0008B8940F2E93302E0002B00F0DE800A89F6
:10BB0000013B12F0020F9BB2F6D0ABB28B8140F238
:10BB1000E93302E0002B00F0D0800A89013B12F0EB
:10BB2000010F9BB2F6D08B891AF8014F40F2E9332E
:10BB300002E0002B00F0C5800A89013B12F0020FE1
:10BB40009BB2F6D00B238B8140F2E93302E0002B4D
:10BB500000F0B7800A89013B12F0010F9BB2F6D0CA
:10BB60008B8940F2E93302E0002B00F0AE800A89B5
:10BB7000013B12F0020F9BB2F6D0A4B28C8140F2CE
:10BB8000E93302E0002B00F0A0800A89013B12F0AB
:10BB9000010F9BB2F6D08B89336833B11A689B884A
:10BBA0005069034214BF538313830135362D85D169
:10BBB00040F2E9331F4802E0002B00F09B8002892D
:10BBC000013B12F0020F9BB2F6D008238381194982
:10BBD00040F2E93302E0002B00F08C800A89013B3F
:10BBE00012F0010F9BB2F6D08B89124840F2E93374
:10BBF00001E0002B7AD00289013B12F0020F9BB2C8
:10BC0000F7D0A02383810B4940F2E93301E0002BF8
:10BC10006CD00A89013B12F0010F9BB2F7D08B89DF
:10BC20000449A02440F2E9330CE000BF86830020E1
:10BC30008783002000380040B0890020048800205D
:10BC4000002B46D00A89013B12F0020F9BB2F7D0BD
:10BC50008C8140F2E93301E0002B3AD00A89013BA4
:10BC600012F0010F9BB2F7D08B8940F2E93300E06C
:10BC70009BB30A89013B12F0020F9BB2F8D000235C
:10BC80008B8140F2E93300E03BB30A89013B12F0BB
:10BC9000010F9BB2F8D08889C0B28306C2D4D8F80D
:10BCA000003013B11A689B88138300233B70BDE8F2
:10BCB000F0870846FEF72CF81BE70846FEF728F841
:10BCC00032E70846FEF724F84BE70846FEF720F86F
:10BCD00062E70846FEF71CF8C7E70846FEF718F8C3
:10BCE000C0B2DAE70B48FEF713F889E60948FEF719
:10BCF0000FF895E70748FEF70BF876E70548FEF7DB
:10BD000007F8D4E60348FEF703F8B3E60148FDF769
:10BD1000FFFF92E6003800401378C3B130B41E2410
:10BD20000B4D14FB01012944801A84181D2C07DCDB
:10BD300001F8013B12F8013F002BF6D130BC7047EF
:10BD400012F8013F0131002BEFD130BC7047704732
:10BD5000347D002070B5264CC1F10301236841EA0F
:10BD60008006F6B213B11A689B8853832149B6B294
:10BD7000102540F2E93301E0002B31D00A89013B64
:10BD800012F0020F9BB2F7D0ABB28B8140F2E933D5
:10BD900000E02BB30A89013B12F0010F9BB2F8D0EF
:10BDA0008B8940F2E93300E0F3B10A89013B12F0DC
:10BDB000020F9BB2F8D08E8140F2E93300E09BB1D4
:10BDC0000A89013B12F0010F9BB2F8D08B89013533
:10BDD000202DCED1236813B11A689B88138370BDC0
:10BDE0000846FDF795FFDCE70846FDF791FFEEE713
:10BDF000048800200038004038B5284BDC7E00283D
:10BE000041D104F0F7042649DC760B6813B11A68B7
:10BE10009B88538340F2E933224801E0002B39D05C
:10BE20000289013B12F0020F9BB2F7D004238381F9
:10BE300040F2E9331B4800E063B30289013B12F092
:10BE4000010F9BB2F8D08389164D40F2E93300E030
:10BE5000E3B12A89013B12F0020F9BB2F8D0A4B2E1
:10BE60001048AC8140F2E93300E07BB10289013B2C
:10BE700012F0010F9BB2F8D083890B6813B11A68D6
:10BE80009B88138338BD44F00804BCE70548FDF7E0
:10BE90003FFFF2E70348FDF73BFFD5E79826002078
:10BEA0000488002000380040144B984223D003F54A
:10BEB000806398421FD0038823F040031B041B0CAF
:10BEC0000380038823F038031B041B0C59B141F491
:10BED0008071002991FAA1F1B1FA81F108BF4FF008
:10BEE000FF310139C900194389B20180038843F049
:10BEF0004003038070474908DDE700BF0038004079
:10BF000008B5054B1B6803B19847044B044A1A60F7
:10BF100072B636F03DFD00BF88310020FCFF0120E5
:10BF2000EFBEADDE08B5034B1B6803B1984772B690
:10BF300036F02EFD88310020074A002302E001334D
:10BF4000102B07D05168814202F12002F7D1581C12
:10BF5000C0B2704700207047C02200200138F0B501
:10BF600040013C4CDFF820C125583B4FDCF83060E5
:10BF7000BD420CBF4FF400154FF4800527182E4327
:10BF80007D68CCF83060354EF960B54283B07B6196
:10BF900051D0334B9D424ED0A3F57A739D4236D09B
:10BFA00003F580639D4232D0A3F57A739D4246D05B
:10BFB00003F580639D4242D0A3F57A739D4240D041
:10BFC00003F580639D423CD0A3F57A739D4234D043
:10BFD00003F580639D4230D0A3F57A739D4232D041
:10BFE00003F580639D422ED0A3F57A739D422CD039
:10BFF00003F580639D4228D0A3F57A739D4226D035
:10C000001849194B8D420CBF1D46002500E0174D05
:10C0100004449209667CE5610021012301A88DF8A2
:10C0200004608DF805208DF806108DF8073031F08A
:10C0300021F903B0F0BD0E4DEAE70E4DE8E70E4DD5
:10C04000E6E70E4DE4E70E4DE2E70E4DE0E7064D64
:10C05000DEE700BFC0220020006002401060024006
:10C0600010640240B864024000800028008800107C
:10C070002080001020800020008020100080001808
:10C080000088002000802020003802400138F0B4F1
:10C0900044010948094D0359094F2E6B2044BB4206
:10C0A0000CBF4FF400134FF4800333432B6301762E
:10C0B0004276F0BC704700BFC0220020003802402A
:10C0C000006002402DE9F04F524C54F8204083B0FC
:10C0D000002C00F09B80256E002D00F09980174603
:10C0E0004D4A9846064604F166032869226004F228
:10C0F00066226361A2614FF400736A68A160C4E9BB
:10C100000333A265A24668B1FFF716FF721CD2B2D4
:10C110000C21FFF7BBFFA36DA9682A696263043392
:10C12000E1636365E868A0B1FFF706FF721C814612
:10C13000D2B20B21FFF7AAFF2346EA7F37494846D0
:10C14000FFF70CFFD5E90212A36D216404332365C8
:10C15000A26394F86500FDF75DFA814694F86400E7
:10C16000FDF758FA8346287F00284CD118F0080FB5
:10C1700036D1BA070DD5B9F1000F0AD00B22731CC6
:10C1800089F8062089F8073048466A7F2221FDF7A2
:10C1900009FBFB0715D4E36B7BB995F82020A97F39
:10C1A0008DF8063001A8930901228DF805308DF82D
:10C1B00004108DF8072031F05DF8504603B0BDE85B
:10C1C000F08FBBF1000FE6D0701C0C238BF807003A
:10C1D0008BF8063058466A7F2221FDF7E3FADAE74A
:10C1E000B9F1000F05D0701C0B2389F8070089F8FE
:10C1F000063018F0100F484614BF022112216A7F42
:10C20000FDF7D0FAC7E730F07FFCAFE7A246D4E7EE
:10C21000AA46D2E7F07B0020403604086589000872
:10C2200000B97047F0B595B0054631F049FAA34E14
:10C23000C368026832600446002B00F00381284680
:10C24000FDF7E8F99E4BC3F8600418B129220023DA
:10C250008271C371227A2A21FDF7A4FA30680CF0AA
:10C2600061FF30F051FC336896491A880968964896
:10C2700022F001021204120C81421A8000F2F480B2
:10C280000025DFF874C2914F1A88914805F1010E1C
:10C29000B1FBFEF14FF0030EB1FBF0F081B2B1FB48
:10C2A000FEF1ACF80010490039808A498B4292B205
:10C2B00012D001F580618B420ED0B3F1804F0BD0CC
:10C2C000A1F580318B4207D001F580618B4203D00C
:10C2D00001F580618B4202D122F0700292B27E4958
:10C2E0008B4200F0B18001F580618B4200F0AC80A0
:10C2F00022F4407201F56C4192B28B421A80D862EE
:10C300001D8540F0D68000221A8601219982E379AA
:10C310006020002200909807CDE902220492ADF837
:10C32000042040F19580DB0003F008030422ADF8FF
:10C330000E30ADF8042000236179306802936A461C
:10C340000CF0CAF8617933680C2910D8DFE801F0E5
:10C35000070F0F0FA80F0F0F9F0F0F0F96001A8BCD
:10C3600022F008021204120C42F008021A83B3F8F9
:10C3700044205A4D42F40042A3F844201A8842F067
:10C3800080021A80E27992074CBF042201228A407F
:10C39000198C92B221EA02011984198C0A431A8479
:10C3A0001A8842F001021A80207D00222921FFF71D
:10C3B0006DFE60224A49207D0023FFF7CFFDE06833
:10C3C000286016F0C5F92868036823F001030360AC
:10C3D00016F0BEF905A816F07FF933686279216975
:10C3E0002868059134331A4440F22A33069209939F
:10C3F0004FF480623B4B0B92079340224FF48053E3
:10C40000002705A908920C934FF480424FF4403363
:10C410000D920F930A970E9716F06FF963793168B2
:10C4200031488C890C2B9CBF304A32F813302A6873
:10C4300088BF3B4623438B811368012143F01003DF
:10C440001360017015B0F0BD1A80D8621D855CE7DD
:10C450005B0003F002034FF48072ADF80C30ADF8CE
:10C460000210ADF8102066E701F1B77505F55855D3
:10C470001F4AB5FBF2F5013DADB202E79A8B22F4FB
:10C4800000621204120C42F400629A836FE79A8BE6
:10C4900022F008021204120C42F008029A8366E7A6
:10C4A0001A8B22F400621204120C42F400621A8306
:10C4B0005DE7104A93423FF426AF26E75C860020F2
:10C4C00098260020409D0020FF6BDC024E86002055
:10C4D00000350C000000014000100040588600208C
:10C4E0001D8D00081C530020548600206C67040832
:10C4F000006CDC02000401404C8600200348D0F8A8
:10C50000EC3113B100F5F07018477047C0220020DD
:10C510000348D0F8CC3113B100F5E07018477047EC
:10C52000C02200200348D0F8AC3113B100F5D07020
:10C5300018477047C02200200348D0F88C3113B14F
:10C5400000F5C07018477047C02200200348D0F89B
:10C550006C3113B100F5B07018477047C02200204D
:10C560000348D0F84C3113B100F5A070184770475C
:10C57000C02200200348D0F82C3113B100F5907090
:10C5800018477047C02200200348D0F80C3113B17F
:10C5900000F5807018477047C02200200348D0F88B
:10C5A000EC300BB1E0301847704700BFC0220020CC
:10C5B0000348D0F8CC300BB1C0301847704700BFEB
:10C5C000C02200200348D0F8AC300BB1A03018478F
:10C5D000704700BFC02200200348D0F88C300BB158
:10C5E00080301847704700BFC02200200248C36E49
:10C5F0000BB1603018477047C02200200248C36C5E
:10C600000BB1403018477047C02200200248C36A6F
:10C610000BB1203018477047C02200200248C36881
:10C6200003B11847704700BFC0220020F8B5624D23
:10C6300004012F190646387A30F066FA3B7A03F087
:10C640001F015B090122032B02FA01F26DD0042BBA
:10C6500066D0022B5CD02B1901361879FCF7DAFF73
:10C66000F6B2074610B11223C67183712B1958799F
:10C67000FCF7D0FF10B11323C67183712B19987981
:10C68000FCF7C8FF10B11423C67183712E190A215B
:10C69000F2793846FDF786F87079FCF7BBFFF2793E
:10C6A0000A21FDF77FF8B079FCF7B4FFF2790A218F
:10C6B000FDF778F82B59414A934246D0404A9342BD
:10C6C0004ED0404A934256D03F4A93425ED03F4AB2
:10C6D00093422FD03E4A934263D02B191B7BE3B980
:10C6E000012002222B59198801F4415141F445716E
:10C6F0000A4302431A809A8B22F400621204120C3D
:10C7000007219A8319821A8842F040021A80F8BDE4
:10C71000304B596A0A435A629DE700200246E1E71E
:10C720002C4B19690A431A6195E72A4B196A0A4387
:10C730001A6290E702F568424FF48010536A43F49E
:10C740008013536216F09AF8C7E702F584324FF46B
:10C750008050536A43F48053536216F08FF8BCE75D
:10C7600002F500324FF48040136A43F480431362B1
:10C7700016F08CF8B1E702F5FE324FF40040136A70
:10C7800043F40043136216F081F8A6E702F5823203
:10C790004FF40050536A43F40053536216F06EF89E
:10C7A0009BE702F564424FF40010536A43F4001310
:10C7B000536216F063F890E77036002000300140B5
:10C7C00000380040003C004000340140005001406F
:10C7D0000054014000380240431C00F014812DE950
:10C7E000F04F4FEAC00808EB00039B00DFF8FC9213
:10C7F00059F803A087B009EB0304BAF1000F00F069
:10C80000FF80143309EB03010022DAF8047049F8C1
:10C810000320C1E90122CA60D4E9025B0346013367
:10C820000190DBB2002D00F008811522EB71AA7196
:10C830009AF81800BBF1000F00F0E68016228BF882
:10C8400006208BF8073030F05FF9BB8823F4407383
:10C850001B041B0CBB802846FDF7F9F85846FDF772
:10C86000F6F811212846FCF73BFE11215846FCF74B
:10C8700037FE0926332405E0013C4FF00A0006D0BC
:10C8800012F03EFB2846FDF709F90028F4D02846AF
:10C89000FDF7D8F8052012F033FB2846FDF7D7F84E
:10C8A000052012F02DFB013EE4D12846FDF7CAF821
:10C8B000052012F025FB5846FDF7C4F8052012F0BC
:10C8C0001FFB2846FDF7C3F8052012F019FB584658
:10C8D000FDF7BDF8019B08EB030409EB840428462F
:10C8E000E37C227C002B0CBF12213221FCF75AFF83
:10C8F000E37C627C002B0CBF122132215846FCF7EE
:10C9000051FF704B9F4200F0B1806F4B9F4200F08F
:10C91000C1806E4B9F4200F0B380BB886C4A6D4C67
:10C9200023F440731B041B0CBB80019B98443B8881
:10C9300009EB880943F0010399F812103B80BD8888
:10C9400002A8002918BF144616F056F8049A624847
:10C95000B2FBF4F325F03F05A0FB02122D04900C6E
:10C960002D0C0543BD8039885C4C4FF496729BB208
:10C9700002FB00F2002BA4FB020221F0010108BF20
:10C9800001239209090443F400430132090C398060
:10C990003A84BB833A88524B42F001023A803A888B
:10C9A000134043F480634FF480423B803A813B88DC
:10C9B00023F080031B041B0C3B809AF81A308DF87F
:10C9C0000830002402A801258DF809408DF80A409E
:10C9D0008DF80B5030F04EFC9DF80B209AF8193072
:10C9E0008DF808308DF809408DF80A40FAB95A09D7
:10C9F000203203F01F033B4905FA03F341F82230CC
:10CA000007B0BDE8F08F704730F07EF8BB8823F4A4
:10CA100040731B041B0CBB802846FDF718F85846D2
:10CA2000FDF715F811212846FCF75AFD21E702A869
:10CA300030F020FC07B0BDE8F08F9AF81800BBF189
:10CA4000000F31D016228BF807308BF8062030F01B
:10CA50005BF8BB8823F440731B041B0C2846BB8087
:10CA6000FCF7F5FF5846FCF7F2FFFEE61E4A136A94
:10CA700043F4001313624FF4001015F007FF4CE766
:10CA8000194A136A43F4000313624FF4000015F0CF
:10CA9000FDFE42E7144A136A43F4800313624FF425
:10CAA000800015F0F3FE38E730F02EF8BB8823F451
:10CAB00040731B041B0CBB805846FCF7C8FFFCF7F7
:10CAC000C6FFD6E60054004000580040005C00401D
:10CAD000009F2400804F120083DE1B43D34D621061
:10CAE000F5FBFFFF00E100E000380240187C002069
:10CAF0002DE9F0410678012E82B0054655D0022E70
:10CB000059D1806841F0800110B104688088608349
:10CB1000686840F2E93402E0002C00F09880068951
:10CB2000013C16F0020FA4B2F6D089B2818140F226
:10CB3000E93102E0002900F08A800489013914F00B
:10CB4000010F89B2F6D0818981894FF0000C4FF432
:10CB50007A714FF6FF764FF0FF0E03E0013989B28C
:10CB6000B1422CD00489A707F8D5A0F80CE04FF407
:10CB70007A7102E0B9B2B14221D00489E40701F12F
:10CB8000FF37F7D58489A4B20AB1147001320CF1D1
:10CB9000010C6345E6D1AB68002B56D01A689B8820
:10CBA0001383012002B0BDE8F08190F90400441C19
:10CBB00001D0032806DD002002B0BDE8F081FDF7BA
:10CBC000A7F8E8E74FEAC00EDFF8BCC00EEB00079D
:10CBD0000CEB87077C68002C48D06D793A626D00B9
:10CBE0004FF00008EDB2BD75F97587F81980BE7673
:10CBF0003B767E7587F81480A388FA61990512D474
:10CC00002388DA050BD44FF4805501E0013D2FD085
:10CC100023889B05FAD4238843F480732380A38858
:10CC200043F44073A38086440CEB8E024FF480548F
:10CC300001E0013C13D0537D002BFAD10CEB8E0E9A
:10CC40009EF8140080F00100B6E70120B4E7CDE9BA
:10CC50000023FDF75DF86868DDE9002374E7094A01
:10CC6000138801339BB21380FFF7B6FD2046A3E77C
:10CC7000044A138801339BB21380FFF7ADFD2846A9
:10CC80009AE700BFD8340020187C002007B50323A2
:10CC900001AA0021FFF72CFF9DF805309DF8040044
:10CCA0001B0243EA00439DF80600184303B05DF8F9
:10CCB00004FB08B5FFF7EAFF014B586008BD00BF51
:10CCC0009826002008B5FFF7E1FF014B186008BD6A
:10CCD0009826002007B506236A46F721FFF708FFCC
:10CCE0009DF801309DF800100B4A1B0143EA013307
:10CCF0009DF8021043EA1113D3609DF804309DF8AB
:10CD000003101B0143EA01339DF8051043EA111398
:10CD1000936003B05DF804FB9826002007B5032359
:10CD200001AAF621FFF7E4FE9DF805309DF80420E6
:10CD30001B0243EA02439DF806201343054AB2F959
:10CD40002020C2F10802D340034A536103B05DF8CA
:10CD500004FB00BFA43600209826002007B502235C
:10CD600001AAF621FFF7C4FE9DF804209DF80530C6
:10CD700043EA0223024A138203B05DF804FB00BFBA
:10CD80009826002070B582B00446062310306A460B
:10CD90004321FFF7ADFEC0B19DF804009DF800608F
:10CDA0009DF801109DF802509DF803209DF8053074
:10CDB00041EA062143EA002342EA0522A4F844108E
:10CDC000A4F84620A4F84830012002B070BD2DE937
:10CDD000F04F90F8583085B00746002B40F0F080B7
:10CDE000754B786993F86434002B00F01F82734B05
:10CDF000984200F09A8003F58063984200F0958095
:10CE0000038823F040031B041B0C0380038823F0DA
:10CE100038031B041B0C3822134303800388BA69B0
:10CE200043F04003038097F8561012B113689288BC
:10CE30005A8340F2E93304E0013B9BB2002B00F03F
:10CE4000328402899607F7D51A23838140F2E933A9
:10CE500004E0013B9BB2002B00F025840289D5073A
:10CE6000F7D5838940F2E93304E0013B9BB2002B04
:10CE700000F0158402899407F7D589B2818140F2C8
:10CE8000E93304E0013B9BB2002B00F008840289E7
:10CE9000D207F7D58389BB6913B11A689B881383BE
:10CEA000012012F02DF87B69444A93424AD002F5E2
:10CEB0008062934246D01A8822F040021204120C7B
:10CEC0001A801A8822F038021204120C08210A4330
:10CED0001A801A8842F040021A804321062302AACF
:10CEE00007F11000FFF704FE002838D09DF80A5023
:10CEF0009DF80B309DF808409DF809109DF80C0036
:10CF00009DF80D2043EA05231BB2A7F846305BB21B
:10CF100041EA042142EA00220133A7F84410A7F8AD
:10CF2000482021D005B0BDE8F08F038823F04003EE
:10CF30001B041B0C0380038823F038031B041B0C09
:10CF4000302269E71A8822F040021204120C1A807B
:10CF50001A8822F038021204120C0021B7E7B7F940
:10CF600046305BB20133DDD197F944300133D9D17A
:10CF70000A262FF0E9FF4FF4FA750CF06BFF044618
:10CF80000CF068FF001BB0F57A7FF9D3013DF4D1B6
:10CF900007202FF035FE4FF47A750CF05BFF044646
:10CFA0000CF058FF001BB0F57A7FF9D3013DF4D1A6
:10CFB000013EDED1FEF7A4FF982600200038004095
:10CFC0001D09013D032D03F00F0300F27183A24AF6
:10CFD00032F8150040FA03F2D60740F169830124C4
:10CFE00004FA03F3013B184035F0BAFA9B4B9C4A14
:10CFF0005B5D184412EBC00500F05A83202100232A
:10D00000A971EB7152F83030964903F13F4202F5B5
:10D010007E02920A895C01F01F024909032904FA81
:10D0200002F200F06183042900F04B83022900F032
:10D030006083AA88D4070BD5196821F00301196011
:10D0400019681960D96821F00301D960D968D960DD
:10D0500090070BD5196821F00C0119601968196047
:10D06000D96821F00C01D960D968D96051070BD576
:10D07000196821F03001196019681960D96821F028
:10D080003001D960D968D96016070BD5196821F02D
:10D09000C001196019681960D96821F0C001D96010
:10D0A000D968D960D4060BD5196821F4407119608C
:10D0B00019681960D96821F44071D960D968D960BC
:10D0C00090060BD5196821F4406119601968196040
:10D0D000D96821F44061D960D968D96051060BD56F
:10D0E000196821F44051196019681960D96821F450
:10D0F0004051D960D968D96016060BD5196821F45A
:10D100004041196019681960D96821F44041D9601B
:10D11000D968D960D4050BD5196821F4403119605C
:10D1200019681960D96821F44031D960D968D9608B
:10D1300090050BD5196821F4402119601968196010
:10D14000D96821F44021D960D968D96051050BD53F
:10D15000196821F44011196019681960D96821F41F
:10D160004011D960D968D96016050BD5196821F42A
:10D170004001196019681960D96821F44001D9602B
:10D18000D968D960D4040BD5196821F040711960B1
:10D1900019681960D96821F04071D960D968D960DF
:10D1A00090040BD5196821F0406119601968196065
:10D1B000D96821F04061D960D968D96051040BD594
:10D1C000196821F04051196019681960D96821F077
:10D1D0004051D960D968D96016040BD51A6822F07D
:10D1E00040421A601A681A60DA6822F04042DA6037
:10D1F000DA68DA6039461C4B41F80C3F284630F0BB
:10D200005BF8AB88B3FA83F3C3F11F03012212FA70
:10D2100003F33FF4E5AD154978690A6813430B60E1
:10D22000134B93F86434002B7FF4E1AD114B98421B
:10D2300000F0288203F58063984200F0238203887F
:10D2400023F040031B041B0C0380038823F03803E6
:10D250001B041B0C38220FE0006704080867040851
:10D26000248800203C65040855890008003C0140E2
:10D270009826002000380040134303800288BB69D1
:10D2800042F04002028013B11A689B88538340F237
:10D29000E93304E0013B9BB2002B00F021820289BC
:10D2A0009507F7D56B23838140F2E93304E0013B16
:10D2B0009BB2002B00F014820289D407F7D5838932
:10D2C00040F2E93304E0013B9BB2002B00F0058201
:10D2D00002899107F7D58023838140F2E93304E086
:10D2E000013B9BB2002B00F0F8810289D207F7D5F1
:10D2F0008389BB6913B11A689B88138396235D4C9D
:10D300005D4EDFF87C815D4DDFF8789101974FF03D
:10D31000100A1F460CF09EFD4FF47A7C4FF0010E70
:10D32000D8F80430C3F30803002B40F08081EFF3FA
:10D330001183002B40F07B812368A96800BF22681D
:10D340009342F9D132680CFB02FBABEB0101B1FB5C
:10D35000F2F10CFB03131B1AB3F57A7FE0D3013F04
:10D36000D8D1019FBB6913B11A689B885383786930
:10D3700040F2E93304E0013B9BB2002B00F0A981AD
:10D3800002899107F7D56823838140F2E93304E0ED
:10D39000013B9BB2002B00F09C810289D207F7D59C
:10D3A00083890321FCF760FDBB6913B11A689B8870
:10D3B00013839623DFF8C880304DDFF8C8900197BB
:10D3C0004FF0100A1F460CF045FD4FF47A7C4FF0E9
:10D3D000010ED8F80430C3F30803002B40F0098194
:10D3E000EFF31183002B40F004812368A96800BF8C
:10D3F00022689342F9D132680CFB02FBABEB0101CE
:10D40000B1FBF2F10CFB03131B1AB3F57A7FE0D3E7
:10D41000013FD8D1019FBB6913B11A689B88538320
:10D420006B217869FCF720FD03217869FCF71CFD6E
:10D43000BB6913B11A689B8813830F2011F060FD3C
:10D44000BB6913B11A689B8853836A217869FCF71A
:10D450000BFD786940F2E93304E0013B9BB2002BFD
:10D4600000F0348102899107F7D51023838140F2BF
:10D47000E9330EE0E4890020E889002010E000E0B4
:10D4800000ED00E0E0890020013B9BB2002B00F0A2
:10D490001D810289D207F7D58389BB6913B11A6848
:10D4A0009B8813830F2011F02BFDBB6913B11A6801
:10D4B0009B8853836C217869FCF7D6FC002178693E
:10D4C000FCF7D2FCBB6913B11A689B8813830F2049
:10D4D00011F016FDBB6997F8574013B11A689B8885
:10D4E000538319217869FCF7BFFC21467869FCF762
:10D4F000BBFCBB6913B11A689B8813830F2011F022
:10D50000FFFCBB6913B11A689B8853831B217869A0
:10D51000FCF7AAFC18217869FCF7A6FCBB6913B1DB
:10D520001A689B8813830F2011F0EAFCBB6913B1C2
:10D530001A689B8853831C217869FCF795FC182195
:10D540007869FCF791FCBB6913B11A689B88138357
:10D550000F2011F0D5FCBB6913B11A689B88538367
:10D5600037217869FCF780FC10217869FCF77CFC96
:10D57000BB6913B11A689B8813830F2011F0C0FC9C
:10D58000BB6913B11A689B88538338217869FCF70B
:10D590006BFC01217869FCF767FCBB6913B11A6861
:10D5A0009B8813830F2011F0ABFC7A69534B9A428E
:10D5B0005BD003F580639A4257D0138823F0400371
:10D5C0001B041B0C1380138823F038031B041B0C53
:10D5D00008210B431380138843F04003138001207C
:10D5E00011F08EFC464A7869012382F86434FFF713
:10D5F000FEBBEFF311818AF31288D5F808B02B68CF
:10D60000DB0344BFC9F800E0D5F808B02368D9F8B7
:10D610000020C9B281F31188316813440CFB01F278
:10D62000A2EB0B02B2FBF1F20CFB0323ECE6EFF3EF
:10D6300011818AF31288D5F808B02B68DB0344BF48
:10D64000C9F800E0D5F808B02368D9F80020C9B2BD
:10D6500081F31188316813440CFB01F2A2EB0B0239
:10D66000B2FBF1F20CFB032375E6138823F04003B1
:10D670001B041B0C1380138823F038031B041B0CA2
:10D680000021A6E7038823F040031B041B0C038042
:10D69000038823F038031B041B0C3022ECE5FCF755
:10D6A00037FBFFF7F8BBFCF733FB7869FFF7DABB12
:10D6B0003946144B41F80C3F00202FF0FDFDFFF7D9
:10D6C0008FBB1149086B02430A63B2E4FCF720FBED
:10D6D000E3E6FCF71DFB786963E6FCF719FB08E657
:10D6E000FCF716FB7869EBE50749086C02430A640E
:10D6F0009FE40549486C02434A649AE400380040BC
:10D7000098260020558900080038024070B582B084
:10D710000446062308306A463B21FFF7E9F9A8B121
:10D720009DF804009DF800609DF801109DF80250DE
:10D730009DF803209DF8053041EA062143EA0023C5
:10D7400042EA0522E18222836383012002B070BD98
:10D75000F0B5C60033189B00244DEA585468A28ADD
:10D7600083B092B20192019A2B4412F4706F1CBFE5
:10D7700001221A75019B13F4E06F07460CD1A38AAE
:10D780003E4423F4706305EB86051B041B0C00224A
:10D79000A3826A7503B0F0BD238BA38823F4806352
:10D7A0001B041B0CA380019B9B05E8D423889805D0
:10D7B000E5D42388D9050DD52388DA05FCD4238840
:10D7C00043F40073238023889B05FCD43846FFF77D
:10D7D00003F8D4E7238843F400732380A38823F459
:10D7E00040731B041B0CA380C9E700BF187C0020FA
:10D7F000F0B583B0441C8DF8073001D0032802DD5A
:10D80000002003B0F0BDC700274E3B1806EB830392
:10D810005C68002CF4D04900C9B29975012500213B
:10D82000DA755D7699761D765D751975A1880DF1AD
:10D8300007028905C3E9072212D42388DA050BD42D
:10D840004FF4805501E0013D25D023889B05FAD493
:10D85000238843F480732380A38843F44073A38018
:10D86000074406EB87024FF4805401E0013C09D0E5
:10D87000537D002BFAD106EB8707387D80F001003D
:10D8800003B0F0BD094A138801339BB21380FEF741
:10D89000A3FF2046B5E7054A138801339BB21380E6
:10D8A000FEF79AFF2846ACE7187C0020D834002009
:10D8B0000378012B47D0022B43D183682DE9F04137
:10D8C00001F07F0113B11C689B88638305461746EE
:10D8D000406840F2E93401E0002C3FD00689013C69
:10D8E00016F0020FA4B2F7D089B2818140F2E9317B
:10D8F00001E0002932D00389013913F0010F89B208
:10D90000F7D0838940F2E93100E021B3048901397D
:10D9100014F0020F89B2F8D0BFB2878140F2E93328
:10D9200000E0C3B10289013B12F0010F9BB2F8D0B5
:10D930008389AB686BB11A689B8813830120BDE8AB
:10D94000F0810020704713460A46417990F904009F
:10D950004EE70120F3E7FCF7DBF9EAE7FCF7D8F93B
:10D960006868CFE701224821A2E7012258219FE7FA
:10D970003122F4219CE7044B93F8202092013432A9
:10D9800002F0FC02F42193E7A43600202E22F421B9
:10D990008EE72DE9F04F85B0019090F858000028EF
:10D9A00040F08684019A137C012B00F0C984022B7D
:10D9B00000F06784C14CC24DC24FC34EDFF80C83E8
:10D9C0004FF0640A4FF010090CF044FA4FF47A71EA
:10D9D0004FF0010C7B68C3F30803002B40F0448236
:10D9E000EFF31183002B40F03F8286462368B06836
:10D9F00000BF22689342F9D10246704696462A68D3
:10DA000001FB02FBABEB0E0EBEFBF2FE01FB03E3E0
:10DA10001B1AB3F57A7FDDD3BAF1010AD4D1019A8A
:10DA2000137C012B00F09684022B00F01384DFF8A6
:10DA30009482A54FDFF894924FF0640B4FF0100AD8
:10DA40000CF008FA4FF47A71D8F80430C3F30803E5
:10DA5000002B40F02982EFF31183002B40F0248249
:10DA60002368BE6800BF22689342F9D1D5F800C090
:10DA700001FB0CF2961BB6FBFCF601FB03631B1AC1
:10DA8000B3F57A7FE0D3BBF1010BD9D1019A137CB6
:10DA9000012B00F09584022B00F0C683894F8A4E3B
:10DAA000DFF828824FF0640A4FF010090CF0D2F929
:10DAB0004FF47A714FF0010C7B68C3F30803002B1D
:10DAC00040F03182EFF31183002B40F02C82864628
:10DAD0002368B06800BF22689342F9D102467046BD
:10DAE00096462A6801FB02FBABEB0E0EBEFBF2FE74
:10DAF00001FB03E31B1AB3F57A7FDDD3BAF1010A08
:10DB0000D4D1019A137C012B00F05184022B00F038
:10DB100075836C4F6C4EDFF8B4814FF00F0A4FF0F5
:10DB200010090CF097F94FF47A714FF0010C7B68F3
:10DB3000C3F30803002B40F0D681EFF31183002BD1
:10DB400040F0D18186462368B06800BF22689342C6
:10DB5000F9D10246704696462A6801FB02FBABEB00
:10DB60000E0EBEFBF2FE01FB03E31B1AB3F57A7F38
:10DB7000DDD3BAF1010AD4D1019991F853300A7C6E
:10DB8000042B34BF18261A26012A00F02C84022AFE
:10DB900000F01E834B4F4C4EDFF830814FF00F0AE0
:10DBA0004FF010090CF056F94FF47A714FF0010C58
:10DBB0007B68C3F30803002B40F0D581EFF311839A
:10DBC000002B40F0D08186462368B06800BF2268F1
:10DBD0009342F9D10246704696462A6801FB02FB41
:10DBE000ABEB0E0EBEFBF2FE01FB03E31B1AB3F51B
:10DBF0007A7FDDD3BAF1010AD4D1019A137C012BCB
:10DC000000F0E883022B00F0CD822E4F2E4EDFF87D
:10DC1000BC804FF00F0A4FF010090CF01BF94FF4C5
:10DC20007A714FF0010C7B68C3F30803002B40F0BE
:10DC3000BA81EFF31183002B40F0B581864623684B
:10DC4000B06800BF22689342F9D1024670469646FA
:10DC50002A6801FB02FBABEB0E0EBEFBF2FE01FBE2
:10DC600003E31B1AB3F57A7FDDD3BAF1010AD4D1ED
:10DC7000019B1A7C93F85660012A194600F07D83B7
:10DC8000022A00F079820F4F0F4EDFF840804FF0EC
:10DC90000F0A4FF010090CF0DDF84FF47A714FF0D5
:10DCA000010C7B68C3F30803002B40F00382EFF301
:10DCB0001183002B40F0FE81864609E0E4890020B4
:10DCC000E889002000ED00E010E000E0E08900209D
:10DCD0002368B06800BF22689342F9D102467046BB
:10DCE00096462A6801FB02FBABEB0E0EBEFBF2FE72
:10DCF00001FB03E31B1AB3F57A7FD2D3BAF1010A11
:10DD0000C9D1019B1A7C93F85760012A194600F08B
:10DD10002B83022A00F01A82C34FC44EDFF810830F
:10DD20004FF0640A4FF010090CF094F84FF47A7138
:10DD30004FF0010C7B68C3F30803002B40F09A817D
:10DD4000EFF31183002B40F0958186462368B0687D
:10DD500000BF22689342F9D10246704696462A686F
:10DD600001FB02FBABEB0E0EBEFBF2FE01FB03E37D
:10DD70001B1AB3F57A7FDDD3BAF1010AD4D1019A27
:10DD8000137C012B00F00A83022B00F0C981A64FFF
:10DD9000A64EDFF89C824FF00F0A4FF010090CF0EE
:10DDA00059F84FF47A714FF0010C7B68C3F3080304
:10DDB000002B40F03F81EFF31183002B40F03A81BC
:10DDC00086462368B06800BF22689342F9D10246B4
:10DDD000704696462A6801FB02FBABEB0E0EBEFBBB
:10DDE000F2FE01FB03E31B1AB3F57A7FDDD3BAF130
:10DDF000010AD4D1019A137C012B00F0C782022BB7
:10DE000000F07881884F894EDFF824824FF00F0AA6
:10DE10004FF010090CF01EF84FF47A727B68C3F3D0
:10DE20000803002B40F0DF80EFF31183002B40F05C
:10DE3000DA802368B16800BFD4F800C06345F8D128
:10DE4000D5F800C002FB0CFBABEB010EBEFBFCFEE9
:10DE500002FB03E31B1AB3F57A7FDFD3BAF1010AA1
:10DE6000D8D105B0BDE8F08FEFF3118E89F3128899
:10DE7000D6F808B03368DA0344BFC8F800C0D6F853
:10DE800008B02368D8F800205FFA8EFE8EF3118860
:10DE9000D5F800E0134401FB0EF2A2EB0B02B2FB3B
:10DEA000FEF201FB0323B3E5EFF311868AF3128838
:10DEB000D7F808C03B68DB0304D50123C9F800305C
:10DEC000D7F808C02368D9F80020F6B286F3118885
:10DED0002E68134401FB06F2A2EB0C02B2FBF6F231
:10DEE00001FB0323CBE5EFF3118E89F31288D6F8FB
:10DEF00008B03368DB0344BFC8F800C0D6F808B0E8
:10DF00002368D8F800205FFA8EFE8EF31188D5F8CA
:10DF100000E0134401FB0EF2A2EB0B02B2FBFEF297
:10DF200001FB032321E6EFF3118E89F31288D6F863
:10DF300008B03368DA0344BFC8F800C0D6F808B0A8
:10DF40002368D8F800205FFA8EFE8EF31188D5F88A
:10DF500000E0134401FB0EF2A2EB0B02B2FBFEF257
:10DF600001FB0323C6E5EFF3118E89F31288D6F87F
:10DF700008B03368DA0344BFC8F800C0D6F808B068
:10DF80002368D8F800205FFA8EFE8EF31188D5F84A
:10DF900000E0134401FB0EF2A2EB0B02B2FBFEF217
:10DFA00001FB032322E6EFF3118E89F31288D6F8E2
:10DFB00008B03368DB0344BFC8F800C0D6F808B027
:10DFC0002368D8F800205FFA8EFE8EF31188D5F80A
:10DFD00000E0134401FB0EF2A2EB0B02B2FBFEF2D7
:10DFE00001FB03233DE6EFF3118E89F31288D6F887
:10DFF00008B03368DB0304D50123C8F80030D6F835
:10E0000008B02368D8F800C05FFA8EFE8EF311883E
:10E010002968634402FB01FCACEB0B0CBCFBF1FC7C
:10E0200002FB03C316E700BF00ED00E010E000E0D4
:10E03000E0890020EFF3118E89F31288D6F808B03A
:10E040003368DA0344BFC8F800C0D6F808B02368C4
:10E05000D8F800205FFA8EFE8EF31188D5F800E024
:10E06000134401FB0EF2A2EB0B02B2FBFEF201FB2A
:10E070000323B8E6EFF3118E89F31288D6F808B0BF
:10E080003368DB0344BFC8F800C0D6F808B0236883
:10E09000D8F800205FFA8EFE8EF31188D5F800E0E4
:10E0A000134401FB0EF2A2EB0B02B2FBFEF201FBEA
:10E0B00003235DE6EFF3118E89F31288D6F808B0DA
:10E0C0003368DA0344BFC8F800C0D6F808B0236844
:10E0D000D8F800205FFA8EFE8EF31188D5F800E0A4
:10E0E000134401FB0EF2A2EB0B02B2FBFEF201FBAA
:10E0F0000323FFE5936913B11A689B885383019E3C
:10E1000038217069FBF7B0FE01217069FBF7ACFEA6
:10E11000B369002B3FF476AE1A689B88138371E6CF
:10E12000936913B11A689B885383019E37217069E4
:10E13000FBF79AFE10217069FBF796FEB369002B7E
:10E140003FF425AE1A689B88138320E69B6913B1C0
:10E150001A689B885383019F19217869FBF784FE15
:10E1600031467869FBF780FEBB69002B3FF4D4ADE4
:10E170001A689B881383CFE59B6913B11A689B8843
:10E180005383019F1A217869FBF76EFE3146786947
:10E19000FBF76AFEBB69002B3FF475AD1A689B88DC
:10E1A000138370E5936913B11A689B885383019EAA
:10E1B0001C217069FBF758FE18217069FBF754FEAB
:10E1C000B369002B3FF421AD1A689B8813831CE5CB
:10E1D0008B6913B11A689B885383019F1B2178694F
:10E1E000FBF742FE31467869FBF73EFEBB69002B28
:10E1F0003FF4D0AC1A689B881383CBE4936913B1C6
:10E200001A689B885383019E6B217069FBF72CFE73
:10E2100001217069FBF728FEB369002B3FF479AC4C
:10E220001A689B88138374E4936913B11A689B88F6
:10E230005383019E6B217069FBF716FE0021706904
:10E24000FBF712FEB369002B3FF428AC1A689B88D9
:10E25000138323E4936913B11A689B885383019E47
:10E2600068217069FBF700FE07217069FBF7FCFD70
:10E27000B369002B3FF4DBAB1A689B881383FFF76D
:10E28000D6BB936913B11A689B885383019C6B2199
:10E290006069FBF7E9FD80216069FBF7E5FDA36993
:10E2A000002B3FF487AB1A689B881383FFF782BB70
:10E2B000FBF7B0F9019B044603F10C05002800F0C0
:10E2C000A1800068564900F13F4303F57E039A0A96
:10E2D00001238A5C02F01F01520920268B40032A89
:10E2E0004FF00001A671E17100F09480042A00F063
:10E2F0008480022A03D14B4A516C0B435364A38898
:10E30000029302A90023039314F0A0F9019A464B4B
:10E31000D360294620462EF0CFFFA388B3FA83F3BB
:10E32000C3F11F03012212FA03F33FF43BAB3F4951
:10E330000A681343019A0B60137C012B7FF437ABFF
:10E3400010468023417D90F914006B22FFF750FAAC
:10E35000FFF730BB10460723417D90F91400682277
:10E36000FFF746FAFFF763BB184619223346497D8B
:10E3700090F91400FFF73CFACEE418461A2233460F
:10E38000497D90F91400FFF733FA7CE410463822F7
:10E39000417D90F91400FFF72BFA33E51046102366
:10E3A000417D90F914003722FFF722FAEFE410467E
:10E3B0006B22417D90F91400FFF71AFAFFF7A9BB11
:10E3C00010465B46417D90F914006B22FFF710FA6E
:10E3D000FFF764BB10461823417D90F914001C22FE
:10E3E000FFF706FA11E4084633461B22497D90F9EF
:10E3F0001400FFF7FDF9FFF7CDBB0A4A116B0B4381
:10E4000013637CE71A46084BD36029462EF054FF6D
:10E41000FFF7C8BA034A116C0B4313646FE700BFE0
:10E420003C6504080038024055890008003C014062
:10E430002DE9F04F814A436983B09342019010D097
:10E4400002F5806293420CD01A8822F04002120436
:10E45000120C1A801A8822F038021204120C302191
:10E460000BE01A8822F040021204120C1A801A885B
:10E4700022F038021204120C28210A431A801A884A
:10E4800042F040021A800BF0E5FC04460BF0E2FC7F
:10E490008442FBD0019C2046FFF77BFAA36913B1AD
:10E4A0001A689B885383019B586940F2E93302E064
:10E4B000002B00F0BE800289013B12F0020F9BB2DC
:10E4C000F6D06A23838140F2E93302E0002B00F0AA
:10E4D000B0800289013B12F0010F9BB2F6D0838914
:10E4E00040F2E93302E0002B00F0A0800289013BFA
:10E4F00012F0020F9BB2F6D01023838140F2E93371
:10E5000002E0002B00F092800289013B12F0010F23
:10E510009BB2F6D08389019B9B6913B11A689B88D3
:10E520001383474C474F484E484DDFF824814FF046
:10E53000640A4FF010090BF08DFC4FF47A714FF024
:10E54000010C7368C3F30803002B4FD1EFF3118361
:10E55000002B4BD186462368A86800BF22689342EF
:10E56000F9D10246704696463A6801FB02FBABEBD6
:10E570000E0EBEFBF2FE01FB03E31B1AB3F57A7F1E
:10E58000DFD3BAF1010AD6D1019B2C4A5B699342D1
:10E5900010D002F5806293420CD01A8822F040021B
:10E5A0001204120C1A801A8822F038021204120C7B
:10E5B00008210BE01A8822F040021204120C1A8083
:10E5C0001A8822F038021204120C00210A431A8021
:10E5D0001A8842F040021A800BF03CFC04460BF013
:10E5E00039FC8442FBD003B0BDE8F08FEFF3118E0D
:10E5F00089F31288D5F808B02B68DB0344BFC8F84C
:10E6000000C0D5F808B02368D8F800205FFA8EFE65
:10E610008EF31188D7F800E0134401FB0EF2A2EB51
:10E620000B02B2FBFEF201FB0323A6E7FBF770FB34
:10E6300071E7FBF76DFB019B586951E7003800401B
:10E64000E4890020E889002000ED00E010E000E00F
:10E65000E08900200220FAF791BB0220FFF778B88A
:10E660000120FAF78BBB0120FFF772B80020FAF700
:10E6700085BB0020FFF76CB8044B187828B1044A1A
:10E680001268520744BF00201870704710720020B3
:10E690000020014043680B4A23F0407323F4807349
:10E6A00043F48073436083681A4042F00202826040
:10E6B000C36A0139C9B223F4700343EA0153C36248
:10E6C000704700BFFDF7FFC01549164B16484A6852
:10E6D00010B4CC681549B2FBF4F203FB02F30360FB
:10E6E000D1F88820124B134C42F47002C1F88820F4
:10E6F0001A68002042F001021A6098601A6822F03D
:10E70000847222F480321A605C601A684FF00064F0
:10E7100022F480221A60D8608C605DF8044B704748
:10E720000000002040420F00409D002000ED00E06E
:10E730000038024010300024104A114B12689A42EF
:10E7400000D0C1E70F4B1B68022B12D80E480F4AAE
:10E7500003EB43035B00191810B41C5A8B884888DC
:10E760005460C2E90230054B5DF8044B00221A6088
:10E77000AAE7024B00221A60A6E700BFF8FF0120BB
:10E78000CEFABEBAF4FF0120505D0408000000205C
:10E79000124B1A89D3E9000110B40132B3F90A40CF
:10E7A00092B201300131A242C3E900011A810CDAB0
:10E7B000DA89B3F910105DF8044B013292B28A4243
:10E7C000DA81A4BF0022DA8170479A895DF8044B90
:10E7D000002101329A811981D9817047082B0020CC
:10E7E00000230122C270837003800371437183711F
:10E7F000C37103724372704700230A2203604360AF
:10E80000C381C0F80630C0F80A300280704700BFEC
:10E810002DE9F843744CE27E237F9A4277D0E27E62
:10E82000E37EC2EBC20204EB8202C3EBC30304EB40
:10E83000830392F83F1093F824608B1E9E4225D0EC
:10E840006A4B216A1B78172B64D00025E37E684A47
:10E850000133A2FB0302520802EB42029B1ADBB215
:10E86000E376002938D00BF0F5FAD4F8A830C01AB6
:10E87000B0F5FA7F04DB002345F0040584F8A530E9
:10E88000D4F8A03083BB2846BDE8F883E37E04F1CA
:10E890002407C3EBC30307EB830361B119440022D0
:10E8A00013F8015B2A44994292B2F9D1D3B203EB37
:10E8B0001222FF2A3AD04D4B216A1B78172BC4D164
:10E8C000B4F878304B4A01339BB20420A4F8783076
:10E8D000538090800025B9E794F8A530002BC2D171
:10E8E000D4F8A030002BCED0434A1268D31AB3F527
:10E8F000FA7FC8D994F87A30032B02D13F4B00221B
:10E900001A800023C4F8A0302846BDE8F883216AA5
:10E910000025A6E7B4F87830364A01339BB20320CD
:10E92000A4F878305380908000258FE7E37E0122A1
:10E930001C2101FB0323FA18FD5CE5B1012D13D165
:10E94000082E38D0294B216A1B78172B7FF47DAF16
:10E95000B4F87830274A01339BB20620A4F8783007
:10E9600053809080002571E7204B1B78172B15D022
:10E97000216A00256AE7192E216A43D01B4B1B78B8
:10E98000172B7FF463AFB4F878301A4A01339BB287
:10E990000620A4F878305380908057E7B4F8783098
:10E9A000144A216A01339BB20520A4F878305380C1
:10E9B000908000254AE794F8A430002BD8D05378F3
:10E9C000102B00F0FD8040F2F880303B012BCFD8B7
:10E9D00052F8010F0A4960619379908888808B71A1
:10E9E0002162002532E700BF082B00200D8800209F
:10E9F000ABAAAAAA10880020E4890020AC4E00200F
:10EA00001C2B002092F802C05578036992F803800D
:10EA100092F804909679D77992F808E00CF0070CF8
:10EA200045EA0C2508F03F0892F80AC01D80957849
:10EA30004FEA481848EAD508957BA3F8028092F877
:10EA400003804FEA890040EA981092F8058008F0A8
:10EA5000010840EA8820988006F00F06507992F865
:10EA60000780F60146EA5000567AD8804FEA4E0EEB
:10EA70004EEAD81E06F0030692F80680D07A07F018
:10EA80007F074EEA462E3F01567BA3F80AE047EA8D
:10EA900018171F8106F00707967A92F809E0C00060
:10EAA00040EA5610167B0CF01F0C46EA072605F0CC
:10EAB0003F05577BD8816D014FEA8C1C45EAD70092
:10EAC0004CEA9E0CA3F80CC01E825882D07B92F8B0
:10EAD0000EE0D77C92F8128092F811C0967C557D9A
:10EAE000800040EA9E1092F810E07F000EF0010EC8
:10EAF00047EAD8170CF00F0C92F8108040EA8E20ED
:10EB00004FEACC1C92F814E098824CEA580C907DA5
:10EB1000A3F816C006F07F0692F811C00EF0030E9F
:10EB200047EA4E27360146EA1C165F8392F814C066
:10EB3000577D1E8305F01F05AD01C00040EA571048
:10EB400045EA9C05D8839D83D57D94F87A6015F0BD
:10EB5000010F40F2147014BF0746AD2715F0020FE5
:10EB600008BFAD2015F0080F0CBF01250325032EAB
:10EB70001F8458841CD1137E94F87B00124FE26FDF
:10EB8000642B04EB4006A8BF64239B02A7FB03731E
:10EB9000B6F8807001305B0900F00F00D21B1A44F8
:10EBA00084F87B000948A6F880301309E2670380E7
:10EBB000074B1B68C4F8A03048E6002B7FF4D8AEA2
:10EBC000012384F8A530D3E61F85EB51AC4E00201D
:10EBD000E489002038B504460BF03CF94F4B002285
:10EBE00083F8AC2093F8AD20012A17D9D3F8B020D0
:10EBF00040F6AC51821A8A4210DD494A1278172A2F
:10EC000009D1B3F878204749013292B20125A3F81F
:10EC100078204A808D80002283F8AD20E2B27E2ADF
:10EC200028D093F8AD1021B393F8AD101B2957D815
:10EC300093F8BC1000296BD0002182F0200283F8E9
:10EC4000BC1093F8AD10022903D1012A08BF83F844
:10EC5000B420197F93F8AD4093F8AD00C1EBC1012A
:10EC600003EB810121440130C0B281F8232083F8F5
:10EC7000AD0038BD93F8AD20012A2BD91A7F2A495F
:10EC8000DC7E0132A1FB0251490801EB4101521A1D
:10EC9000D2B294420AD093F8AD40197F1A77C1EBF3
:10ECA000C10103EB8101621E81F83F2093F8B4207B
:10ECB0003AB10121002283F8AC1083F8B420C3F8E4
:10ECC000A800174A1278172A1CD00022C3F8B800EF
:10ECD00083F8BC20012283F8AD20C3F8B00038BD12
:10ECE0000F4A12780021172A83F8AD10C1D1B3F86A
:10ECF00078200C49013292B20220A3F878204A8091
:10ED0000888038BDD3F8B8200649821A0A80DCE72B
:10ED10007D2A96D1012283F8BC2038BD082B002023
:10ED20000D88002010880020ABAAAAAA03788B4285
:10ED300083BF034B03EB4101B1F8C00000207047D3
:10ED4000082B0020044B93F8D80018B1002283F858
:10ED5000D8200120704700BF082B0020F0B4C24D1E
:10ED600095F8FF6005F1DC020244B41E1444A2428F
:10ED700000F07881013A013C002341F2210112F8B0
:10ED8000017F83EA07231FB2BBB2002FACBF5B0039
:10ED900081EA43039BB21F0454BF5B0081EA430333
:10EDA0009BB21F0454BF5B0081EA43039BB21F0464
:10EDB00054BF5B0081EA43039BB21F0454BF5B0056
:10EDC00081EA43039BB21F0454BF5B0081EA430303
:10EDD0009BB21F0454BF5B0081EA43039BB21F0434
:10EDE00054BF5B0081EA4303A2429BB2C7D10644F1
:10EDF000B21E013E2A442E4492F8DC1096F8DC2024
:10EE000002EB012292B29A4201D0F0BC704795F811
:10EE10000021002A00F02181431CDBB25C1C2C4441
:10EE20002B444FF4AF6193F8DC6094F8DC3003EBD3
:10EE300006239BB201FB03F31B1303F54873012A5E
:10EE4000A5F8C03000F00981C31CDBB25C1C2C4467
:10EE50002B44022A93F8DC6094F8DC3003EB0623A1
:10EE60009BB201FB03F34FEA233303F54873A5F884
:10EE7000C23000F0F280431DDBB25C1C2C442B44FA
:10EE8000032A93F8DC6094F8DC3003EB06239BB292
:10EE900001FB03F34FEA233303F54873A5F8C430AD
:10EEA00000F0DB80C31DDBB25C1C2C442B44042A25
:10EEB00093F8DC6094F8DC3003EB06239BB201FB93
:10EEC00003F34FEA233303F54873A5F8C63000F087
:10EED000C48000F10903DBB25C1C2C442B44052ADE
:10EEE00093F8DC6094F8DC3003EB06239BB201FB63
:10EEF00003F34FEA233303F54873A5F8C83000F055
:10EF0000AC8000F10B03DBB25C1C2C442B44062AC2
:10EF100093F8DC6094F8DC3003EB06239BB201FB32
:10EF200003F34FEA233303F54873A5F8CA3000F022
:10EF3000948000F10D03DBB25C1C2C442B44072AA7
:10EF400093F8DC6094F8DC3003EB06239BB201FB02
:10EF500003F34FEA233303F54873A5F8CC307CD094
:10EF600000F10F03DBB25C1C2C442B44082A93F8FD
:10EF7000DC6094F8DC3003EB06239BB201FB03F367
:10EF80004FEA233303F54873A5F8CE3065D000F17E
:10EF90001103DBB25C1C2C442B44092A93F8DC607F
:10EFA00094F8DC3003EB06239BB201FB03F34FEA3A
:10EFB000233303F54873A5F8D0304ED000F1130386
:10EFC000DBB25C1C2C442B440A2A93F8DC6094F8D6
:10EFD000DC3003EB06239BB201FB03F34FEA233340
:10EFE00003F54873A5F8D23037D000F11503DBB232
:10EFF0005C1C2C442B440B2A93F8DC6094F8DC3026
:10F0000003EB06239BB201FB03F34FEA233303F523
:10F010004873A5F8D43020D000F11703DBB25C1C94
:10F020002C442B440C2A93F8DC6094F8DC3003EB7E
:10F0300006239BB201FB03F34FEA233303F5487326
:10F04000A5F8D63009D000F11903DBB25A1C2A44C6
:10F050002B4493F8DC3092F8DC30012385F8D8306B
:10F06000F0BC70470023C2E6082B002070B55C4C52
:10F0700006460AF0EFFED4F80431C4F80401C01AC1
:10F08000B0F5FA5F1AD9002384F8083184F8093101
:10F09000A12E2FD0A22E00F09C8094F8092194F884
:10F0A000FF300025A2B16A1C6119D5B2F6B29D42AB
:10F0B00081F8DC6084F808510CD070BD94F80851D8
:10F0C000002DE5D094F8092194F8FF30002AEAD108
:10F0D0009D42F2D194F80A31052B72D0062B03D150
:10F0E00094F8DD301E2B0DD0002384F8093184F80C
:10F0F000083170BD01221B2384F8092184F8FF30F8
:10F100000025D0E76A1E002A4FF0000150DD0846B6
:10F110000B462344013093F8DC30DBB283EA01056F
:10F12000ED074FEA530348BF83F08C0383EA510590
:10F13000EE074FEA530348BF83F08C0383EA91053F
:10F14000ED074FEA530344BF83F08C03DBB283EA3D
:10F15000D105EE074FEA530344BF83F08C03DBB2C3
:10F1600083EA1115ED074FEA530344BF83F08C0384
:10F17000DBB283EA5115EE074FEA530344BF83F035
:10F180008C03DBB283EA9115ED074FEA530344BFCA
:10F1900083F08C03DBB283EAD1155908EB0748BF33
:10F1A00081F08C01C0B248BFC9B282420346B0DCD4
:10F1B000224492F8DC308B4296D10320FFF7CEFD3B
:10F1C00092E70020FFF7CAFD94F8DD301E2B8BD1AB
:10F1D00098E70122232384F8092184F8FF308FE780
:10F1E000082B002007299DBF034B03EB8101B1F8D9
:10F1F0000C010020704700BF082B00201A4B93F829
:10F200002C2132B193F830210021A82A83F82C1147
:10F2100001D00020704793F84321002AF9D110B49F
:10F22000DFED126A03F5987103F5847003F5A0729F
:10F23000B4EE047ACC780B7903EB042307EE903A12
:10F24000F8EEE77AB0EE666AA7EE876A02318A4284
:10F25000FCEEC67A17EE903A40F8043FEAD101205E
:10F260005DF8044B704700BF082B00200080BBC333
:10F2700010B504460AF0EEFD0F4BD3F84821C3F851
:10F280004801801A41F288329042E4B205D983F8ED
:10F290003041012283F84C2110BD93F84C2199187C
:10F2A000142A81F8304103D1012283F82C2110BDAA
:10F2B0000132D2B2EEE700BF082B0020034B03EB74
:10F2C0004101B1F85001C008704700BF082B002071
:10F2D000724B93F87021002A00F0C28070B493F84A
:10F2E0007141B3F8725103EB4401002091F877614A
:10F2F00091F8782183F8700142EA0622954202D003
:10F30000002070BC704793F87521012A00F0AA8094
:10F31000812AF6D10320102C40F2A68093F879417F
:10F3200093F8775193F8781193F87A2141EA0521FF
:10F3300042EA04221024A3F85011A3F8522183F8C2
:10F34000714193F87B1193F87C21032C42EA01224E
:10F35000A3F85421D5D093F87D1193F87E21042C85
:10F3600042EA0122A3F85621CBD093F87F1193F8FB
:10F370008021052C42EA0122A3F85821C1D093F83C
:10F38000811193F88221062C42EA0122A3F85A2126
:10F39000B7D093F8831193F88421072C42EA012215
:10F3A000A3F85C21ADD093F8851193F88621082C41
:10F3B00042EA0122A3F85E21A3D093F8871193F8C3
:10F3C0008821092C42EA0122A3F8602199D093F800
:10F3D000891193F88A210A2C42EA0122A3F86221BA
:10F3E0008FD093F88B1193F88C210B2C42EA0122D9
:10F3F000A3F8642185D093F88D1193F88E210C2CFD
:10F4000042EA0122A3F866213FF47BAF93F88F1103
:10F4100093F890210D2C42EA0122A3F868213FF4D1
:10F4200070AF93F8911193F892210E2C42EA0122C9
:10F43000A3F86A213FF465AF93F8931193F89421F0
:10F44000102C42EA0122A3F86C217FF45AAF93F802
:10F45000951193F8962142EA0122A3F86E2150E714
:10F4600000207047104656E7002C3FF44AAF93F84F
:10F47000771193F87821012C42EA0122A3F8502158
:10F480003FF43FAF93F8791193F87A21022C42EAC6
:10F490000122A3F852217FF454AF32E7082B002059
:10F4A00038B504460AF0D6FC444AD2F89C31C31A57
:10F4B000B3F57A6F16D892F8A031C2F89C01B3B1B7
:10F4C000022B1FD0242B92F8711175D90133023110
:10F4D000DBB249008B4282F8A0311BDB01318B4249
:10F4E00063D038BD0023C2F89C0182F8A031A82C5B
:10F4F000F7D1002382F87031A2F8723192F87111BD
:10F50000204603E0E0B282F871010146D51885F883
:10F510007401DBE7B2F87231E4B283EA042424B266
:10F52000002CB8BF41F22101A3B2B4BF81EA43036A
:10F530005B009BB21C0446BF41F2210181EA4303F8
:10F540005B009BB2180446BF41F2210181EA4303EC
:10F550005B009BB2190446BF41F2210181EA4303DB
:10F560005B009BB21D0446BF41F2210181EA4303C7
:10F570005B009BB21C0446BF41F2210181EA4303B8
:10F580005B009BB2180446BF41F2210181EA4303AC
:10F590005B009BB2190446BF41F2210181EA43039B
:10F5A0005B009BB2A2F8723138BD0021012382F8C2
:10F5B000A01182F8703138BDE0B2A7E7082B002017
:10F5C000F8B5124D95F8B92102B9F8BD104B1C6879
:10F5D0002368DE693EB1204605F5D271B0470023AD
:10F5E00085F8B931F8BD05F5D277BE1800E023687B
:10F5F0009B68204698470028F9D0236817F8011B1C
:10F600001B6820469847B742F1D1E8E7082B002055
:10F61000B052002003788B4210D9094B03EB8101D3
:10F6200093F8EC31D1F8BC011BB900F5777080B2CA
:10F630007047400800F5777080B27047002070472F
:10F64000082B00202DE9F041C54C94F8F40108B9CD
:10F65000BDE8F08194F8F511002384F8F431002915
:10F6600000F03B8194F8F831BE4D94F808225BB26B
:10F6700013F1630FB8BF95F90030002A40D013F1A1
:10F68000310F80F2AD8113F1380F80F2CC8113F18C
:10F690003D0F80F2CC8113F1420F80F2CC8113F147
:10F6A000450F80F2CC8113F1470F80F2CC8113F12A
:10F6B000490F80F2CC8113F14A0F00F0CC8113F195
:10F6C0004B0F00F0CB8113F14C0F00F0CB8113F105
:10F6D0004D0F00F0CA8113F15C0FB8BF642680F2B1
:10F6E000C781D4F80C02A04F00FB06F087FB007620
:10F6F000C017C0EB661004EB820680B2C6F8BC01EE
:10F700002B7094F8047294F8053294F8060294F879
:10F7100007621B0443EA0763334343EA002303F011
:10F72000F020B0F1E02F00F0CF80102794F81602FF
:10F7300094F8FA31D4F8186294F81CC23678034170
:10F7400003F00F039E4210D90B2B0ED8002A40F075
:10F75000FF8094F8FA8194F8FBE104EB83030CEA50
:10F7600008080EEB082EC3F8BCE194F8FC31034105
:10F7700003F00F039E4210D90B2B0ED8002A40F045
:10F78000EB8094F8FC8194F8FDE104EB83030CEA30
:10F7900008080EEB082EC3F8BCE194F8FE310341D3
:10F7A00003F00F039E4210D90B2B0ED8002A40F015
:10F7B000F68094F8FE8194F8FFE104EB830308EAF5
:10F7C0000C080EEB082EC3F8BCE194F8003203419C
:10F7D00003F00F039E4210D90B2B0ED8002A40F0E5
:10F7E000E28094F8008294F801E204EB83030CEACF
:10F7F00008080EEB082EC3F8BCE194F8023203416E
:10F8000003F00F039E4240D80D2F24DD94F80432FC
:10F81000034103F00F039E4210D90B2B0ED80AB1FF
:10F820009A420BD094F8048294F805E204EB830327
:10F830000CEA08080EEB082EC3F8BCE1102F0AD121
:10F8400094F8063243FA00F000F00F00B04202D202
:10F850000B2840F29380A1B394F8B9318BB394F89C
:10F86000FA311B062DD40AF0F5FAD4F8F03100F580
:10F870007A70A8601BB15A68121A002A1BDB3B4938
:10F880003B4AEB6001200A60E2E60B2BBCD80AB1D0
:10F890009A42B9D094F8028294F803E204EB83030D
:10F8A0000CEA08080EEB082EC3F8BCE1ACE75A6876
:10F8B000121A002AE4DA03F108019B68002BF6D142
:10F8C000DEE70120BDE8F08194F8FA0100063FF57B
:10F8D0002CAF28480C27036028E70AF0BBFA214D1B
:10F8E000254B6A78A3FB00135B0C12B394F8F80164
:10F8F00094F8F921D2B2122A18BF012A08D002F0D6
:10F90000EF02A2F1A202B2FA82F2520902B96A70BF
:10F91000D4F8101294F8082299B18B4247D0591AA2
:10F92000012947D094F8F511A4F81402C4F8103254
:10F93000E7E694F8F82194F8F90100EB022080B290
:10F94000E6E7A4F81402C4F8103294F8F511D8E6EA
:10F9500093427FF4FEAE08E793427FF412AF1CE7B8
:10F96000082B0020200000201F85EB51F82C0020E0
:10F97000240000204401002083DE1B4312B190428A
:10F980003FF469AF94F8062294F8073204EB800044
:10F9900002EA0C0C03EB0C23C0F8BC315BE793428A
:10F9A0007FF407AF11E79A427FF41BAF25E794F885
:10F9B000F511A6E6002AB5D0B4F81462D4F80C12FA
:10F9C0002D4F861B143E01FB06F187FB0176C917FC
:10F9D000A1EBE60104EB820689B2C6F8BC11A1E7EF
:10F9E0006FF0300C0126254806F1FF3800EB480E79
:10F9F00000EB46069EF801E0777810F91860A7EB57
:10FA00000E07981B00FB07F0ACEB060690FBF6F028
:10FA1000704440B2002801DA002662E66428A8BFDC
:10FA2000642006465DE66FF0370C0226DBE76FF0D8
:10FA30003C0C0326D7E76FF0410C0426D3E76FF0A8
:10FA4000440C0526CFE76FF0460C0626CBE76FF097
:10FA5000480C0726C7E79C460826C4E76FF04A0C07
:10FA60000926C0E79C460A26BDE79C460B26BAE756
:10FA70006FF05B0C0C26B6E76766666668360408AE
:10FA8000324B5B68C3F3080370B4B3B9EFF311836F
:10FA90009BB92F4A2F4D1368AC6800BF11688B4289
:10FAA000F9D12D4A15684FF47A7101FB05F2141B48
:10FAB000B4FBF5F401FB034320E0EFF311811023C5
:10FAC00083F31288234C254AA5682368DB0344BFCF
:10FAD000012313601E4B48BFA5681E681368C9B296
:10FAE00081F311881C4A14684FF47A71334401FB86
:10FAF00004F2521BB2FBF4F201FB0323184AD2F8C2
:10FB00002012C2F820325B1A41F288318B420AD9A6
:10FB1000C0B2012382F8F80182F82432002382F86F
:10FB2000F43170BC704792F824320F2BF9D8D118F9
:10FB30000133DBB2C0B2102B81F8F80182F8243215
:10FB4000ECD1012382F8F43170BC704700ED00E085
:10FB5000E489002010E000E0E8890020E08900202E
:10FB6000082B0020036933F8110000EB8000C0105F
:10FB700000F55C7080B27047436993F82320002A37
:10FB800000F0C3802DE9F043714ADC7D127800213A
:10FB9000162A04F0040604F0080583F8231000F088
:10FBA000B680002E40F0BE801DB11A8C42F00102DA
:10FBB0001A8493F80290997993F801C00269DE786B
:10FBC00093F80480DF7909F0070001F00F014FEA94
:10FBD000C11E4CEA002106F03F06187A1180997880
:10FBE00093F80AC0760146EAD106D97856804FEAE2
:10FBF000880848EA911193F805809E7B08F0010877
:10FC000041EA8821918059794EEA5101D18007F06B
:10FC10007F07997993F807E03F0147EA1117597A6E
:10FC20001781400040EADE1001F0030140EA412064
:10FC30005F7BD97A50810CF01F0C587A4FEA8C1CEC
:10FC40004CEA90009081187B93F80AC007F00707F0
:10FC500040EA072006F03F065F7B1082C90041EAB8
:10FC60005C117601D18146EAD7015182D97B93F8A4
:10FC70000E8093F810E093F811C0DE7C9F7C587DD5
:10FC8000890041EA98110EF0010E41EA8E2191821D
:10FC900093F812E0197C0CF00F0C76004FEACC1CA4
:10FCA00046EADE1E4CEA51011E7D93F811C0D18256
:10FCB00007F07F073F01997D47EA1C1706F003060E
:10FCC00093F814C017834EEA46265F7D568314F0DE
:10FCD000010F40F2147300F01F0014BF1E46AD2642
:10FCE000800114F0020F4FEAC10140EA9C0008BFF6
:10FCF000AD2341EA5711002D9083D183168453849C
:10FD00000CBF01200320BDE8F08310467047114965
:10FD10001F8C0C8066B147F002021A8412B29DB9A2
:10FD20004A8046E71A8C4DB942F002021A8440E735
:10FD300045B147F001021A8412B2F1E742F0030222
:10FD40001A8436E73AB2EBE747F003021A84F3E786
:10FD50000D8800201088002038B50C4605460AF0B2
:10FD600079F8E36940F6AC52C31A934205DD0023EB
:10FD700084F822300F2D19D038BD94F82220002AA3
:10FD8000F8D0182AF8D8511CC9B2192984F82210C1
:10FD9000A55410D10A4A1278162A08BF094A4FF012
:10FDA000010184F8231008BF938038BD0123E0616E
:10FDB000257084F82230002384F8233038BD00BF3A
:10FDC0000D88002010880020094BDFED0A6ADFED66
:10FDD0000A7A03EB810191ED8A7AB8EE477AE7EE71
:10FDE000267AFCEEE77A17EE903A98B2704700BF99
:10FDF000082B002001F11F3F00405C44714A92F83B
:10FE0000683233B192F86E320021162B82F86812F4
:10FE100001D00020704792F86D32022BF0B440F20E
:10FE2000CE8002F51B70184402F26E21D32311F824
:10FE3000014F634013F0800F4FEA430318BF83F074
:10FE4000D503DBB213F0800F4FEA430318BF83F0F2
:10FE5000D503DBB213F0800F4FEA430318BF83F0E2
:10FE6000D503DBB213F0800F4FEA430318BF83F0D2
:10FE7000D503DBB213F0800F4FEA430318BF83F0C2
:10FE8000D503DBB213F0800F4FEA430318BF83F0B2
:10FE9000D503DBB213F0800F4FEA430318BF83F0A2
:10FEA000D503DBB213F0800F4FEA430318BF83F092
:10FEB000D5038842DBB2BAD192F88512994202D0BA
:10FEC0000020F0BC704792F8740292F8736292F8C6
:10FED000781292F87C3292F8804292F87052B2F81E
:10FEE00070C2D2F8707200F00F00C00140EA5600F4
:10FEF00001F01F0192F87762C2F83402890141EAE9
:10FF0000960103F03F0392F87B6292F87F02C2F8F9
:10FF100040125B0143EAD60392F86F12C2F84C32EA
:10FF200004F07F04B2F87432D2F87462240105F050
:10FF3000070544EA101041EA0521C3F30A13C2F889
:10FF40005802B2F87852C2F82812B2F87A42D2F8BF
:10FF50007C02B2F87E12C2F83832D2F88032C0F396
:10FF60008A10C1F34A01C3F3CA13CCF3CA0CC7F316
:10FF70008A37C6F3CA366D09C4F30A04C2F85002C0
:10FF8000C2F85412C2F82CC2C2F83072C2F83C62F5
:10FF9000C2F84452C2F84842C2F85C3292F8843245
:10FFA00092F88302B2F88212DB0043EA5013C1F3E5
:10FFB0008A01C2F86432C2F86012012081E7D323BB
:10FFC0007AE700BF082B002070B5044609F042FF15
:10FFD000714AD2F8AC3203F24C4383420BD392F80D
:10FFE000B03243B1022B8ABF92F86D020520023075
:10FFF00098420BDC70BD0121002382F8B012C2F8D8
:020000040801F1
:10000000AC0282F86C4282F8683270BD591CC9B2E9
:1000100088421344D4BF0125002582F8B01283F82A
:100020006C4282F86852E5DC92F86E520023162D7D
:1000300082F8B032DED06B00290648BF83F0D503CA
:10004000DBB213F0800F4FEA430318BF83F0D503F0
:10005000DBB213F0800F4FEA430318BF83F0D503E0
:10006000DBB213F0800F4FEA430318BF83F0D503D0
:10007000DBB213F0800F4FEA430318BF83F0D503C0
:10008000DBB213F0800F4FEA430318BF83F0D503B0
:10009000DBB213F0800F4FEA430318BF83F0D503A0
:1000A000DBB292F86D4213F0800F4FEA430318BFA2
:1000B00083F0D503022CDBB247D938490C44023116
:1000C00011F8016F734013F0800F4FEA430318BF1C
:1000D00083F0D503DBB213F0800F4FEA430318BF60
:1000E00083F0D503DBB213F0800F4FEA430318BF50
:1000F00083F0D503DBB213F0800F4FEA430318BF40
:1001000083F0D503DBB213F0800F4FEA430318BF2F
:1001100083F0D503DBB213F0800F4FEA430318BF1F
:1001200083F0D503DBB213F0800F4FEA430318BF0F
:1001300083F0D503DBB213F0800F4FEA430318BFFF
:1001400083F0D5038C42DBB2BAD1024492F86B2221
:100150009A427FF44FAF7A2D08D07C2D06D0282DFF
:100160007FF448AF0E4B01221A7070BD0D4A136E1A
:10017000572B3FF73FAF0C490C480D684C680821DE
:10018000995413440121C3F80150C3F80540136E7C
:1001900001700933136670BD082B0020742D0020F8
:1001A000A4520020B4520020792D0020A552002036
:1001B00070B54A4E4A4C33782BB1D4F8B4328342EE
:1001C0009CBF00233370474B1B68DA070FD594F8A8
:1001D000B81294F8C052D4F8BC228D42A0EB0203AE
:1001E00033D1002B2BDD012084F8C10270BD9D04AA
:1001F0003DD405463C4883689847C10713D500F0B5
:100200000202002A3949D4F8C43214BF0122002264
:100210000A742B440CBF0121002101223170C4F863
:10022000B43284F8C122D4F8BC32420748BF01225C
:10023000A5EB030348BF84F8E022002BD3DC94F83D
:10024000C13293B994F8E00270BDD4F8C45284F876
:10025000C01205442549C4F8B4520020012283424B
:10026000087484F8C1223270BDDC012070BDB4F87E
:10027000C83223BBB4F8CA320BBBB4F8CC32F3B9E2
:10028000B4F8CE32DBB9B4F8D032C3B9B4F8D23254
:10029000ABB9B4F8D43293B9B4F8D6327BB9B4F868
:1002A000D83263B9B4F8DA324BB9B4F8DC3233B9C6
:1002B000B4F8DE321BB9D4F8BC22831A91E7D4F823
:1002C000C4320A49D4F8BC220344C4F8B43200232F
:1002D0000B740121831A317083E700BF0A4D00209F
:1002E000082B0020409B00201886002020000020C2
:1002F000002070470020704701207047024B03EB3D
:100300004101B1F8E4027047082B0020044B93F838
:10031000080318B1002283F808230120704700BFAA
:10032000082B0020024B03EB8101B1F80C0370474E
:10033000082B002038B5044609F08CFD2E4BD3F86D
:100340004423821AB2F5FA7F14D90022C3F8440379
:1003500083F8482383F84923E1B2042924D02029D3
:1003600022D093F84C230AB9552C35D0A24216D18D
:10037000002209E093F8492392B993F84823C3F87F
:100380004403E1B2002AE8D093F84A039C180138EC
:10039000824284F854131BD0013283F8482338BDBD
:1003A000013A83F8492338BD002202244FF6FF703A
:1003B00083F85043A3F84E039C18481E824283F8EA
:1003C0004C1383F84A1383F84B2384F85413E3D176
:1003D000012283F8742338BD01201F2583F84C4384
:1003E000A3F84E2383F8541383F84B0383F8500388
:1003F00083F84A53D0E700BF082B002003788B42D4
:1004000083BF034B03EB4101B1F878030020704731
:10041000082B002038B5394C054609F01BFDD4F8EF
:10042000CC33C4F8CC03C01AB0F57A7F1CDD0023AE
:10043000282284F8D03384F8D23384F8D33384F874
:10044000D1233D2D42D03E2D0DD12D4AC4F8D423C9
:10045000012384F8D2330123157084F8D03394F843
:10046000D1239A4220D038BD94F8D023002AE8D076
:10047000531CDBB2D4F8D41384F8D033062B8D543C
:10048000EDD194F8D233012B27D094F8D333012B3C
:1004900027D00023282284F8D03384F8D23384F87C
:1004A000D33384F8D12338BD94F8D233012B04BF61
:1004B000022384F8D23394F8D333012B15D00022D1
:1004C000282384F8D02384F8D13338BD0D4AC4F8EA
:1004D000D423012384F8D333BDE78B78282BD4D8D9
:1004E000F1E78B78092BD4D8EDE7022384F8D333D6
:1004F00009F0B0FCC4F8D803E1E700BF082B0020E6
:10050000AC2E0020A02E002030B40246002305258A
:100510001E2400E00232032BD4BF0021012100F889
:1005200013100133042B04D0122B5470F2D130BCC1
:1005300070475570EEE700BF024B03604360836075
:10054000C3607047E803D007024B03EB4101B1F8E9
:10055000C8027047082B0020024B03EB4101B1F8A1
:10056000C8027047082B002030B4264C94F8D233D0
:10057000022B02D0002030BC704794F8A653EDB196
:10058000013D04F2A53353FA85F504F569700022A4
:1005900010F8013B534083EA0313DBB2120AD9007F
:1005A00042EA0322854281EA131382EA0302EFD171
:1005B00022B1002084F8D20330BC7047B4F8A433D1
:1005C0005BBA9BB243F60162934209D043F60362E1
:1005D000934205D0002384F8D233012030BC704709
:1005E000094AA2F12E0102F12005D0799379023255
:1005F00003EB0023C3F3CC03AA4221F8023FF4D15A
:10060000E8E700BF082B0020AC2E002070B540F2B8
:10061000014444EA800409F01DFC0C4E054696F89E
:10062000FC3306EB8303D3F8DC03E3070AD5F9F7C1
:100630000EFA640805F1340507D009F00BFC854279
:10064000FBD8ECE7F9F7FEF9F3E770BD082B0020C3
:100650000D49B1F8FD3330B508224AF2010580EAB0
:10066000030414F0010F4FEA530318BF6B4002F16B
:10067000FF3218BF9BB212F0FF024FEA5000EED1DA
:10068000A1F8FD3330BD00BF082B002008462CF038
:10069000DFB800BF0FB400B583B004AB054953F811
:1006A000042B01930020FAF705F803B05DF804EB82
:1006B00004B070478D0601080EB470B583B007AC66
:1006C0000646482054F8045B2CF0C2F820202CF099
:1006D000BFF830462CF0A8F83A202CF0B9F82A469A
:1006E0002346094901940020F9F7E4FF04460A2053
:1006F0002CF0AEF8054A136803341B1B136003B0DB
:10070000BDE8704003B070478D0601086C8600207C
:100710002DE9F04FDFF820913D49D9F800543D4BC9
:100720002C4685B005F1300B05F1100244F8040B9E
:100730005E46029209F20C4A09F5836809F22447E1
:10074000FAEC016AB8EC017AF7EC017AB1EC010A33
:100750000193FDEEE66AFDEEE77ABDEEC77AE4ECC2
:10076000016AC4ED057A84ED027A0091039132F0BA
:100770009FFC019B0099F3EC017A26F8020BFDEE39
:10078000E77A17EE902AB280029A9442D8D1224991
:1007900005F12803F1EC017AFDEEE77A17EE902AD5
:1007A00023F8022B5B45F5D11C4B1D4A5888117864
:1007B0001A88AA879A88DB88E887A5F84020A5F8D8
:1007C000423071B105F14403164A03EB4101F2ECEA
:1007D000017AFDEEE77A17EE900A23F8020B8B42BE
:1007E000F5D111481149124A124BB9F85A444088C0
:1007F0004968526A1B88A5F85E40A5F86400A5F810
:100800006610AA66A5F86C3005B0BDE8F08F00BF91
:10081000349B00209C4D00200C4D002010880020AF
:10082000F1490020382F00205C4D0020644D00204D
:10083000984A0020AC4E0020082B0020F8B50F4B42
:10084000D3F80054D3F80444D3F80864A9B1831E44
:1008500000EB410727441E4404441D4434F9022B95
:1008600036F9023F35F9020F134403EBD373A0EBC3
:1008700063002CF0A9F8A742F0D1F8BD082B0020A6
:100880002DE9F04F5F4D85B0D5F864440093904654
:1008900000290CBF04230623621C0F9F01936ED016
:1008A0000E9BA34247DDDFF870A157B1109BDA1B06
:1008B00004FB02F20123B95CD5F86C248B4013428F
:1008C00031D0009BD5F860B4A3EB080304FB03F41C
:1008D00008EB0406BBF1000F3AD158F8040031F0E0
:1008E00021F900F1050948462BF052FF002836D1C6
:1008F000DAF8000095F86814A0EB0900CAF80000C7
:10090000002936D1012385F86834BBF1000F2AD1C4
:1009100058F804002BF088FF96F904104B1C02D005
:100920003948FFF7B7FED5F864440E9B01349C426A
:10093000C5F86444B9DB0E9BA3424DD0D5F86004E2
:10094000019B834294BF0020012005B0BDE8F08FD9
:100950004FF0030948462BF01BFF0028C8D00120A8
:1009600005B0BDE8F08F5E4428483179FFF792FE6C
:10097000D9E72C202BF06CFFD5F860B4C5E7D5F88B
:1009800060A49A4503D3002005B0BDE8F08F204B4A
:10099000039103EB8A030646DA690292104631F0AE
:1009A000C1F80B302BF0F4FEDDE9022104460028EB
:1009B000D5D1BAF1030F98BF31461648FFF76AFE4A
:1009C0001549D5F864240B6885F868441B1A541C33
:1009D0000B60C5F8644463E701202BF0D9FE0028C2
:1009E000ACD10D4A13680A20013B13602BF030FF95
:1009F000D5F860044FF0FF330130C5F86004C5F846
:100A000064349DE7082B00202C7704083477040811
:100A1000683604081C7704086C860020F8B5444C3E
:100A2000444D38220021204632F066F9424B95F8B9
:100A30007464B3F85020A283103393E8070095F84C
:100A4000733484F820600C2B04F1080686E8070054
:100A500013D90023A377227F032A17D0227F042AE9
:100A600057D0092A05D8012000FA02F111F4587F65
:100A70003BD1002B59D10020F8BD01229A4012F43D
:100A8000E85FEBD112F0810FF3D0E4E72B492C4B58
:100A9000A277C4E9001307202A4A2B491368487536
:100AA00043F002034FF480711360A1822368204851
:100AB0009847B5F880344FF47A7262627BB1234E66
:100AC00006F16C07B5F88034616A00EE103A3046E2
:100AD000B8EE400A2436FAF76BF9B742F2D195F82E
:100AE0007234A3B1A3770120F8BD1949144BA07744
:100AF000063AC4E90013032A15D8DFE802F002041D
:100B000006120920C8E70A20C6E70B20C4E7012027
:100B1000F8BD104B0A4A236001236260A3770820C6
:100B2000BAE70C20B8E70820B6E7012BA3D090E77E
:100B3000744D0020082B0020C09200204D89000831
:100B40000DD70008944A0020200000208C2F0020A0
:100B50005D890008458900082DE9F04F904CA37885
:100B6000032B18BF032389B04FF0800018BFA37078
:100B700022F0AEFC0746002800F0AB80802122F076
:100B80009DFC7E79874B97F902C053F82620864D4D
:100B90000092B2F5613F14BF002702270023022113
:100BA00085F8F004CDE901171A466046802122F04D
:100BB000D1FA0C3E7D4B032E186040F29080D5F8A0
:100BC000F4347B4A03EB4303A2FB03235B0900F0ED
:100BD000E480402BA8BF4023DBB2764A1370002884
:100BE00077D075497548764AB4F8009091F815B0F9
:100BF000744B076892F800809979E678724C95F802
:100C0000602693F805E064887048A5F85C4619F101
:100C1000FF3918BF4FF00109BBF1000FC7F3C03710
:100C200018BF012718F1000818BF4FF0010811F094
:100C3000FD0F14BF01210021A2F11904069100212A
:100C4000BEEB010EB4FA84F4614BD0F800C0DFF8BB
:100C50008CA16048C5F8F8144FEA541418BF4FF03F
:100C6000010E012A14BFA3464FF0010B761A03F1BF
:100C7000140418BF01261CF0020F03F1840208BF00
:100C80000E46C5F80044C3E9011103F1F404C3E9B9
:100C90000311DAF80030C5F80424C5F8084490F8C8
:100CA00000A00593CCF3800C0A460C460120079661
:100CB000D3B2591E152918D8DFE801F03030303092
:100CC000303030302C1A2420151A4A3E3E3E3A4E1F
:100CD000281A414B00221A7009B0BDE8F08F354B3D
:100CE00040221A707BE7069931B100FA02F10C43F9
:100CF0000133DBB2162B33D80132D9E77146002914
:100D0000F3D1F9E761460029EFD1F5E74146002923
:100D1000EBD1F1E759460029E7D1EDE79A4534BF19
:100D2000002101210029E3D000FA02F10C43DFE7A2
:100D300049460029D9D1DFE7059E02EB4201314443
:100D400011F82E1C003118BF01210029ECD1CFE78A
:100D500039460029C9D1CFE707990029C5D1CBE78A
:100D60001B20C5F86C4419F037FE1B4CD5F86816EB
:100D7000D5F8702685F862060023022020706B608B
:100D80002B81AB81EB812B6085F87836C5F8641632
:100D9000C5F86C2609B0BDE8F08F01231DE700BF40
:100DA000FC5F002090570408082B0020708600206C
:100DB000D34D62107486002044910020409B002097
:100DC0000D880020744B00205C4D0020944A0020C8
:100DD00000300020F149002058810020605100209F
:100DE00008B5084B9B78032B06D0FFF7B5FE064BE2
:100DF000012283F8792608BD802030F0D7FA002838
:100E0000F3D008BDFC5F0020082B00202DE9F04F37
:100E10002DED028B9E4B1B7D012B87B000F0D783FD
:100E2000022B9C4B01931A460CBF0723002382F828
:100E30007A36994B1B78132B00F2278101229749B0
:100E40009A400A4208BF0023954A0199954F81F8BC
:100E50007B360024112323201460C2E90144D460AE
:100E600081F87C4687F85830BC610EF0A3F806AADA
:100E70000125682602F80B4D07F110002B4675215D
:100E80003C757E753D74FBF733FE002840F01881F9
:100E9000854BB8697B6102233B74002800F0AA836C
:100EA0001C2200238271C3710921F8F72FFD7D4BAD
:100EB0001C469869F8F7CBFD4FF480716069FAF72A
:100EC000F3FFA36913B11A689B885383754B1C46C3
:100ED00058696B21F8F7C8FF80216069F8F7C4FFF3
:100EE000A36913B11A689B88138306236F4CDFF83C
:100EF000C8816F4DDFF8C49100936E4F4FF0960E8E
:100F00004FF0100C4FF47A767B68C3F30803002B84
:100F100040F04A81EFF31183002B40F045812168B6
:100F2000AA6800BF23689942F9D1D8F8000006FBEF
:100F300000F39A1AB2FBF0F206FB01217B68C3F3BF
:100F40000803002B40F01081EFF31183002B40F0D9
:100F50000B812368A86800BF22689342F9D1D8F8B2
:100F600000A006FB0AF2101AB0FBFAF006FB03031E
:100F70005B1AB3F57A7FE1D3BEF1010EC4D1494BC0
:100F80009B6913B11A689B885383464B586940F29A
:100F9000E93302E0002B00F015830289013B12F0D7
:100FA000020F9BB2F6D0F523838140F2E93302E0D1
:100FB000002B00F007830289013B12F0010F9BB266
:100FC000F6D08389838940F2E93302E0002B00F0F8
:100FD00008810289013B12F0020F9BB2F6D0FF2379
:100FE000838140F2E93302E0002B00F0FA800289AD
:100FF000013B12F0010F9BB2F6D08389DBB29B4616
:10100000284B986910B1036882881A835B46682B65
:1010100000F0EC83009B013B13F0FF0300937FF48F
:101020006CAF04AC1F4A204B5361022313749069C8
:10103000019B93F87D56002800F01883002D00F0E6
:101040001E83184B1D469869F8F7FCFCF52168696A
:10105000F8F70AFF0123224600216869F8F7D4FE59
:10106000A869F8F7F4FC9DF81030712B00F0528459
:1010700040F22584AC2B00F05084AF2B40F0478425
:101080000923084A82F8503036E00023DCE600BF2E
:10109000109B0020082B00200D88002048800800AD
:1010A000309B0020C092002000300140E4890020E5
:1010B00010E000E000ED00E0E8890020E089002079
:1010C000AC482B4621460DF10E021030FBF710FD07
:1010D0009DF80E3003F07E038DF80E3000283DD1D0
:1010E0009DF80D3003F07E03682B8DF80D3000F075
:1010F000BB83702B00F0B6839E489F4990F8502028
:10110000019CC36C8979C4F88036032A4FF0000330
:1011100080F8551080F8523066D0042A00F08E8393
:10112000092A00F25B820123934013F4587300F004
:101130005582924B8F4D92481968924CE861063A5D
:1011400091482C6041F001016860032A00F27E831F
:10115000DFE812F07A02830271025802682BBFD1D5
:10116000844B83F85050C7E7EFF311808CF312885B
:10117000D5F808A02B68DB0304D50123C9F800309B
:10118000D5F808A02368D9F80020C0B280F31188F0
:10119000D8F80000134406FB00F2A2EB0A02B2FBEF
:1011A000F0F206FB0323E3E6EFF311828CF31288DF
:1011B000A8682B68D90303D50123C9F80030A868B3
:1011C0002368D9F80010D2B282F31188D8F8002031
:1011D000194406FB02F31B1AB3FBF2F306FB0131C1
:1011E000ACE6F8F795FD0BE7644980F852200A68F1
:1011F000614D044642F001020A60EB716349644BA1
:101200002160EA785E48E061062119755E4B6360F3
:10121000AB78002A00F05B83072A00F081835549F0
:1012200091F850300A2B00F0DF8152499FED597A36
:10123000002381F85330012307EE903AF8EEE77A65
:101240004C4C67EE877A013BFCEEE77A84F8573026
:10125000514B84F85620C3ED007A20462368984706
:10126000454B1B780BB184F852304C4C2DF04CFEA2
:101270004B4A494B019F4B491D684B4BB3FBF5F360
:1012800020464FF4FA7640F81C1B9BB24FF47A715B
:10129000B3FBF1F302F12801C7F89826C7F88436AA
:1012A000A8321023C7F89416A7F8886620211426C0
:1012B000A7F89036C7F8A426A7F8A0168022002128
:1012C000A7F89C6687F88A3631F016FD8022002147
:1012D00004F19C0031F010FD002104F58E70802295
:1012E00031F00AFD9FED315ADFED3B5ADFED303A28
:1012F0009FED302ADFED302A9FED303A9FED301A16
:10130000DFED301ADFED306A04F5CE71002307E01F
:101310000133F6EE007A202BE1EC017A00F08B80AD
:1013200007EE903AB8EEE77A27EE057A77EE257A5F
:10133000BDEEE76A16EE102A2032402AE8D8B4EE55
:10134000E57AF1EE10FA40F3BB819FED206A01E0EF
:10135000F0EE477AF4EEC67AF1EE10FA37EEE67A5E
:10136000F6DCB4EEE37AF1EE10FA40F1A6819FEDDF
:10137000186A35E0C0920020109B0020944A00209B
:1013800090C1793D31E40008499D0008CFCD0008A7
:101390002000002000007A44309B0020943100207F
:1013A0009C3604080000F84140420F003C8C4F3E40
:1013B000DB0F49C092E741B99730083C15A82ABE17
:1013C000DB0FC9BFDB0F4940DB0FC940E4CB16413F
:1013D000E4CB16C1E5A6C539DB0FC93FB0EE677A8D
:1013E000B4EEC67AF1EE10FA77EE267AF6D4F4EE81
:1013F000E57AF1EE10FA40F3588171EEE77A27EEC4
:10140000A76AB0EE624AA6EE024A0133202BF0EE44
:10141000430AE4EE060AB7EE007A66EE674A77EE14
:10142000677AB6EE007AE4EEA07A67EE877AE1ECAE
:10143000017A7FF475AF0C2303FB05F305EE903AB8
:10144000F8EE655A5FED1D7A5FED1D0AD14BDFEDB9
:10145000D23A9FEDD24A9FEDD22ADFEDD22A9FEDFC
:10146000D23ADFEDD26AFCEEE55AF0EE601AF8EE01
:10147000655A03F16C0265EEA75A03F1D80EFDEE32
:10148000E57A75EEA00A17EE90CAFDEEE07A0CF14F
:10149000200C17EE907A00212037F7EE004A0EEB71
:1014A0000100C824BCF1400F848000F20C81F4EEEE
:1014B000E35AF1EE10FA40F3BE81B0EE657A9FED8B
:1014C000BC5A9FEDBC6A01E0B0EE677AB4EEC67A12
:1014D000F1EE10FA77EE457AF6DCF4EEC47AF1EE2E
:1014E00010FA40F1A5819FEDB25A9FEDB36A01E079
:1014F000F0EE477AF4EEC67AF1EE10FA37EE857A1E
:10150000F6D4B4EEE17AF1EE10FA40F32E8133EE28
:10151000C77A67EE077AB0EE621AA7EE821A402FFA
:10152000B0EE430AA1EE270A27EE275A9FEDA36AE1
:10153000A5EE007AB0EE641AF0EE647AA7EE061A11
:10154000E7EE467A87EE810A40F2C480B0EE667A12
:10155000B6EE006AB7EE005AC4EE817A0831984EB2
:10156000984D994C9948166018299560D46010617F
:1015700003F1240302F1240203ED050A26EE276A93
:1015800025EE275A67EE277A03ED096A03ED076A0D
:1015900003ED085A43ED067A43ED036A43ED046A0E
:1015A00043ED016A43ED026A42ED086A42ED036AC7
:1015B00042ED046A42ED016A42ED026A7FF46FAFC8
:1015C00001200CE0F8F7A4FB814B5869FAE4814B49
:1015D00001931A46042382F87A362AE4184607B0A3
:1015E000BDEC028BBDE8F08F012381F853309FEDF5
:1015F0007A7A21E61420F8F70DF8B86100283FF454
:1016000053AC4DE4754A19600B211175704A0123E2
:1016100082F852307249CA788B78C979002A40F032
:101620009381002900F07C8169489FED6E7A052145
:1016300080F8531000E6694A19600A211175644A5E
:10164000012382F85230E5E7644A196008211175D8
:101650005F4A012382F85230DCE7604A19600921B1
:1016600011755B4A012382F85230D3E71420F7F753
:10167000D1FF574B9861002D7FF4E3AC18B11C22C9
:1016800000238271C371524B1D4698690921F8F7F6
:101690003DF9A869F8F7DBF904216869FAF704FC59
:1016A000019A012382F87D36CBE4F4EEC17AF1EEA3
:1016B00010FA48BF73EEE77AA1E6F0EE477A96E6B5
:1016C000B0EE677A4DE6B7EE000A402FB0EE401A52
:1016D0003FF63CAFF4EEE15AF1EE10FA40F3EC8045
:1016E000B0EE607A9FED325A9FED326A01E0B0EEC3
:1016F000677AB4EEC67AF1EE10FA77EE457AF6DC48
:10170000F4EEC47AF1EE10FA0FD5B0EE677A9FEDE1
:10171000285A9FED296A01E0B0EE677AB4EEC67AE6
:10172000F1EE10FA77EE857AF6D4F4EEE17AF1EE86
:1017300010FA24DD73EEE77A27EEA76AB0EE625A5C
:10174000A6EE025AF0EE438AE5EE068A27EE868A76
:10175000B8EE007AE8EE287AB6EE006A34EEE75A80
:1017600027EE877A25EE066AF6E6DFED1F7AB4EEFD
:10177000E77AF1EE10FA48BF34EE477AC9E69FEDFA
:101780001A7AF4EEC77AF1EE10FA48BF74EE677A6F
:10179000D2E700BFB0330020DB0F4940DB0F49C068
:1017A00092E741B99730083C15A82ABE0000000016
:1017B000DB0FC940E4CB1641E4CB16C1F304353F3F
:1017C00000DFCD3E00DFCDBEBA32BDBE0184483E53
:1017D000C0920020082B0020D14563442000002047
:1017E000109B00200000FC41DB0FC9BFF8F72AF96D
:1017F0005D4B1D468C21586904ACF8F735FB01237D
:10180000224600216869F8F7FFFAA869F8F71FF97E
:101810009DF81030142BFFF405AC182B03D9543B62
:10182000062B3FF6FFAB504A032382F8503063E4A7
:10183000B0EE677A65E6F0EE657A4EE64A494B4BC4
:101840004B4ACB614B4BC1E900234B4B1A684B49C8
:1018500042F001021A6007220A75434A012382F806
:101860005230D7E604230CE44548062302241946E7
:1018700004AA80F84040A0F11005FBF739F99DF863
:1018800015309DF813209DF81110A34052002240FE
:1018900003F00403134301F001021343F0B1EBB171
:1018A000012B55D0022B29D003F00303032B25D0A5
:1018B000032007F07BFC1FE4F0EE607A20E7122B98
:1018C00022D0702B7FF418AC0523FFF7DABB264833
:1018D0009FED2C7A032180F85310ADE401230DF124
:1018E0000F020C212648FBF703F90028E0D09DF8F1
:1018F0000F3013F00F03DBD0042B2ED01A4A012334
:1019000082F85130FFF7F8BB0823FFF7BABB732BFF
:101910007FF4F2AB0623FFF7B4BB0723FFF7B1BB9D
:10192000114890F850100A2907D00C29CFD1022174
:1019300080F853109FED147A7EE40B489FED137AE4
:10194000042180F8531077E4072A7FF468AC68E636
:10195000002385F85130FFF7CFBB034A002382F8FC
:101960005130FFF7C9BB00BFC092002090C1793D44
:1019700093D9000885CD0008944A0020200000205B
:10198000D09200200000FA4200009C43E438DE427E
:10199000F0B5184E002383B004460821D6F8980904
:1019A00086F8AD3002ADF7F7C3FCD6F8980981216F
:1019B000F7F7BEFC8923D6F8986925F8023DE71DA4
:1019C00014F8010B3246294613F0A4F8BC42F7D1B3
:1019D000BDF806301A0A52FA83F3C3F1FF039BB233
:1019E0003246D8B20021ADF8063013F093F803B0B8
:1019F000F0BD00BF082B002010B5174C08F02AFAE4
:101A0000D4F8A830C31AB3F5FA6FC4BF002384F822
:101A1000AC3094F8AC305BB1104B1B78172B15D061
:101A200000220F49206A12F06DFD94F8AC301BB90A
:101A300000232362012010BD0A48FFF7A9FF0023FD
:101A400084F8AC3000232362012010BDD4F8A82014
:101A5000054B801AD880E3E7082B00200D88002072
:101A6000B42B0020C43704081088002038B50D4C72
:101A700005460146D4F89C09F7F75AFCB4F8A009CA
:101A8000082380EA052041F2210210F4004F4FEABA
:101A9000400018BF5040013B80B2F6D1A4F8A00925
:101AA00038BD00BF082B00202DE9F8438846017897
:101AB000A9B10C4E04468146354606F10807284672
:101AC00031F031F938B1B842A0EB06003CBFA9EBC8
:101AD000040308F8003019F8011F0029EFD1BDE810
:101AE000F88300BF886804082DE9F8432C220446D7
:101AF000002131F001F90123174D184ADFF8648005
:101B00002375292040F26C731549A07513262020F7
:101B1000A261A3830E22022384F82060616284F80C
:101B2000220084F828202372A377C1462E4605F1AF
:101B300008074121304631F0F6F830B1B842A0EB49
:101B400005003CBFA9EB0803235419F8011F002925
:101B5000F0D1BDE8F88300BF88680408DC051A04EA
:101B600075034308387704082DE9F04FE24C94F8E8
:101B700074338BB023B9002318460BB0BDE8F08F47
:101B800094F84B3394F84A030022012B84F8742311
:101B900045D094F85453023D15F0FF0500F0A8819C
:101BA00004F555710D444FF6FF7311F8012B9B1A84
:101BB000A9429BB2F9D11A0A204490F853139142DA
:101BC000D9D190F85223DBB29A42D4D194F84C3355
:101BD000202B40F0868194F850138B1C09938B1DA9
:101BE000019301F10803029301F10A03039301F148
:101BF0000C03049301F10E03059301F11003069306
:101C000001F11603079301F1180301F1040A01F130
:101C1000120801F11407089301F11A0BAFE094F8D0
:101C20005013B4F84EE38B1C671854FA83F60993EB
:101C300001F1040A97F8543397F855C396F85453B2
:101C400096F8557354FA8AF673448A1D96F855E34C
:101C500001921D4496F8543354FA82F605EB0C2594
:101C600001F1080296F855C302922B4496F854539A
:101C700054FA82F603EB072301F10A0254FA82F7C1
:101C80002B4496F85453039203EB0E2301F10C02FC
:101C900097F855E396F8556304921D4497F854332A
:101CA00054FA82F705EB0C2501F10E0254FA82FC7E
:101CB0001D4497F85433059205EB062501F11002F7
:101CC0009CF8546397F855739CF855C306922B44BF
:101CD00054FA82F503EB0E2301F1120895F855E34F
:101CE000334495F8546354FA88F503EB072301F164
:101CF000140795F85593334495F8546354FA87F5CF
:101D000001F1160203EB0C23334495F854C30792F8
:101D100054FA82F603EB0E2301F1180295F855539D
:101D20000892634496F854E396F855C303EB0923ED
:101D300054FA82F6734401F11A0B96F854E396F8BC
:101D4000556303EB052354FA8BF52044734495F84F
:101D500054E390F8539395F8555390F8520303EBDE
:101D60000C239E440EEB062E0EEB052E00EB0929EC
:101D70001FFA8EFE1FFA89F9F1457FF4FCAE9DF83B
:101D8000243054FA83F29DF8043054FA83FC9DF811
:101D900008309CF855939CF854C354FA83F301938C
:101DA0009DF80C3054FA83F69DF8103054FA83F500
:101DB0009DF8143054FA83F09DF8183054FA83F3E8
:101DC000029354FA88F303939DF81C3092F85583DC
:101DD00092F8542354FA83F3214405939DF820305C
:101DE00054FA8AFE54FA87F791F855A391F85413E0
:101DF000049754FA83F39EF8557306939EF854E3C0
:101E0000019B01EB0A2102EB08220EEB072E93F84F
:101E1000558393F85473C4F80C1396F85533019313
:101E20000CEB0921C4F8181395F855C396F85463C0
:101E300095F85453019BC4F8102306EB0326049B2A
:101E4000029AC4F814E393F855E393F8543392F8E4
:101E5000559392F85413039A019603EB0E23C4F89A
:101E60003433059B90F855A3019E90F85403C4F8B1
:101E7000206307EB082701EB092192F8558392F8BC
:101E8000542393F85563C4F82C1354FA8BFB93F83E
:101E90005413069BC4F81C7305EB0C2500EB0A20B9
:101EA00002EB0822C4F82453C4F8280393F85553CE
:101EB0009BF85503C4F8302393F854239BF854330C
:101EC00001EB062103EB0023C4F83813C4F84033B8
:101ED000012302EB05221846C4F83C230BB0BDE8F1
:101EE000F08F064812F05EF8002384F8490343E6B9
:101EF000FF224FF6FF735FE6082B00205C2E0020C8
:101F0000F8B507F0A7FF274E054600F1FA0734465B
:101F100096F8FC3306EB8303D3F8DC03F7F7BEFD3A
:101F200038BB94F8FC3304EB8303D3F8DC03F7F7F6
:101F3000B5FD28B307F08EFFD4F8A839401B9842AE
:101F4000C4F8A4092BD805F5FA7594F8FC3304EB12
:101F50008303D3F8DC03F7F7A1FDB0B994F8FC33A1
:101F600004EB8303D3F8DC03F7F798FD90B100206E
:101F700005E007F06FFFB842CAD94FF0FF30F8BD57
:101F800007F068FFB842CCD9F7E707F063FFA84233
:101F9000DBD9F2E707F05EFFA842DFD9EDE70120C9
:101FA000EDE700BF082B002038B50024054604707B
:101FB000FFF7A6FF431C11D0012803D12B78A040C6
:101FC000184328700134082CF2D1054A2B7892F876
:101FD000AC194B4082F8AC39012038BD0020FCE739
:101FE000082B00202DE9F843204C214D2668074698
:101FF0000236A84695F8FC3305EB8303D3F8DC03DF
:10200000F7F74CFD10BB07F025FF00F1270607F09E
:1020100021FF8642FBD800252C464FF0010998F895
:10202000FC3308EB8303D3F8DC03F7F737FD18B173
:1020300009FA05F31C43A4B2092D06F134060BD0AE
:1020400007F008FF8642FBD80135E8E723689E4287
:10205000D0D80020BDE8F88340F201232340B3F537
:10206000007FF6D164083C700120F3E7E48900208A
:10207000082B002037B502ADFF2305F8013D0446CB
:102080002846FFF7AFFF00B91CB99DF8070003B061
:1020900030BD013CF4E773B5204C002284F8FD23E9
:1020A00084F8FE2384F8AD2984F8AE290144FF2288
:1020B0008DF807200546CEB22846FFF793FFF8B10A
:1020C00015F8010BFEF7C4FAEBB2B342F4D194F861
:1020D000AF39EBB11248FFF785FF88B11148FFF720
:1020E00081FF68B10DF10700FFF77CFF40B1B4F844
:1020F000FD23B4F8AD399A4202D0C2238DF80730DF
:102100009DF80700A0F130035842584102B070BD5D
:102110000DF10700FFF766FFF2E700BF082B002074
:10212000B5340020B634002070B5194C94F8FC3357
:102130000D4604EB8303013D0646EDB2D3F8DC0304
:102140002AF000FD0135002384F8FD3384F8FE33C6
:1021500035443078FEF75AFA16F8010BFEF778FA94
:10216000AE42F6D194F8AF393BB194F8FD03FEF7D7
:102170004DFA94F8FE03FEF749FA94F8FC3304EBA9
:1021800083042021D4F8DC03BDE87040F7F7BEBB20
:10219000082B002013B5FE23ADF8043000238DF882
:1021A000063003788DF80730044613B901238DF803
:1021B000063004210DEB0100FFF7B6FF0220FFF708
:1021C00059FFFF280CD121786068FFF7ADFF282068
:1021D000FFF750FFA0F130035842584102B010BD44
:1021E0000020FBE737B5054608461446FFF7D2FF47
:1021F00078B10123022101A88DF805308DF8045033
:10220000FFF792FF2046FFF735FFA0F13003584259
:10221000584103B030BD07B50E4B0268934317D049
:10222000FF230421ADF8043043788DF8063083781D
:102230008DF807300DEB0100FFF776FF0220FFF766
:1022400019FFA0F130035842584103B05DF804FB78
:102250000120FAE700FFFF0037B5054608460C46A7
:10226000FFF7D9FF60B123788DF80450022101A84F
:102270008DF80530FFF758FF21786068FFF70BFFF6
:1022800003B030BD10B5064CD4F89C09F7F74DF8F3
:102290000028F9D0D4F89C09BDE81040F7F73FB802
:1022A000082B002010B5FFF7EDFF0A4AB2F8B3394A
:1022B00083EA00239BB2082141F2210413F4004F6A
:1022C0004FEA430318BF634001399BB2F6D1A2F82D
:1022D000B33910BD082B002038B50B4B03EBC004FD
:1022E0000D4694F83822094803EB8203D3F86411B1
:1022F00016F09FF894F83E322BB1691C0448BDE8F3
:10230000384016F096B838BD683604081F6E0408C9
:10231000CFA40408F8B50C4C0C4E0D4F04F51C75F9
:10232000206816F0A5F8616811B1304616F081F802
:10233000A16811B1384616F07CF8103416F017F980
:10234000AC42EDD1F8BD00BF60390408166E040838
:102350001C6E04082DE9F04F82468FB091460E4660
:10236000154600273378089373780993F3780A9316
:1023700096F904300B9396F9028096F905300C9388
:10238000B3790D93B8F1000F4AD0B9F1000F4ED0D8
:102390002B78089C6A7895F90210E87895F904C0C2
:1023A00095F905E095F806B09C423ED1099C94420F
:1023B0003BD1884539D10A9C844236D10B9C644577
:1023C00033D10C9C744530D10D9C5C4514BF002466
:1023D0000124CDE90121CDE9030C0093CDE905EB02
:1023E0003B46144A2146504616F0B4F90D9B06931D
:1023F0000C9B05930B9B04930A9B0E4ACDE9028329
:10240000099B0193089B009321463B4650460137A8
:1024100016F0B6F9102F06F1070605F10705A1D150
:102420000FB0BDE8F04F16F0A2B80024D1E74C463B
:10243000DCE700BF226E04087FB5094B0493094B0B
:102440000393094B0293094B0193094B0093094AEB
:10245000094B0A490A4816F02BF907B05DF804FB4E
:10246000836E040817730408886E0408916E0408CC
:102470009D6E04083F6E0408B39100204D6E040861
:10248000586E04082DE9F84316F071F81748184DF6
:1024900016F0A2FD14242D21D5F8B809F7F70FFD89
:1024A000013CF8D116F063F8124D134E134FDFF8CC
:1024B00054802B7EE11006EB830304F00702013108
:1024C0003846D3F8649115F0B4FF6A7E49464AB1A4
:1024D0000B4816F0EDF80134102C05F12005E8D179
:1024E000BDE8F883404616F0E3F8F4E7A36E04086D
:1024F000082B0020C022002068360408B96E0408AA
:10250000CA6E0408347404082DE9F04F324C87B0C9
:102510000746324A2378608802EB8303D3F864814C
:1025200020F09CFCD0E901A304932D4B93F8BC3917
:1025300013B9CDF810A09A4607F04003DFF8ACB00D
:1025400005930025A379002B08BF01239D4206DBDC
:10255000244B08349C42DCD107B0BDE8F08FA3883F
:10256000049A2B440135D65C1AF80330F21AD2F1E2
:10257000000949EB020993B9009543465A4649467A
:10258000384616F0E7F8C6B9059B002BDAD100955E
:1025900043465A464946384616F0F2F8D2E703F069
:1025A0000F021B0940330292CDE900530E4A434605
:1025B0004946384616F0CEF8E5E706F00F0336092F
:1025C00040360293CDE900564346074A494638460D
:1025D00016F0D6F8B6E700BFA0380408683604083D
:1025E000082B002060390408E56E0408D16E040849
:1025F0002DE9F04F674BDA7891B09846002A00F049
:102600009F80654816F0E8FC0025DFF8A0A1DFF800
:10261000B0B10795A94608A9E8B220F043FB9DF8A0
:102620002830002B65D0012D0C9C40F09680002CAA
:1026300000F08A8007EE904ADFED586AF8EEE77AFC
:1026400086EEA77AFDEEC77A17EE906A9AF8BE4931
:10265000089B012C7AD996FBF4F41A4601215048C4
:1026600015F0E7FE0D9A002A00F08B8041F28830C9
:1026700002FB04004FF47A73B0FBF3F00F9B002BC6
:1026800000F0818041F2883103FB04114FF47A7C21
:10269000B1FBFCF1052D03D0079F0F448144079740
:1026A00098F803C0BCF1000F6FD04FF47A7C0E9FF6
:1026B000B7FBFCFCCDF810C04FF00A0C91FBFCFE00
:1026C0000CFB1E11CDE902E190FBFCF10CFB1100AB
:1026D000CDE900102146334815F0EAFF012D08D15D
:1026E0009AF8BE39012B04D9324609992E4815F0C3
:1026F000DFFF0135192D8ED198F80330EBB12B494E
:10270000D1F8C829D1F8C409D1F8CC1952094FF42D
:102710007A73B0FBF3F3264815F0CAFF0798079BBE
:102720000A2293FBF2F302FB130799FBF2F10097E5
:1027300002FB11921F4815F0BBFF11B0BDE8F08FEE
:102740001D4816F049FC5FE726467FE7099A1B48BB
:10275000012115F06EFE344684E75CB107EE904A25
:10276000DFED0E6AF8EEE77A86EEA77AFDEEC77A1D
:1027700017EE904A089A0A48294615F05AFE002694
:1027800070E710467AE7194684E72146584615F067
:102790008FFFA3E7AC910020FB6E0408002474496E
:1027A000506F0408726F0408966F0408082B00200D
:1027B000A66F0408C66F0408466F04085F6F04081C
:1027C000A26F04082DE9F043694B6A48196891B07B
:1027D0004FF47A73B1FBF3F115F06AFF05A8F7F730
:1027E0003FFE58B1644A05A90023B2F9002008A8A9
:1027F000F8F73EF808A9614815F05AFF604B614DA3
:102800001B78614A6149127809886148DFF8E091D4
:1028100005EB830305F27C58D3F8683515F048FFC3
:102820005C4B5D4819685D4BB1FBF3F115F001FE9F
:102830001FF082FF4FF47A72594BB0FBF2F102FBAA
:102840001102B3F900300A2092B289B2B2FBF0F261
:10285000544815F0EEFD544B1F68002405F29C55BA
:1028600058F82410A300C1B10126A6403E4212D060
:10287000F20610D019F804205B594C4853F8222076
:1028800015F0D7FD022E06D1494B93F8211011B156
:10289000484815F0CEFD0134E2E7474C15F067FEDD
:1028A000B4F8D059454A4649464815F001FF464A12
:1028B000464B4748ADB2D31A2946B4F8D22915F091
:1028C000F7FE44490A6D002A42D007EE902ADFED58
:1028D000426AB8EEE77AC6EE877AFDEEE77ACDED8A
:1028E000037AD1F8EC305BB107EE903ADFED3A6A4B
:1028F000F8EEE77A86EEA77AFDEEC77A17EE903A01
:10290000C96959B107EE901ADFED336AF8EEE77A3C
:1029100086EEA77AFDEEC77A17EE901AB4F8D409BE
:102920002E4E2F4F6428CDE900310146039B2D48E0
:10293000A8BF642115F0BCFE2B4815F099FD2B4B68
:102940001C68012534B915F012FE11B0BDE8F08302
:102950000392C6E794FAA4F3B3FA83F305FA03F2F9
:1029600056F82310384624EA020415F062FDE9E720
:10297000E4890020F46F0408185300200E70040846
:10298000724B002068360408624D00205C4D002028
:102990001F700408409D00204570040840420F004D
:1029A000EC5F002055700408944A002076700408FB
:1029B000744D00207E700408082B0020F0FF0120D9
:1029C0000008000082700408008000080040000831
:1029D000A67004084801002000247449F057040838
:1029E00034740408E070040826710408585100206B
:1029F000340000202DE9F84F0024DFF85C90DFF868
:102A00005CB0804625464FF00D0A0AFB049641460D
:102A10003768384630F0C3F978B13946584615F072
:102A200008FD0021304615F097FD15F0A0FD304659
:102A300015F052FE15F09BFD0135013440F23D13B7
:102A40009C42E2D125B90348BDE8F84F16F0C4BA5C
:102A5000BDE8F88F3C710408744404089DA4040880
:102A600038B50C4D0446204615F07AFC30B10A4BBF
:102A70000A485978BDE8384015F01ABE204630F0B3
:102A80001DF8052804D8C0B21FF0A0F92C46EAE7CB
:102A900038BD00BF17730408AC91002049710408C9
:102AA000052810B50C460FD81FF090F9074816F00E
:102AB000C9FD0748FFF7D4FF15F059FD214608204E
:102AC000BDE8104015F058BD10BD00BF5871040896
:102AD0001773040870B50B4E0B4D0446204615F0D5
:102AE0003FFC30B1074B09481978BDE8704015F03C
:102AF000DFBD20462FF0E2FF022802D830702C46BE
:102B0000ECE770BDAC910020177304084D71040808
:102B1000022810B50C460FD805F0D4FB074816F074
:102B200091FD0748FFF7D6FF15F021FD214604204F
:102B3000BDE8104015F020BD10BD00BF5C71040859
:102B40001773040838B5044615F00AFCA0B3244BEB
:102B5000DB690133172B25D822490C2202FB031213
:102B60001C46D2F8B85555B91E4A0C210134172C11
:102B70001ADD002401FB0420D0F8B855ADB1184B84
:102B8000DC6120F07FFD2A462146174815F090FDB4
:102B9000144B0C2202FB043494F8B005BDE8384015
:102BA00020F08ABD1C46DFE7E4D99C42DED10F4805
:102BB000BDE8384016F010BA20462FF07FFF1728E6
:102BC000044607D8074A0C2303FB0023D3F8B85563
:102BD000002DD4D121460648BDE8384015F068BD27
:102BE00020000020683604088E710408647104080F
:102BF000787104082DE9F04F014691B006468548EA
:102C0000854D15F055FD854BC3F800D000232B7082
:102C1000834B40241C70834B0622197830461EF0EB
:102C20006FFA0A200CF0C6F92B78DBB20C2B40F2BD
:102C3000ED809DF80C90B9F1FE0F2ED0B9F1FF0F89
:102C400015BF0F241524002601269C4240F0DE808B
:102C5000611EC9B2684611F0E5F810AB1C4414F8C7
:102C6000413C834240F0CE8006F1FF38B8F1010FBD
:102C70009DF80D4013D904F01F07650961374C46D4
:102C8000694815F0F5FB022E71D0013D042D6AD87C
:102C9000DFE805F00A5D616965000226D5E79DF869
:102CA0000E709DF80F50EBE7604816F095F96048FC
:102CB000DFF8D091DFF8D0B115F0DAFB00254FF046
:102CC000030A1DF805104846013515F0B2FB0C2D1E
:102CD00055D115F04CFC022E5BD06422B4FBF2F10E
:102CE00002FB11423B46D2B2C9B2524815F0E0FC99
:102CF0005FFA88F8B8F1010F7BD84F4A4F4B9DF827
:102D000010104F484F4D00290CBF1146194615F0C1
:102D1000CFFC9DF811104C4B4C4800290CBF2946A4
:102D2000194615F0C5FC022E63D19DF812404848A3
:102D300015F09EFB9CB3FF2C41D00A22B4FBF2F1AC
:102D400002FB1142D2B2434815F0B2FC2AE04248DD
:102D500016F042F9ABE7414816F03EF9A7E74048C4
:102D600016F03AF9A3E73F4816F036F99FE700233B
:102D70000DF11F008DF83F3016F02EF997E795FB07
:102D8000FAF303EB43039D429BD1584615F070FBC9
:102D900097E73A462146344815F08AFCA8E72846CA
:102DA00016F01AF99DF81340304815F061FB54B144
:102DB000FF2C21D021462E4815F07AFC06E02D4844
:102DC00016F00AF9EEE71F4816F006F91D4D1E4EE3
:102DD000284F00240DEB04031A7D8AB1FF2A14BF8B
:102DE00032463A4621462448013415F061FC042C51
:102DF000F0D111B0BDE8F08F1E4816F0EDF8E5E710
:102E00002A46EFE71D4816F0E7F8F2E71C4816F0EF
:102E1000E3F8EEE7C37104080E4A0020004A0020E0
:102E20000F4A0020F1490020D4710408DF71040822
:102E30000D72040824720408AC710408A37104081C
:102E40005B720408B3710408BE750408727204084A
:102E5000797204088D720408E6710408EE710408A2
:102E6000F67104080572040840720408957204089B
:102E700034770408B7710408A5720408B072040816
:102E8000C07204081F72040871A2040838B50D4608
:102E90002FF014FE0C4B19788842044605D20146E7
:102EA0000A48F7F783FD204638BD2DB1FF2803D12E
:102EB0000748F7F77BFDF6E701390648F7F776FD97
:102EC0004FF0FF34EFE700BFF1490020C97204085A
:102ED000DC720408F17204082DE9F341054615F08F
:102EE0003FFA044620B116F07EF802B0BDE8F0814A
:102EF000284601AA2A49DFF8A8802FF018FE2746A5
:102F00000546264675B9022CEDD1A7F57A73B3F5BF
:102F10007A7F1FD94FF4FA624FF47A71214815F085
:102F2000D4FBE2E74CB1012C0FD001AA41460020AE
:102F30002FF0FDFD01340546E4E701212846FFF7A7
:102F4000A5FF431C0646F0D1CFE728462FF0B6FD7B
:102F50000746EAE7B8B217F043F9FF2EBCEEC00A05
:102F6000114B0BD1114AF8EE407A1278AA4212DCCA
:102F700010EE101A0E4815F09BFBB6E7F8EE407AFB
:102F800003EB860310EE102A31460A48C3ED007A9F
:102F900015F08EFBA9E7E3EC017A0135E6E700BF07
:102FA00040A2040893750408E0340020F149002091
:102FB00025730408187304082DE9F347054615F036
:102FC000CFF9044618B9324B9B78042B04D816F07D
:102FD0000AF802B0BDE8F08701AA2E49DFF8B890E0
:102FE000DFF8B8A0DFF8B88028462FF0A0FD012751
:102FF000264610B918F02AFCEBE766B90121FFF765
:1030000045FF431C0446E4D001AA224900200136B2
:103010002FF08DFDEDE72FF051FD2F28054630D81C
:1030200007B318F0E7FB062D08D105200BF0C2FF0F
:10303000FF2C24D0E0B2FFF7DDFD08E001200BF00B
:10304000B9FFEAB298F80010E0B21EF059F829462C
:10305000504615F02DFB052D18DC14200BF0AAFFAF
:103060000027D1E70628E3D0EBE7FFF7C3FD98F888
:103070000030F8B2834207F10107F6D8E7E70027EE
:10308000F5E72F21484615F013FBBDE70027BBE706
:10309000449D002040A204084573040834730408CA
:1030A000F1490020024BD3F8F80928F08FBC00BF8B
:1030B000082B00200A4C08B505460A4815F0D8F937
:1030C000D4F8B809F6F7EEFED4F8F8091FF060FF5F
:1030D00017F0FAF80DB1F8F713FFF8F723FF00BF68
:1030E000082B0020657304080A4D0B4808B516F03C
:1030F000A9FAD5F8B809F6F7D5FE084B002485F8EB
:10310000FC49C5F8FC4A1C7017F01EFA2046FFF770
:10311000D1FF00BF082B002071730408504F00201E
:10312000044808B516F08EFA05F002F90020FFF702
:10313000C1FF00BF98730408034808B516F082FA6F
:103140000120FFF7B7FF00BF9F73040870B5064664
:103150002EF0E8FC124C054690B1112200212046C9
:103160002FF0CAFD2A460F4930462FF0F1FD38B145
:10317000102D2A46314628BF102220462FF0FAFD96
:103180002378074A002B08BF0121064B1CBF0021F2
:1031900013460120044ABDE8704015F0F1BA00BFA3
:1031A000CE5F002071A20408BD7304082DE9F04130
:1031B00088B0804615F0D4F8074608B33E4CDFF8D7
:1031C0000481002519274FF46176237917FB0363E7
:1031D0000493E37817FB03630393A3780293637864
:1031E000019314F8053B009342462B460021012031
:1031F000013515F0C5FA0A2DE7D108B0BDE8F08118
:1032000040462FF05BFC092805464FDC8400261859
:1032100008F101008DF81F7015F0AAF8074660B19B
:103220002FF04CFC0D2808D8244B334483F8000BB6
:103230009DF81F3001338DF81F30384615F098F88F
:10324000074670B12FF03AFC431E042B09D81B4BE4
:103250006219134483F8010B9DF81F3001338DF878
:103260001F30384615F084F8074670B12FF026FC61
:10327000431E072B09D8114B2C441C449DF81F30CA
:1032800084F8020B01338DF81F300B4CF11C0DF14B
:103290001F022144384615F078F89DF81F30052BA1
:1032A000ABD0A2190023A3511371A6E70922394616
:1032B000034815F00AFAA0E708360020082B002082
:1032C000DB730408C57304087F2810B5044607D9CA
:1032D00064F07F00C0B2E40929F0BAFA7F2CF7D875
:1032E000E0B2BDE8104029F0B3BA00BF38B5194DBF
:1032F0000446472029F0ACFAD5F86C341B0305D5F9
:10330000D5F804341868201AFFF7DEFF124C207D30
:10331000FFF7DAFFD5F8F8342068C01A29F054FB1B
:10332000D5F8FC346068C01A29F04EFB2089FFF7FD
:10333000CBFFE089FFF7C8FF208AFFF7C5FFD4E97C
:103340000023217D85F80815C5F80025C5F804354A
:1033500038BD00BF082B002054AA0020F0B52A4C2D
:103360002A4D2768D4F8346B294A2A492A48D4F8C8
:1033700070362D781278097890F82000B74285B021
:1033800026DB84F83C5BC4F8383B84F83D0B84F8BA
:103390003E1B84F83F2B01AD532029F059FAD4F895
:1033A000380BFFF791FF94F83C0BFFF78DFF94F873
:1033B0003D1B94F83E2B94F83F3B03932846CDE900
:1033C000011229F04DFA00232360012005B0F0BD61
:1033D000D4F8386B8DF80850B3428DF80B20019368
:1033E0008DF809008DF80A1001AD04F6383204D0CA
:1033F00095E8030082E80300CEE7696853689942C4
:10340000F6D10020E2E700BF082B0020B04E0020DC
:103410006A8600200A4D0020344D00202DE9F04F2F
:103420007A4C23898BB08046002B40F0FF80784B8C
:103430001B88002B00F09A804046FDF769F9D4F80C
:1034400000644920354629F003FA6068FFF73CFF25
:1034500055F8040BFFF738FF28462EF0D1F806F197
:1034600010002EF0CDF8D4F86C34D90300F19F8011
:10347000D4F86C349A0300F19180D4F86C345B0377
:1034800000F1C080032106F1280029F08FFA614B7A
:10349000B6F92E001B8AC01AFFF716FFD4F86C3459
:1034A000DF0400F1A0809D0400F19380180500F175
:1034B0008780190467D4032106F1300029F076FAD9
:1034C000D4F86C34DA0254D49B0261D4B6F9443097
:1034D00007EE903A504BF8EEE77A93ED007A77EEEC
:1034E000C77AFCEEE77A17EE900AFFF7EDFE4B4B3A
:1034F0001B78012B0ED906F1440707EB430706F1B1
:10350000460535F9020BB6F94430C01A29F05CFAC9
:10351000AF42F6D1D4F86C349F0520D4D4F800041F
:103520003F49404B404AC4F80404451A2D1103FB9F
:1035300005F3013382FB0352A2EBE37202EB42027A
:103540009B1AC3EBC30301EB03130122C4F8080465
:10355000C4F8003484F878260BB0BDE8F08FB6F9D3
:103560005E00A0F2DC5029F02FFAD7E7FFF7F6FE55
:1035700062E7032106F1360029F018FAD4F86C341A
:103580009B02A3D504E0B6F86C00FFF79DFE92E71E
:10359000042106F13C0029F009FA97E7306A29F086
:1035A00013FAD4F86C345B037FF56CAF2AE0F06952
:1035B00029F00AFAD4F86C349A037FF55EAFEDE790
:1035C000B06E29F001FAD4F86C3419047FF573AFAA
:1035D000D9E7B6F86600FFF777FED4F86C34180523
:1035E0007FF567AFECE7B6F86430B4F85C06C01A54
:1035F000C0F30D00FFF768FED4F86C349D047FF52E
:1036000055AFE6E7706A29F0DFF93BE7082B0020A9
:10361000FC5F0020449D002048360020F149002036
:1036200014300020B76DDBB656555555D4F86856A2
:10363000D4F86436AB4207D0C14BC4F864561B784B
:10364000093B012B40F2CF81D4F87056D4F86C6658
:10365000B54207D0BA4BC4F86C561B78093B012B16
:1036600040F2B481E389002B40F00981B54B1B88FF
:10367000002B00F00481FFF771FE4046FDF748F88B
:103680005020D4F80094D4F804A429F0E1F8D4F838
:103690000034D4F80824D4F8041412681B680868AD
:1036A0001344A3EB400002AE29F08EF90AF10402A4
:1036B00009F1040130462DF0CDFC30462DF0A0FF7D
:1036C0000AF1100209F1100130462DF0C3FC30461A
:1036D00029F0C6F810250127D4F86C3407FA05F252
:1036E0001A4240F021810135132DF5D109F128024C
:1036F0000AF1280009F13007314632F9023B30F96E
:10370000025B9742A3EB050341F8043BF5D106AAFF
:10371000002552F8043DAD0003F10801EDB233B1CC
:103720000F2903F1800300F2F88045F0010596426D
:10373000EFD14FF0000B284629F08AF85F465A4631
:1037400005F00303022B00F0DE80032B00F0CC8099
:10375000012B00F0BE800137042F4FEA9505EFD111
:10376000002A40F05E81D4F86C3413F4805706D000
:10377000B9F86420BAF86410521A029201279D0425
:103780000AD5B9F86620BAF866000AA901EB8701E4
:10379000121A41F8202C0137180503F400422ED5E7
:1037A000D9F86830DAF868100AA800EB87005B1ACD
:1037B00040F8203C0137002A7FD1012F00F03B81E7
:1037C0007B1E06EB8702002052F8041D4000013BDF
:1037D000C0B209B140F00100591CF5D129F038F808
:1037E000002501E0BD420EDA56F825300135002BE8
:1037F000F8D0D81780EA4300FFF766FDF2E7002A09
:103800005BD1002FD9D103213020FDF717F8D4F870
:103810006C34DD0200F1FE80980200F1F6804A4B24
:1038200044201978FDF70AF8D4F86C34990506D5C8
:10383000B9F95E00BAF95E30C01A29F0C5F8D4F8BB
:1038400000044249424B434A451A2D1103FB05F33C
:10385000013382FB0352A2EBE37202EB42029B1A9A
:10386000C3EBC30301EB0313D4F80424C4F80034FE
:103870000123C4F80404C4F8082484F87836364BCD
:103880001B681A067FF568AE344DD4F8F8342A6800
:103890009A4265D0482028F0DBFF286829F094F888
:1038A000686829F091F8D5E900234046C4F8F82467
:1038B000C4F8FC34FFF71AFD4EE6B9F86C30BAF8DC
:1038C0006C100AAA02EB87025B1A42F8203C01370F
:1038D00073E756F82710002A40F08F804FEA011B4B
:1038E0005FFA8BFB1A4636E756F827000192002A4A
:1038F00054D1C0F3072028F0ABFF16F8270028F0BA
:10390000A7FF019A27E756F827000192002A58D10D
:10391000C0B228F09DFF019A1DE7FF2B94BF45F030
:10392000020545F0030502E7AB0009EB030253442F
:1039300052F8240C53F8243CC01A29F045F8D2E67A
:1039400058810020FC5F0020F14900201430002045
:10395000B76DDBB656555555409B0020A08400201E
:103960006A68D4F8FC349A4294D1B4F90A30E289F6
:1039700003EBD373B2EB630F64D0354B94F8082597
:10398000197D914204D11968D4F8002591424CD098
:103990004046FFF7ABFC0BB0BDE8F08FC0F303303F
:1039A00040EA0B0028F054FF56F82700C0F3071038
:1039B00028F04EFF56F82730019A1B015FFA83FB6F
:1039C000C9E6C0F3031040EA0B00F1E7452028F0F8
:1039D0003FFF1E2028F03CFF2846FFF775FC3046CD
:1039E000FFF772FC3EE6452028F032FF002028F069
:1039F0002FFF2846FFF768FC26E601F00F0141EA99
:103A00000B0028F025FF0022A5E604213C20FCF74E
:103A100015FF04E703213620FCF710FFD4F86C34BF
:103A2000FAE6584628F014FF9DE65A68D4F80435A3
:103A30009A42ADD190E5029BD81780EA4300FFF788
:103A400043FCE0E6A3895B063FF424AF95E700BFA3
:103A500054AA0020194BD3F8F41400221F295A60ED
:103A60001A819A81DA811A6020D03F291AD04FF446
:103A7000FA42B2FBF1F159811148B3F90A200188E9
:103A800029B1914201DD1F2A14DC92FBF1F1198268
:103A900081780C48003118BF01211202C3F8342B81
:103AA000017070474FF400725A81E5E74FF480626D
:103AB0005A81E1E701211982EAE700BF082B0020C3
:103AC000FC5F0020588100202DE9F0418F4C2378C5
:103AD000013B90B006460A2B14D8DFE813F04A00E9
:103AE000E9016C00A100C200DC0000012F019B0174
:103AF000BF01CD0180202DF059FC08B11FF012FB51
:103B0000FDF72AF8824B1B79012B07D0022B02D13B
:103B10002378012B47D010B0BDE8F0817D4D7E4E5B
:103B20007E4B1B78DB072ED53268D5F8641B2378D3
:103B3000914233D8012BEED095F87926002AEAD0AD
:103B40000B2B0DD801229A4040F6030112EA01071F
:103B50000BD112F4C06F03D0093B012B40F2288532
:103B60003368C5F864340B232370002385F8793655
:103B7000D1E76A4B1B78D807BCD4654B1B79012B66
:103B80000FD1644D644E16F07DFE0028CCD0326813
:103B9000237802F59C520832C5F8642B012BBAD168
:103BA00002E0022BB7D15B4D95F87936002BB2D1EC
:103BB000FDF716F9AFE7574D574E28F005FED5F83B
:103BC00064343268643393429CD2402028F0E0FD94
:103BD000002897D1D5F86034514EDFF85C8140273A
:103BE0000EE028F035FED8F80020D5F86034013A10
:103BF0000133013FC8F80020C5F8603400F0D084DC
:103C0000334493F8D0361846002BEAD100214FF008
:103C1000FF320423C5F86014C5F86424237057E00C
:103C200028F0D2FD3F4A0292A2F10C032621019313
:103C30000091A2F10A035021163A4920FCF720FE18
:103C400000287FF45FAF384B1B68190636D5314D1D
:103C50004FF0FF320523C5F86004C5F864242370D3
:103C600036E028F0B1FD314B022000210090A3F195
:103C70000802CDE901114820FCF702FE00287FF47C
:103C800041AF244D4FF0FF320623C5F86004C5F85C
:103C9000642423701CE028F097FD254A0292A2F1CB
:103CA0000C03072101930091A2F108030021143AAB
:103CB0004720FCF7E5FD00287FF424AF154D0021D7
:103CC0004FF0FF320723C5F86014C5F86424237051
:103CD0000F4B1B79012B7FF41EAF0F4E20E728F00E
:103CE00073FD144B052000210090A3F10802CDE9DB
:103CF00001115320FCF7C4FD00287FF403AF054DEC
:103D00000823C5F860042370E2E700BF5881002053
:103D1000FC5F0020082B0020E4890020084D0020D3
:103D2000683604089E3D0408409B0020583F040864
:103D3000743F0408BC3F04086C860020A04D28F0A6
:103D400043FD05F5346393ED000A2FF0B1F905F654
:103D5000443393ED000A06462FF0AAF907464020A7
:103D600028F016FD00287FF4CDAE964AD5F86034D1
:103D700092F801C04A2B00F2F983DFE813F07501D5
:103D80006A016301280222021B0214020D020602CC
:103D9000FF01F801F101EA01E101D701D001C10100
:103DA000BA01B301F003E603DC03D203C803B9038D
:103DB000AA039B03900385037A036F0364035903EB
:103DC0004E0343033B03300327031F0317030F0373
:103DD00007037D0274026B0263025B025202490216
:103DE000410239025B0153011A0113010C01050163
:103DF000FE00F600EE00DB00D400CD00C600BF00E0
:103E0000B800AB00AB01A4019D0196018F018801B0
:103E100082017B011B2016F03BFEB8B1684D2B8957
:103E2000A3B945206F6828F013FD0E2028F010FD7F
:103E30003846FFF749FA3046FFF746FAD5F8343BE3
:103E40002B6030460A232370FFF7E8FAFAF7A0FC4C
:103E50005D4B1B79012B7FF459AE5FE6584D95F809
:103E600062360BB31B2016F013FEE8B995F87936CD
:103E7000D3B909232370E9E7514D544ED5F8643482
:103E80003268C833934220D24F4B9B78032B00F00B
:103E900079834D4B1B790122934222703FF440AE4F
:103EA000022B7FF438AE7FE63046FFF7B7FACDE756
:103EB000464E434D33684649C5F864340322002317
:103EC000C5F860340B60227002E728F09DFC0028E2
:103ED000DAD117E63F4B404993F820203F48FCF7E2
:103EE000EBFBD5F860340133C5F860340AE6394B92
:103EF00039499A7F3A48FCF7DFFBF2E795F8602BE7
:103F000035493848FCF7D8FBEBE795F8532B324995
:103F10003548FCF7D1FBE4E7344B2F495A79344854
:103F2000FCF7CAFBDDE795F873242B493148FCF711
:103F3000C3FBD6E7B5F870349FED2F7A26492F489A
:103F400007EE903AF8EEE77A67EE877AFDEEE77AC9
:103F500017EE902AFCF7B0FBC3E7294A2949538A98
:103F60002948D289FCF7A8FBBBE7254A2549138AD3
:103F700026489289FCF7A0FBB3E7214B16495A79F2
:103F80002348FCF799FBACE71D4B13491A792148EC
:103F9000FCF792FBA5E71A4B0F49DA781E48FCF7AD
:103FA0008BFB9EE795F8492B0B491C48FCF784FBDB
:103FB00097E795F8482B08491948FCF77DFB90E7EF
:103FC000082B0020AC910020FC5F0020E489002039
:103FD0006C8600204491002034770408387B040864
:103FE000247B04080C7B0408FC7A04089C610020F4
:103FF000EC7A0408DC7A04080000C842D07A04088D
:10400000109B002008780408BC7A0408AC7A0408E5
:104010009C7A0408887A04087C7A04086C7A04087C
:10402000707A0408994B9A491B689A485A8DFCF794
:1040300043FB56E7954B96491B6897481A8DFCF74A
:104040003BFB4EE7954B964A96499748FCF734FB65
:1040500047E7964A964B97499748CDE90032974BE8
:10406000974AFCF729FB3CE7964A97499748FCF7A3
:1040700023FB36E7964B86491A689648FCF71CFBEB
:104080002FE7927882499448FCF716FB29E7934B77
:104090007F49DA899248FCF70FFB22E78F4B7C4976
:1040A0001A889048FCF708FB1BE78C4B78499A78F4
:1040B0008D48FCF701FB14E7884B75491A798B484A
:1040C000FCF7FAFA0DE78A4B71491A7A8948FCF72E
:1040D000F3FA06E7864B6E4993F822208648FCF7F0
:1040E000EBFAFEE6854B6A499A788548FCF7E4FAD4
:1040F000F7E6844B66491A688348FCF7DDFAF0E678
:10410000824B9B79012B7FF4ECAE814A8149B2F955
:1041100000308148B2F90220FCF7CEFAE1E6B5F8AA
:104120005C267E497E48FCF7C7FADAE677487D4987
:1041300083784278007800907B48FCF7BDFAD0E69F
:10414000D5F86C34DA0400F141820F23C5F86034ED
:10415000C7E6764B71499A8A7548FCF7ADFAC0E616
:10416000BBB2B2B26B497348FCF7A6FAB9E64FF09E
:104170007E5271497148FCF79FFAB2E6574B4449A9
:104180005A8A6F48FCF798FAABE6544B40491A8AB2
:104190006C48FCF791FAA4E66B4B3D491A886B48D2
:1041A000FCF78AFA9DE6B5F9102039496848FCF712
:1041B00083FA96E6B5F90A2035496648FCF77CFA99
:1041C0008FE6654A40496548FCF776FA89E605A816
:1041D000F6F746F9624B05A9B3F9002008A80023B9
:1041E000F6F746FB08AA38495E48FCF765FA78E618
:1041F000264B27491B685C485A8FFCF75DFA70E62E
:10420000224B23491B6859481A8FFCF755FA68E678
:104210001E4B1F491B68564893F83720FCF74CFA91
:104220005FE61A4B1A491B68524893F83620FCF790
:1042300043FA56E6154B16491B684F489A8EFCF711
:104240003BFA4EE6114B12491B684C485A8EFCF75C
:1042500033FA46E60D4B0E491B68494893F82D206A
:10426000FCF72AFA3DE6094B09491B68454893F8D3
:104270002C20FCF721FA34E6044B05491B68424820
:1042800093F82720FCF718FA2BE600BF60510020B6
:1042900034770408587A0408487A0408886E0408B9
:1042A000916E0408847704088C7704083F6E040834
:1042B0001773040860770408707704089D6E04087B
:1042C0004D6E0408447704081F6E040850770408F4
:1042D0006C830020DC7B0408D07B0408449D002014
:1042E000BC7B0408AC7B0408987B0408847B04082E
:1042F00044910020707B0408547B0408109B00202C
:1043000070780408309B002064780408744B002007
:104310004E7F00200878040854780408C8B40408C4
:104320004C780408307804083C780408744D002068
:104330001C78040810780408F4770408FC77040853
:10434000E8770408DC770408FC5F0020D4770408D1
:10435000C8770408BC770408CE5F0020B077040853
:10436000185300209C7704083C7A04082C7A04082F
:10437000147A0408F8790408E4790408CC7904086C
:10438000B8790408A879040898790408934B9449EB
:104390001B6894489A8CFCF78FF9A2E58F4B9049E3
:1043A0001B6891485A8CFCF787F99AE58B4B8C492E
:1043B0001B688E48DA8BFCF77FF992E5874B8849BA
:1043C0001B688B481A8CFCF777F98AE5834B844984
:1043D0001B68884893F82620FCF76EF981E57F4B2F
:1043E00085491E688548337FF27E767F0096FCF70C
:1043F00063F976E5794B7A491B6881481A7EFCF7A8
:104400005BF96EE5754B7C491E687E48B37D727D15
:10441000F67D0096FCF750F963E5704B76491E680F
:104420007948F37CB27C367D0096FCF745F958E577
:104430006A4B71491E687548337CF27B767C009626
:10444000FCF73AF94DE5654B6B491E687048737B84
:10445000327BB67B0096FCF72FF942E55F4B66494D
:104460001E686C48B37A727AF67A0096FCF724F9E3
:1044700037E55A4B60491E686748F379B279367A56
:104480000096FCF719F92CE5544B5B491E6863480C
:104490003379F27876790096FCF70EF921E54F4BE7
:1044A00055491E685E4873783278B6780096FCF7F6
:1044B00003F916E55B4B50495B4803EB0C1C9CF879
:1044C0000B609CF80A309CF809200096FCF7F4F881
:1044D00007E5544B4849554803EB0C1C9CF8086011
:1044E0009CF807309CF806200096FCF7E5F8F8E405
:1044F0004C4B41494E4803EB0C1C9CF805609CF862
:1045000004309CF803200096FCF7D6F8E9E4454B0C
:104510003349484803EB0C1CBCF80E20FCF7CCF8E0
:10452000DFE4404B2E49444803EB0C1C9CF80C2064
:10453000FCF7C2F8D5E43B4B2949404803EB0C1C7F
:104540009CF80120FCF7B8F8CBE44FEA0C1C354B83
:10455000234913F80C203A48FCF7AEF8C1E495F86B
:10456000BE291F493748FCF7A7F8BAE428F04CF9F0
:1045700000283FF4C7AAD5F8343B2B600A232370E8
:10458000FFF7A6BB304F38681EF0A4FD95F8F03455
:104590000022022B3A607FF47CAC1EF0C9FF78E465
:1045A000334493F8D036002B7FF4ACAAFFF72EBB30
:1045B000452028F04DF9FF2028F04AF9234828F03B
:1045C00033F9384628F044F9FFF7CABA204B21499D
:1045D0001A782148FCF770F883E400BF605100208E
:1045E0003477040884790408747904086879040825
:1045F0005879040844790408C47804083C7904080C
:104600003479040828790408207904081879040802
:10461000107904080879040800790408F47804087B
:10462000EC780408E6800020E4780408DC780408CC
:10463000D0780408B4780408A87804089C780408A2
:10464000947804088078040870860020E87B0408C9
:10465000497F0020C8B40408247804082DE9F04FED
:1046600089B0FCF7D3FB054618B18C4B1868FCF7F2
:10467000D5F98B4B1A785F79012A6DD0022A29D19E
:104680005978884C98782270013949B20229DBBFE9
:10469000854E06EB01110022D1F8682B6260F4F719
:1046A000B9FFA060052F4FD8DFE817F0D90014003C
:1046B000D9005E002500250067791FBB7621617156
:1046C0007A4A7848D021F8F713FA96F8D03B582B5D
:1046D00022D067710924F9F7CFFF0028FBD1F9F741
:1046E000CBFF28B1013CF6D1284609B0BDE8F08FD8
:1046F0001DF080FFF6E76C4E14200AF05BFC237877
:10470000012BD9D00123694A6648D021F8F7F0F986
:1047100096F8D03B582BDDD11823654A6148654E89
:104720008821F8F7E5F93122F4215E48F9F7C0F85D
:1047300061486249624B634A6361C4E90601624BA6
:104740002661E26023620427604A614913688F751D
:1047500043F004031360BDE7D978524C18792270F6
:104760004B1E237160719DE74F4E0DF107070A2024
:104770000AF020FC2378012B78D03A460123A021AF
:104780004848F8F7B5F90028B6D09DF80730FF2B58
:10479000B2D000274348DFF8549101221E218346FE
:1047A000F9F786F84FF42F600AF0AAFB4FF0A00843
:1047B0004FF0000A022302AA41465846ADF808A06D
:1047C00008F10208F8F794F99DF808209DF80930DF
:1047D0005FFA88F843EA0223B8F1B00F29F8023FE4
:1047E000E8D1B6F8CECB00230CF47F4EA6F8CEEB82
:1047F0000CF00F0C1946012021F001023244B2F8EE
:10480000C02B002A18BF002011F0010F1ABFD2B22E
:10481000534083EA1223082213F4004F18BF83F495
:10482000C053013A4FEA4303F6D101311029E3D1D5
:104830004EEA0C0EA6F8CEEB48BBC3F303339C45FF
:1048400025D1244A244B25482549E2602361254A85
:10485000254BC4E90501C4E90723032774E7124E79
:1048600096F8983B002B43D002276DE76279002A27
:1048700083D13A4677276771A0210A48F8F738F9BB
:10488000074638B19DF80730FF2B03D082E7002F91
:104890003FF432AF002363712EE700BF309B00204E
:1048A0009C610020984A0020082B0020D836002068
:1048B000DC3600206188000871D90008D5CC0008DA
:1048C000638800080000D85979860008944A0020BF
:1048D00020000020102710276BD90008C5CC000845
:1048E00065D90008B3CC0008B7840008C63600209C
:1048F00014200AF05FFB2378012B0DF1070700F06D
:1049000095803A460123D0215648F8F7F1F800285F
:104910003FF42DAF9DF8073086F8B33B0322552BAB
:10492000A6F8BC2B7FF423AF3A460123D1214D4892
:10493000F8F7DEF89DF807304A4803F00F011F0929
:1049400002AA162386F8B41BAA2186F8B57BF8F7CD
:10495000CFF89DF808E09DF80C009DF809109DF82F
:104960000D309DF80A709DF80B209DF80EC041EAAD
:104970000E2143EA00239DF80F00A6F89C1B42EA93
:1049800007229DF811109DF81070A6F89E2B40EAA2
:104990000C209DF813209DF812C0A6F8A03B41EA18
:1049A00007219DF815309DF81470A6F8A20B42EA75
:1049B0000C229DF817009DF816C0A6F8A41B43EA28
:1049C00007239DF819109DF81870A6F8A62B40EA49
:1049D0000C209DF81B209DF81AC0A6F8A83B41EAC0
:1049E00007219DF81D309DF81C70A6F8AA0B42EA1D
:1049F0000C2243EA0723A6F8AC1B1B4FA6F8AE2BEC
:104A00001A481B491B4AA6F8B03BDFF86CE0DFF8F8
:104A10006CC0C4F80CE00123C4E90570C4F810C0F0
:104A2000C4E9071286F8983B02278DE66279002ACE
:104A30007FF467AF4FF0770C3A46D021094884F8ED
:104A400005C0F8F755F810B9002363718FE69DF89B
:104A5000073086F8B33B0322552BA6F8BC2BF3D1C5
:104A600062E700BF984A00205DCD000877D90008B2
:104A70001DCD000865880008701778698DD9000879
:104A8000023990ED007AD0ED017AD0ED026A062964
:104A900013D8DFE801F0424D56616A790400B1EEA7
:104AA000676AF1EE666AF1EE477A80ED006AB0EE71
:104AB000467AC0ED017AC0ED026A384B93F8203097
:104AC00053BB374B93ED036A93ED005AD3ED065A6F
:104AD00027EE866AA5EE076AA5EEA66A80ED006A53
:104AE00093ED046A93ED015AD3ED075A27EE866AD7
:104AF000A5EE076AA5EEA66A80ED016A93ED055A58
:104B0000D3ED025A93ED086A67EE857AE5EE877A6F
:104B1000E6EE267AC0ED027A7047B1EE476AC0ED44
:104B2000007AB0EE677A80ED016AF0EE467AC4E76B
:104B3000B1EE477AF1EE677A80ED007AC0ED017A46
:104B4000BBE7B1EE676A80ED017AF0EE477A80ED5F
:104B5000006AB0EE467AB0E7B1EE477AF1EE666AE7
:104B600080ED007AC0ED026AA7E7B0EE476AF1EE89
:104B7000666A80ED017AC0ED007AB0EE677AC0ED2A
:104B8000026AF0EE467A98E7F1EE677AF1EE666A2D
:104B9000C0ED017AC0ED026A8FE700BF200000205F
:104BA000F8360020944B954A596AB2F87034A2F84E
:104BB0008034002900F00D8107EE903AB8EE676A64
:104BC00007EE901AF8EE677A9FED8D7A9FED8D0AC9
:104BD000DFED8D2A9FED8D3A9FED8D1ADFED8D1A59
:104BE0009FED8D2A9FED8D5A26EE276AF0EE400A42
:104BF00026EE076A2DED028BFDEEC67A36EE000A30
:104C000017EE900AFDEEC07A02F2844317EE901A76
:104C10002030203102F59E62F7EE004A402800F273
:104C2000A580B4EEE26AF1EE10FA40F3DC80B0EE5B
:104C3000467ADFED7B5ADFED7B6A01E0B0EE677A02
:104C4000B4EEE67AF1EE10FA77EE657AF6DCF4EE81
:104C5000C37AF1EE10FA40F1BD80DFED715ADFED5D
:104C6000726A01E0F0EE477AF4EEE67AF1EE10FABD
:104C700037EEA57AF6D4B4EEE07AF1EE10FA00F34E
:104C8000A280DFED6A7AB4EEE77AF1EE10FA48BF5F
:104C900033EE477A67EE077AB0EE614AA7EE814AB3
:104CA0004029F0EE423AE7EE843A67EE275ADFED0C
:104CB000606AA5EEA37AB0EE644AF0EE647AA7EEDD
:104CC000264AE7EE667AC7EE843A55D8B4EEE06A33
:104CD000F1EE10FA40F38A80B0EE407ADFED505AE0
:104CE000DFED506A01E0B0EE677AB4EEE67AF1EEFD
:104CF00010FA77EE657AF6DCF4EEC37AF1EE10FA8C
:104D000077D5DFED475ADFED486A01E0F0EE477AEC
:104D1000F4EEE67AF1EE10FA37EEA57AF6D4B4EEB8
:104D2000E07AF1EE10FA51DCDFED407AB4EEE77A8A
:104D3000F1EE10FA48BF33EE477A67EE077AF0EEED
:104D4000616AE7EE816AF0EE428AE7EEA68A67EED4
:104D5000275AB8EE008AA5EEA87AF6EE006A74EE3D
:104D6000C75A27EE087A65EEA66A0BE0F7EE003A1E
:104D70004029B0EE634AA9D9B0EE457AF6EE006A52
:104D8000F7EE005AC4EE847A243343ED053A67EE19
:104D9000A66A67EEA55A27EE877A43ED096A43EDC6
:104DA000076A43ED085A03ED067A03ED035A03ED53
:104DB000045A03ED015A03ED025A9A427FF42EAFD2
:104DC000BDEC028B704732EEC77A63E732EEC77AEA
:104DD000B3E77047B0EE677AB4EEE07AF1EE10FA1E
:104DE0007FF74FAFEFE7F0EE467A30E7F0EE407A2C
:104DF00082E7B0EE677A92E7744D0020082B00201E
:104E000027D4D236DB0FC93FDB0F4940DB0F49C047
:104E100092E741B99730083C15A82ABE000000006F
:104E2000DB0FC940E4CB1641E4CB16C1DB0FC9BF91
:104E3000F304353F254B5B68C3F3080370B4B3B983
:104E4000EFF311839BB9224A224C1368A06800BF7C
:104E500011688B42F9D120490D684FF47A7404FB34
:104E600005F1081AB0FBF5F004FB03031FE0EFF3B4
:104E70001180102383F31288164A18499568136825
:104E8000DB0342BF01230B609568114AC0B216686C
:104E90000B6880F3118810490C684FF47A70334422
:104EA00000FB04F1491BB1FBF4F100FB03130C48B8
:104EB0000C49126882600124022280F8214081F8A6
:104EC000182CC1F8143C70BC704700BF00ED00E026
:104ED000E489002010E000E0E8890020E08900205B
:104EE000344D0020082B0020274B5B68C3F30803D8
:104EF00030B4B3B9EFF311839BB9244A244C13683F
:104F0000A06800BF11688B42F9D1224A14684FF49F
:104F10007A7101FB04F2101AB0FBF4F001FB0303F9
:104F200020E0EFF31181102383F3128818481A4A06
:104F300084680368DB0344BF01231360134B48BF3D
:104F400084681D681368C9B281F31188114A10681A
:104F50004FF47A712B4401FB00F2121BB2FBF0F20A
:104F600001FB03230D490E488A68022403F5B71399
:104F700003F5587302F2DC5280F8184CC0F8143C68
:104F80008A6030BC704700BF00ED00E0E48900207B
:104F900010E000E0E8890020E0890020344D002086
:104FA000082B00202DE9F04F844C854E854FDFF80B
:104FB0006082854DB6F818C0844A8549854BDFF874
:104FC0005492E160C4E90178002085F8190C85B09D
:104FD0000FFA8CF1C5F8C43205F6184002F1240E20
:104FE000D9F8003022F8021F03F59673964540F871
:104FF000043FF5D1DFF82092DFF820A2D9F800E0D5
:10500000754B1EF4805F08BFB6F92410AAF806108D
:1050100003F1640007E08AB2597804312AF81120BC
:10502000053398421AD01A78002AF9D193F802B0C1
:10503000DA789345F4D20BF1FF3101EB810101EBFA
:10504000810101F561710132BBF1000FE3D102EB87
:10505000820202EB820202F56172DDE71EF0080FA8
:105060002DD11EF4804F3CD11EF0010F0EF40053E1
:1050700014D1E3B91EF4004F1DD1737D13B1022387
:1050800085F87A3096F828202178131D8B42A8BF26
:105090000B4685F83C3D05B0BDE8F08F44F6206234
:1050A00062805BB308224D4B22706360E2E744F6F6
:1050B00020636380F6E7012385F87A30E2E7337AEC
:1050C0000C2B20D8DFE813F0AC00AC00680208021B
:1050D000B2022501250166019E01D601AC001F0028
:1050E0002700122344F6206223703D4B62806360E8
:1050F0003C4A3D4BA260C5F8C432B5E70C223B4B9D
:1051000022706360B6E70820F4F766FFD9F800E084
:10511000C4E90178A5E70A224FEA0C13344993FB4E
:10512000F2F3344A6260A3F5B06321619BB20022BE
:1051300021F812300132122AFAD142F6F8202E4913
:105140002E4B608040202270C4E902131EF0C0F98B
:105150000028D8D0B37A717A90F90200284A002B3F
:105160000CBF00230823002918BF43F001034FF0B0
:10517000030C4FF4E131CDE901C30091002340213C
:105180001DF0E8FFC5F89809002800F0B9801D4B14
:105190001A78002A40F0CA821B4A1C491160022278
:1051A0001A70012395F87A2085F8A430002A40F07F
:1051B000A780032385F87A30A2E000BF188600207C
:1051C00044910020F1020108082B00200EB60020B7
:1051D000F9020108A08601006C370020590501087A
:1051E000FD0201080D030108400D030049050108F7
:1051F0002038002065FB000811E80008F9190108B3
:10520000D5EB000817520020E04A00209119010850
:10521000F5020108E4890020409B002010B6002020
:105220004020C5F818421EF053F9824600283FF48A
:105230006AAF4FF0000B85F8F5B10FF0B7FD327A89
:10524000012A03460FD0C0F08B820A2A1DD1D9F85B
:10525000002012F480621CBF80F00102D2B202F082
:10526000010285F8F5210321072285F8161285F839
:105270001C2201214FF4006285F8EC11C5F80C22C4
:105280000C2142F6F82221706280717AA948AA4A5C
:10529000A2600031606018BF01214AB29AF9020091
:1052A00095F8F5C1002B40F01C82BCF1000F40F0D6
:1052B0003B8296F80AC0BCF1000F00F08382012304
:1052C00042F008024FF4E131CDE9013200910023B0
:1052D0009A4A40211DF03EFF994B1860737D227859
:1052E000013BDBB29A4285F808329CBF002385F867
:1052F000083228B195F8F53113B1012385F8C83C7F
:10530000031C18BF0123002B3FF4FDAED9F800E0C9
:10531000A7E6062B4FF00C0240F0B08185F80A3169
:105320002270002385F80021DFF868A285F8D830C4
:10533000212285F8093185F8083185F8FF20814A56
:10534000814B42F6F82140206180C4E901231EF020
:10535000BFF8834600283FF4D6AE0FF027FD717AE0
:105360009BF902C0B37A003118BF01214AB200286C
:1053700000F0DE81002B40F04E8203220291019268
:10538000CDF800A06046714A40211DF0E3FE704B4D
:105390001860B5E70E236F4A23706F4B4FF0000A79
:1053A00044F62061402085F84CA36180C4E90123C4
:1053B0001EF08EF800283FF4A6AEB0F800C0717A57
:1053C00090F90200B37AB1EB0A010CF4825C18BFC9
:1053D0000121BCF5825F4AB200F0DE8185F849A365
:1053E000002B00F0958142F008024FF0010C4FF4C1
:1053F000E1310292CDE9001C5346584A40211DF08C
:10540000A9FE7DE7102041F27C535549554A207092
:105410004FF0000A6380402028236160A26085F875
:10542000D0A385F8D1331EF053F800283FF46BAEBB
:10543000B27A737A4C4990F90200009152450CBF40
:1054400052460822534518BF42F001020321534639
:10545000CDE90112454A40211DF07CFE0121C5F82D
:10546000140DF3F753FFD5F8143DB3EB0A0318BF3F
:10547000012348E73E490A234FEA0C1292FBF3F25C
:105480000023A2F5B06241F823200133102BFAD19A
:10549000384A2370384B41F60B2140206180C4E923
:1054A00001231EF015F800283FF42DAE737A334A1D
:1054B00090F902000092003318BF01230322CDE9C6
:1054C0000123402100232E4A1DF044FE2D4A031CD7
:1054D00018BF0123106016E710232B4A23702B4BB3
:1054E00042F6F82140206180C4E901231DF0F0FF5D
:1054F000824600283FF407AE0FF058FC717A9AF903
:1055000002C0B37A003118BF01214AB2002800F06E
:10551000D580002B40F08D814FF0030E4FF4E13227
:105520000291CDE9002E6046194A40211DF012FE7D
:105530002DE700BF15F6000845F6000881FA0008BF
:10554000B05200202DED000845ED00086DF0000878
:105550001052002025030108691B010835030108CA
:10556000FD0301086905010848E801001504010868
:10557000302D0020C9FD0008FDFD0008A0680600D0
:10558000C9FF0008A0520020BDF20008D1F20008B7
:10559000A1F4000890D00300AD49AE4B63600A202F
:1055A0004FEA0C1292FBF0F201F12400A2F5B06276
:1055B000216192B26061002321F813200133122B84
:1055C000FAD142F6F821A44A237040206180A260FB
:1055D0001DF07EFF824600283FF495AD0FF0E6FBFC
:1055E000737A96F80AC09D499AF902200091002822
:1055F0000CBF01210321002B14BF06230723BCF19C
:10560000000F0CBF4FF0000C4FF0080C43EA0C03E6
:105610008246019102931046914B924A40211DF01F
:1056200099FDBAF1000F3FF46BAEB0E608238E4A45
:1056300023708E4B42F6F82140206180C4E901239B
:105640001DF046FF824600283FF45DAD0FF0AEFB33
:10565000727A9AF902100032034618BF012200B391
:105660004FF0030C4FF4E1330292CDE9003C0846C1
:1056700000237F4A40211DF06DFD88E60023227043
:1056800085F8002185F8D8301B2285F8093185F886
:105690000831052385F8FF2085F80A314FF4E13AF7
:1056A0004DE64FF0010E4FF4E13C02920846CDE981
:1056B00000CE6F4A40211DF04DFD21E6002B00F089
:1056C000898042F008024FF0010E4FF4E13102925E
:1056D0000346CDE9001E6046664A40211DF03AFDB2
:1056E0000EE6BCF1000F4DD1B37A8BB342F0080344
:1056F0004FF4E1310322CDE90012029363465E4A82
:1057000040211DF027FD5D4B18605D4B1860E5E5FD
:105710004FF0010C4FF4E132CDE901C1009240217C
:10572000584A1DF017FDEBE50323C9E5002339E5D1
:10573000002B65D042F0080201210292034601913C
:10574000CDF800A06046504A40211DF003FDD7E58A
:105750004FF0030C4FF4E132CDE901C10092CEE7E6
:105760000222032185F816224FF4806285F81C126C
:10577000C5F80C22072145F2F05285F8ECB12170F2
:10578000628082E54FF4E13342F008020321009386
:10579000CDE901120023B2E785F849A33BBB42F0F3
:1057A00008024FF0030C4FF4E1310292CDE9001CE6
:1057B000344A40211DF0CEFC344A354B10600022A3
:1057C0001A709DE54FF0010C4FF4E132CDE901C1B3
:1057D00000927DE54FF0010E4FF4E1320291CDE9E8
:1057E000002E6046234A40211DF0B4FC88E542F0BB
:1057F00008024FF0030C4FF4E13102925346D5E713
:10580000012202910192CDF800A060461E4A40217B
:105810001DF0A0FC74E542F00802032302920193FC
:10582000CDF800A060460023174A40211DF092FCED
:10583000ADE542F0080203214FF4E133CDE9003138
:105840000292604600230B4A40211DF083FC9EE536
:10585000D437002065FB000879FB0008A086010012
:10586000F837002059FD0008E5F10008FDF10008B7
:1058700071F20008A1F4000881FA0008B05200207B
:1058800010520020350301086DF00008984F0020E9
:10589000704F0020C1B1013910B450FA81F1441E9B
:1058A000002014F8013F434083EA0313DBB2000AEF
:1058B000DA0040EA0320A14282EA131380EA0300DF
:1058C000EFD15DF8044B704708467047F7B50023E9
:1058D000494C4A4E8DF803306023C4F8A839337818
:1058E000152B07460ED0122B0CD0012B0CBF022516
:1058F0008C25FCF705FB002807DA013DF9D10020D3
:1059000003B0F0BD44F62065F3E70A25FCF7F8FA8A
:105910000130F4D0013D15F0FF05F7D1D4F8A429EA
:10592000930803EB5203C4F8A839FCF7E9FA431CC7
:10593000E5D00028F9DC00230DF1030084F8AC3930
:10594000FCF732FB0028DAD09DF803301B2BD6D1B0
:105950000DF10300FCF728FB0028D0D09DF80320B0
:1059600094F83D3D9A42CAD10DF10500FCF71CFBAD
:105970009DF80530012BC2D801A8FCF715FB9DF856
:105980000430002BBBD00DF10300FCF70DFB002809
:10599000B5D09DF803300E2BB1D10DF10300FCF70B
:1059A00003FB0028ABD09DF8032033789A42A6D1A0
:1059B0000DF10300FCF7F8FA0028A0D09DF80330A1
:1059C000002B9CD13D46BDF80430EA1B92B2023B4D
:1059D0009A4209DB0DF10300FCF7E6FA94F8AC09F2
:1059E000B0FA80F040098BE72846FCF7DDFA002882
:1059F00085D00135E7E700BF082B0020ECB500207B
:105A000070B5274C94F83E3D4340064684F83E3D31
:105A1000082594F8FC3304EB8303D3F8DC03F30785
:105A200016D5F4F714F8402009F06AFA94F8FC331C
:105A300004EB8303D3F8DC03F4F704F8402009F007
:105A40005FFA013D15F0FF054FEA5606E1D170BD42
:105A5000F3F7FDFF202009F053FA94F8FC3304EB30
:105A60008303D3F8DC03F3F7EDFF202009F048FAB5
:105A700094F8FC3304EB8303D3F8DC03F3F7E7FF7C
:105A8000202009F03DFA94F8FC3304EB8303D3F8AB
:105A9000DC03F3F7D7FF202009F032FAD1E700BF8B
:105AA000082B002010B50D4C94F83E0DFFF7A8FF11
:105AB00094F8FC3304EB8303D3F8DC03F3F7C7FF5C
:105AC000202009F01DFA94F8FC3304EB8304202114
:105AD000D4F8DC03BDE81040F3F718BF082B002012
:105AE00010B5104C94F8FC3304EB8303D3F8DC03BB
:105AF00027F028F8FF20FFF783FFFF20FFF780FF44
:105B00007F20FFF77DFF00231B2084F83E3DFFF739
:105B100077FF94F83D0D0130C0B284F83D0DBDE82B
:105B200010406DE7082B00200B4B10B501241C70B2
:105B3000FFF7D6FF0020FFF763FF2046FFF760FF67
:105B40000E20FFF75DFF2046FFF75AFFFFF7AAFF81
:105B50000248BDE81040B9E6ECB50020EDB50020E4
:105B6000F8B504780546002C3DD004F10A0600275C
:105B7000FFF7B6FF300AFFF743FFF0B2FFF740FF31
:105B80000E20FFF73DFF1A4B1878FFF739FF384614
:105B9000FFF736FF2046FFF733FF0020FFF730FF07
:105BA0000020FFF72DFF0020FFF72AFF0020FFF75E
:105BB00027FF0020FFF724FF0020FFF721FF002030
:105BC000FFF71EFF6B681878FFF71AFF6B68013C40
:105BD000013314F0FF046B60F4D1FFF763FF054855
:105BE000BDE8F84072E64FF485760127C0E700BFB4
:105BF000ECB50020EDB5002038B505460478FFF778
:105C00006FFF0020FFF7FCFE0420FFF7F9FE0E20D7
:105C1000FFF7F6FE0A4BB4FA84F418786409FFF72C
:105C2000EFFE2046FFF7ECFE2878FFF7E9FEA02004
:105C3000FFF7E6FEFFF736FF6868BDE8384045E647
:105C4000ECB5002038B5154B02689343044622D0CA
:105C5000134B06251D70FFF743FF0020FFF7D0FE12
:105C60000520FFF7CDFE0E20FFF7CAFE2846FFF7FE
:105C7000C7FE0020FFF7C4FE0020FFF7C1FE6078DA
:105C8000FFF7BEFEA078FFF7BBFEFFF70BFF05484E
:105C9000BDE838401AE6012038BD00BF00FFFF0014
:105CA000ECB50020EDB500202DE9F04FAE4CDFF84B
:105CB000C482C4F89C09D1B01DF0E4FC08F11409B9
:105CC000002584F8B35984F8B459FCF7EBFA2F286F
:105CD000F7D101210020F3F7C7FEADF80850FCF71B
:105CE000E1FA0190FCF7DEFA8DF81500FCF7DAFA1C
:105CF0008DF81600FCF7D6FA0027064610ADFCF723
:105D0000D1FAE8550137FBB29E42F8D1FCF7BAFA56
:105D10008DF80D00FCF7B6FA8DF80C00BDF80C708C
:105D2000B4F8B33901219F4214BF03270027002094
:105D3000F3F79AFE002F40F08880019B0695303BD8
:105D4000102B00F23682DFE813F068009300D702D0
:105D500097001100AC003402D500A701DD01050257
:105D60004D0234022B027802A000AD02012602ADE2
:105D7000B2460021084684F8A01984F8A119F3F767
:105D800073FED4F89C09F3F79CFA2E20FBF76EFE05
:105D90000198FBF76BFE9DF81500FBF767FE9DF879
:105DA0001600FBF763FE50460AF1FF3A5FFA8AFAE3
:105DB000FBF75CFE0AF1010AAA44D4F89C09F3F748
:105DC000B1FA0028F9D015F8010BFBF74FFE554545
:105DD000F3D13846FBF74AFE94F8A119D4F89C0990
:105DE000F3F7A6FA94F8A019D4F89C09F3F7A0FAEF
:105DF000D4F89C09F3F760FA00210846F3F734FE63
:105E0000002E3FF45DAF94F8403D002B40F07F82C0
:105E100015F01CFD51B0BDE8F08F94F8AF39A3B177
:105E200094F83F3D013B032B18D8DFE803F0020252
:105E30001302FD2302210AA8ADF82830FCF774F9FB
:105E40000120FCF717F9C12808D1002602AD4FF058
:105E5000010A8EE7FFF768FE0028F6D1002684F8D5
:105E6000AF6984F8B06902AD4FF0010A0F2780E7EF
:105E70006B238DF80830E8E74FF43273ADF8083043
:105E8000002602AD4FF0020A73E72B785A1E032A50
:105E900000F2378284F83F3D002602AD4FF0010A40
:105EA00067E72B7894F8402D9A4205D8002602AD7A
:105EB0004FF0010A08275CE784F8FC3394F83F3D73
:105EC000042B0ED8012202FA03F313F0160F08D0A8
:105ED000002302210AA8ADF8283084F8AF29FCF786
:105EE00023F9002684F8AF6984F8B06902AD4FF059
:105EF000010A3EE72B7894F8402D84F8AF799A4256
:105F000084F8B079D2D984F8FC33032694F83F3D65
:105F1000042B31D0FFF708FE70B3012113482BF09A
:105F2000EFFB48B3022112482BF0EAFB20B3B4F890
:105F3000AF3949F2073223F00801914207D049F204
:105F40000A32934203D049F20B42934214D1032305
:105F500084F83F3D94F83F3D84F8B2390026044D63
:105F60004FF0040A05E700BF082B0020B8340020DA
:105F7000B7340020DC3F0408B8F8002098F802305D
:105F8000ADF81020BB4A8DF812300AAB106851688A
:105F90001D4603C508324A452B46F7D1D9F8000003
:105FA00099F80420286015210AA82A71FCF7BCF88A
:105FB000082107A8FCF76FF800285FD09DF8102093
:105FC0009DF81C309A4259D19DF811209DF81D3042
:105FD0009A4253D19DF81E209DF812309A424DD11D
:105FE0009DF81F3084F8B1399DF8203084F8B0391D
:105FF0009DF8213084F8AF39B4F8AF394FF2103240
:1060000023F02001914211D04FF2104293420DD063
:106010004FF29032934209D04FF65002934205D08E
:1060200003F5BA520F3292B2012A03D8012384F841
:106030003F3D8FE723F0080249F207318A4207D03B
:1060400049F20A32934203D049F20B42934203D100
:10605000022384F83F3D7DE741F60672934209D062
:1060600043F20632934205D023F4807343F2064292
:10607000934203D1042384F83F3D6BE7013E16F0C1
:10608000FF067FF443AF84F8AF6984F8B0697A4DB6
:106090004FF0040A0F276CE694F83F3D032B40F0C5
:1060A0008880764B12251D70FFF71AFD0020FFF740
:1060B000A7FC0720FFF7A4FC0E20FFF7A1FC284651
:1060C000FFF79EFC1420FFF79BFC0020FFF798FCD5
:1060D000AC20FFF795FC8820FFF792FC1320FFF718
:1060E0008FFC7620FFF78CFCFFF7DCFC6448FFF7A1
:1060F000EDFB00287FF4A9AE002602AD4FF0010AA7
:106100000F2736E694F83F2D012A01D0042A50D1FA
:106110002B788DF80830042A0CBF9B005B00DBB2A3
:106120008DF8153005A800238DF81630FCF773F8AC
:106130000028E1D04FF4817302210AA8ADF828307D
:10614000FBF7F2FF4FF42F70FBF794FF30283FF47A
:106150007CAED1E72B788DF8143094F83F3D5A1E71
:10616000032A26D8DFE802F002020F02022B05A95B
:106170000CBF07200320FCF76FF80028BCD09DF867
:1061800014A00026F5E505A8FFF75CFD0028B3D0B4
:1061900014223A4B0DEB02001A70FFF72DFDECE7CD
:1061A0002B788DF8143094F83F3D022B07D0032B49
:1061B0000AD0002602AD4FF0010A0227D9E505A951
:1061C0000420FCF749F8D8E705A8FFF73BFD0028B5
:1061D00092D02A4B162205A81A70FFF70DFD002851
:1061E000CDD189E794F83F3D8DF81460013B032B36
:1061F0003FF62BAEDFE803F00202110205A8FCF720
:106200000AF800283FF478AFFA2205A90120FBF72D
:10621000E9FF00287FF419AE6EE705A8FFF712FD2D
:1062200000283FF469AF154B132205A81A70FFF739
:1062300097FC00287FF409AE5EE794F83F3D8DF8A7
:106240001460022B05D0032B1CD0012B7FF454AF1C
:10625000AFE705A8FBF7DFFF00283FF44DAF40F2A2
:10626000DC5205A90520FBF7BDFF00287FF4EDAD4A
:1062700042E700BFE03F0408B7340020ECB500203F
:10628000EDB5002005A8FFF7DDFC00283FF434AF92
:10629000294B152205A81A70FFF762FC00287FF42D
:1062A000D4AD29E794F83FBDBBF1040F81D105A817
:1062B0008DF81460FBF7AFFF00283FF41DAF05A871
:1062C000FBF768FF00283FF417AF4FF482730221F9
:1062D0000AA8ADF82830FBF727FF1420FBF7CAFE09
:1062E00030283FF4B2ADC0287FF406AF002602ADDF
:1062F0004FF0010A5F463CE50026104D4FF0090AB9
:1063000037E5002602AD4FF0010A092731E5013BD0
:10631000DBB284F8403D04EB8303D3F8DC0310B117
:106320000221F3F7DDF894F8403D04EB8303D3F842
:10633000DC03F3F787FB66E5ECB50020E1730408A6
:1063400038B5054612F00CF8044628B9062207496C
:106350002846F4F7DBF840B9054813F073F902F06A
:1063600087F814B10020FCF7DBFE38BDF275040895
:10637000EB7304082DE9F047214FDFF8A480DFF824
:106380008490DFF8A0A0054628462BF0CBFB0646FC
:1063900060B91C4B1C4893F860261C4B03EB82032E
:1063A000BDE8F047D3F88C1912F082B9024639469D
:1063B0002846F4F7ABF878B91548164C164D12F08C
:1063C00057F854F8041F19B1284612F032F8F8E7CC
:1063D000BDE8F04712F0CBB8002458F8241021B9DA
:1063E0000E48BDE8F04712F0F7BD32462846F4F7F4
:1063F0008DF801340028F0D189F860465546C3E78E
:106400004B6F0408082B0020017404086836040848
:106410000B740408F43F0408347404083C71040845
:10642000F83F0408177304082DE9F347054611F0F7
:1064300097FF044610B112F0D6FD22E0284601AACB
:106440002749DFF8A880DFF8A890DFF8A8A02CF093
:106450006EFB2646054627463DB9224B3246A1B281
:10646000D3F8F80925F06AFC0BE06FB1012FE2D1F7
:10647000B31E594259412846FCF708FD421C044608
:1064800022D102B0BDE8F08728462BF04BFB4146F5
:10649000064602462846F4F739F8A0B13246494686
:1064A0002846F4F733F8B8B1324651462846F4F797
:1064B0002DF898B132460C492846F4F727F8002801
:1064C000B9D1032600E03E4601AA054900202CF080
:1064D0002EFB01370546BFE70126F5E70226F3E765
:1064E00040A20408082B00201F7404081674040836
:1064F000197404081C7404082DE9F74F80462BF02A
:1065000011FB4A4E0446D6F8447DE8B94848494D47
:10651000DFF8448111F08DFF0C2620461DF0A0F815
:10652000384205D006FB04534046996811F081FFBC
:106530000134162CF1D117B93F4811F099FF03B07F
:10654000BDE8F04F12F013B802463C49DFF8E49082
:106550004046F3F7DBFF054678B9394811F088FF6C
:106560002C46384D09EB0403284699680C3411F089
:1065700060FFB4F5907FF5D1E1E798F800302D2B5E
:1065800003BF08F1010804F1FF344FF0010A4FF096
:10659000000A00250C2303FB05924046D2F808B000
:1065A000019322465946F3F7B1FF019BA0BBBAF114
:1065B000000F1CD0162D0CD1234BC6F8443D2348A8
:1065C00011F056FF1F48594603B0BDE8F04F12F0D6
:1065D0006FB8172D04D1D6F8483DC6F8443DEEE714
:1065E00028461DF03DF83843C6F8440DE7E7162D60
:1065F00005D1C6F844AD164811F03AFFE2E7172D71
:1066000002D1C6F8487DF6E728461DF029F827EAAA
:106610000000C6F8440DEEE70135182DBBD10D483A
:1066200003B0BDE8F04F12F0D7BC00BF082B00202C
:1066300022740408183C04082C7404084B6F0408E6
:106640000B74040834740408FFFF3F003874040816
:10665000417404083C710408337404082DE9F84FB0
:1066600005462BF05FFA374F0446D7F80090B0B9D3
:106670003548364D364F11F0FBFE012655F82410F3
:1066800049B106FA04F313EA090F02D0384611F0B3
:10669000D0FE0134F2E7BDE8F84F11F068BF0246C2
:1066A0002C492846F3F732FF78B92B482B4C2C4D58
:1066B00011F0DEFE54F8041F0029ECD00B78002BFB
:1066C000F8D0284611F0B5FEF4E72B78DFF87CB05F
:1066D0002D2B03BF013504F1FF344FF0010A4FF0B9
:1066E000000A00265BF82680B8F1000F04D11D488F
:1066F000BDE8F84F12F070BC224641462846F3F739
:1067000005FFE8B90120B040830504D51648BDE86F
:10671000F84F12F061BCBAF1000F0AD0F3F75CFC3D
:10672000124811F0A5FE41460D48BDE8F84F11F0A2
:10673000BFBF40EA090038600D4811F099FEF2E74A
:106740000136CFE76C8300204974040864400408D4
:10675000537404084B6F04080B7404086040040869
:10676000347404083C71040857740408387404082D
:10677000417404082DE9F0478AB005462BF0D2F9A0
:10678000024630B992490120FBF7E4FD0AB0BDE8AA
:10679000F08705228F492846F3F7B8FE0446B8B9BA
:1067A0008D4D0146702205F555602CF0A5FAC5F80F
:1067B000C04DC5F8CC4DC5F8D84DC5F8E44DC5F869
:1067C000F04DC5F8FC4DC5F8084EC5F8144EDDE790
:1067D000042282492846F3F799FE044620BB284646
:1067E00011F0C6FD07460028D0D02BF09BF9DFF84A
:1067F0001482064658F824501DB9794812F0ECFB73
:10680000C4E7324629463846F3F780FE50B92046A1
:1068100012F040FF2946734811F04AFF7248FFF713
:10682000A9FFB3E70134E5E7072270492846F3F7EB
:106830006DFE044600287BD1202128462CF073FAF7
:1068400006462BF06FF9054680BB694811F0F1FD53
:106850002C46684D21462846013411F0EAFD0E2CE5
:10686000F8D111F084FE644EDFF89C91634FDFF89D
:106870009C8100242146484611F0DBFDDFF890A101
:10688000002532680123AB40134214BF394641460C
:106890005046013511F0CDFD0E2DF2D1013411F02D
:1068A00066FE082C06F10C06E4D16FE7304601AA1B
:1068B0005349534E2CF03BF902AD002843D0022C33
:1068C00018D1029B072B30D803990D292DD80278B7
:1068D000722A1AD06E2A28D13F4A0C2000FB0323CB
:1068E000012202FA01F1D3F8C02D22EA0102C3F815
:1068F000C02D16E02CF0E2F801AA45F8240031463C
:1069000000202CF014F90134D7E7334A0C2000FBA7
:106910000323012000FA01F1D3F8C00D0843C3F8A6
:10692000C00D3248FFF726FF30E712F05CFBF8E7B6
:10693000284601AA3249324E2CF0F9F8002402AD63
:1069400078B1082C02D112F04EFB1FE72CF0B6F8FC
:1069500001AA45F82400314600202CF0E8F8013463
:10696000EEE7082CEFD1029B0F2BECD8DDF80CC022
:10697000BCF1070FE7D8049F0D2FE4D8059E06F160
:106980006402C82ADFD8069DFF2DDCD8079864284A
:10699000D9D808996429D6D88842D4DA099C032C1E
:1069A000D1D8C3EBC3020C4B134483F8540D83F8C6
:1069B00050CD83F8517D83F8526D83F8535D83F891
:1069C000551D83F8564D0848FFF7D4FEDEE600BF9C
:1069D0005838002063740408082B002069740408E8
:1069E0003C7104086E740408177304087874040872
:1069F000206E040880740408C83800201FA504080D
:106A000040A20408F83F040834770408BF7504085E
:106A1000857404082DE9F04F87B004462BF082F806
:106A2000064628B94120FBF76FFD07B0BDE8F08F9F
:106A3000024689492046F3F769FD002836D1874888
:106A4000874D12F0C9FA14242D21D5F8B809F3F7AF
:106A500036FA013CF8D1834C834E844FDFF83C82F8
:106A600011F085FD04F5C4752168A379A28801F1B0
:106A70003F4106EB830301F57E01B2FA82F2890AF7
:106A80004131D3F86431C2F11F02384611F0D1FC14
:106A9000E17911B1404611F0CCFC083411F067FDEA
:106AA000A542E1D1724812F097FABEE7204605AA46
:106AB0007049DFF8B4812CF03AF808F50E77824679
:106AC0000024B94617F8343008EB83033246D3F874
:106AD00064115046E500F3F719FD30B10134182C6C
:106AE000F0D1654812F078FA9FE705AA61492CF0C9
:106AF0001EF8A84407462BF0E1FF98F83E22064610
:106B0000002A40F09580002800F39B80A944B9F842
:106B100002001CF0A3F93D78002D00F08680F3B24E
:106B2000B9F80460D0F804805449019338461E44F3
:106B3000F3F710FD50B908F8060018F80670B7B959
:106B40004F4812F049FA70E7012275E0602D8CBFC2
:106B5000613D413D072D68D8781C2BF0AFFF0F2811
:106B600063D8013540EA051508F80650E5E73846D0
:106B7000F2F750FD8146002857D03B09403302937D
:106B8000DFF81C8107F00F030026039300252EE099
:106B9000B8F802001CF062F9B8F8043042682B44DF
:106BA000D15CB94222D1B44204D101998D421DD0A9
:106BB0000021D154DDE9021232485FFA85FB5FFA09
:106BC00086FA11F036FC59465046FBF785FBB44275
:106BD00009D12D4811F02DFC50465946FBF77CFB9E
:106BE0002A4811F026FC2A4812F0F6F9013598F8E7
:106BF0000630002B08BF01239D42C9DB0136182E49
:106C000008F10808C2D1D9F80010B9F804202148C9
:106C100001F13F4101F57E01B2FA82F2890AC2F127
:106C20001F02413111F044FDFFE612F0DCF9FCE6F1
:106C3000002801DDB24206DA0121174811F045FDB6
:106C4000F3E6012880D105AA0A4900202BF06FFF46
:106C5000013E07465AE700BF4B6F04088B740408D7
:106C6000082B00202488002068360408C974040812
:106C7000D474040840A2040806750408E06E0408F1
:106C80000E75040820750408447504084775040847
:106C9000B0A9040851750408DB730408CFA40408E4
:106CA000A03804082DE9F74F81462AF03BFF05463E
:106CB00028B1012822D199F800302A2B1ED1724820
:106CC000DFF8DC81714F12F087F900244FF00D09D5
:106CD00009FB04863846316811F0ABFB291C18BF4C
:106CE0000121304611F038FC013411F040FC40F233
:106CF0003D139C42ECD103B0BDE8F08F3D214846E6
:106D00002CF011F8002800F0B880074617F8013C75
:106D1000202B07F1FF3248D0A7EB090701300646C8
:106D200001303378202BFAD0DFF874A14FF000083F
:106D3000D346FFB20D2303FB08A52C6820462AF09A
:106D4000F1FE2146024601904846F3F7DFFB044678
:106D5000002840F08580019BBB4240F081802B7968
:106D600003F03003102B22D0202B4DD06BBB3046CC
:106D70002BF0A4FEB5F9053001B28B4225DCB5F944
:106D800007308B4221DB284611F044FB0D2303FB27
:106D900008B83F48D8F8001011F04BFB00212846F6
